:020000040800F2
:1000000000A0002035230108A597000879140108F5
:10001000A3970008A19700089F9700080000000020
:100020000000000000000000000000009D97000894
:100030009B970008000000009997000849B100084C
:100040009D2301089D2301089D2301089D2301088C
:100050009D2301089D2301089D2301089D2301087C
:100060009D2301089D2301089D2301089D2301086C
:100070009D23010821D70008BDE100089D23010848
:100080009D2301089D2301089D2301089D2301084C
:10009000D58F00089D2301089D2301089D23010899
:1000A0009D230108D1DF000877DF0008F5DF000895
:1000B000C5DF0008B5DF0008A5DF00089D230108A3
:1000C0009D2301089D2301089D2301089D2301080C
:1000D0009D230108B5E10008ADE100089D2301085A
:1000E00059B100089D230108B50C01089D230108A2
:1000F00085DF00089D23010895DF00089D23010886
:100100000000000000000000000000009D23010826
:100110009D2301089D2301089D2301089D230108BB
:100120009D2301089D2301089D2301089D230108AB
:100130009D2301089D23010800000000000000002D
:100140009D2301089D2301089D2301080000000054
:10015000000000000000000000000000000000009F
:1001600000000000000000009D2301089D230108FD
:100170009D230108000000000000000000000000B6
:08018000000000009D230108AE
:100188002DE9F04F2DED028B754E764B3360AFB0F5
:10019800002373600FF052F818B90FF071F806F0E9
:1001A800DFFF07F097F8704B704C1A7842F00102A5
:1001B8001A706F4A4FF47001C2F888100022099231
:1001C8000A92226842F4803222600493236803F47E
:1001D80000330A93099B013309930A9B1BB9099BB6
:1001E800B3F5A04FF2D1236813F4003318BF0123ED
:1001F8000A930A9B012B00F089805D4F5D4BFB60E1
:10020800636AB360636ADFF8A4B1DFF8A481DFF83A
:10021800A49143F080736362636943F4FC032EADD9
:10022800636103238DF86A3041F6FF7325F8503D6A
:100238004FF0904029460DF065FB4FF6FF734E488E
:10024800ADF8683029460DF05DFB4C4829460DF0A5
:1002580059FB4B4829460DF055FB584629460DF0E9
:1002680051FB294647480DF04DFB284606F0E6F8B5
:100278001A9B454AB3FBF2F3444A1360444B454A80
:100288004FF0000AC3F800A0434B5A60F02287F8E9
:1002980023200722C3F808A0404F1A60D8F8083076
:1002A8003B6099E80F0085E80F0063691A9843F4EA
:1002B80000136361636943F4001363614FF4885367
:1002C800ABF828304FF48843ABF828301BA90DF061
:1002D80019FB1DA91C980DF015FB64200AF0E9FD17
:1002E8004FF48C722E48514614F0D1F8E3692D4A28
:1002F80043F00703E361A36943F4C523A36163697A
:1003080043F4F013636102F1E00E55E0264B12222C
:100318001A606368636063686360636843F480635A
:100328006360636823F47C136360636843F4E813D1
:100338006360236843F08073236022680B4B92014B
:10034800FBD55A6822F003025A605A6842F002024A
:100358005A60636803F00C03082BFAD14DE700BF1D
:10036800900100200F6A0008D42B002000100240E2
:1003780000ED00E00005FA05000400480008004808
:10038800000C00480014004840420F00C014002030
:100398001C1500203F19010010E000E0E81F0020B4
:1003A80064150020B87D01080020024000100048B4
:1003B80048200020A45D0108937B506892F80FC084
:1003C80003F00701DB0800EB83038900186A4FF08C
:1003D8000F0A0CFA01FC0AFA01F120EA010119627C
:1003E800196A10324CEA010172451962E4D10022FF
:1003F80095490023535401320E2AF9D1DFF87CA223
:100408000AF11A02FF2199540133072BF6D18F4ABA
:100418008F4B1360DFF868B28E4A03930321117083
:1004280058460021242214F032F814228BF80020B8
:100438008949039B3F6801228BF8182098F805B07A
:1004480081F800B0A3F5EE71CAF824108349A3F52A
:100458008E730B60824B03EBCB035B78CAF82830B2
:10046800BB0648BFCAF8282000237E4A40F2DC5168
:1004780022F813100133082BF7D113A800211C22EE
:1004880014F005F8BBF10E0F03D00BF0EF03082BA7
:1004980002D101238DF85C3002200AF0DBFB18B191
:1004A8004088003018BF0120C7F340038DF8523050
:1004B800C7F380138DF85430C7F340338DF84C30B0
:1004C800C7F3C03300F001008DF84F3017F4006314
:1004D8008DF8510007D098F8863103F1FF3EDEF120
:1004E800000343EB0E038DF85030C7F300438DF83B
:1004F8005530B36AB8F84801ADF86000003318BF4A
:1005080001238DF85630C7F300538DF85730B8F8EB
:100518004A31ADF85A30F804B8F8563148BF524855
:10052800ADF85830C7F380438DF85330B8F85431DC
:1005380044BFB0F85001ADF86000B3F5FA7FADF8EC
:100548005E3084BF0023ADF86030484898F8D63153
:1005580086F82C30002386F82D3043709DF85C30E7
:1005680007F00101002BC7F3C0028DF84D108DF87C
:100578004E200CBF0023022301B902B1013309EB5D
:1005880083094FF0000AD9F810309A1E1A330392E3
:100598000593039A32F8023F03924FF6FF72934293
:1005A80000F072819DF855004FEA132EDAB25FFA17
:1005B8008EF330B110012E4F3F582E48874200F07D
:1005C8005E819DF8520050B1294F2B4807EB021766
:1005D8007968814203D13889012800F050819DF85B
:1005E8004F0050B1224F244807EB02177968814227
:1005F80003D13889042800F042819DF8500050B199
:100608001B4F1D4807EB02177968814203D13889CF
:10061800022800F03481BEF1020F02D19DF84C107F
:1006280004E0BEF1010F04D19DF84D10002900F03F
:1006380026819DF8561051B39DF85C1039BB9DF882
:100648005410F9B1111F1FE09C0100205012002026
:10065800382200209D10002010090020F8160020E4
:10066800908301081010002048200020BD010020C0
:10067800B87D0108004401400008004890010020AE
:1006880054120020A2F10801012998BF0423CA4F7F
:100698009DF857104FEA02194F4431B19DF85C108C
:1006A80019B9043A032A40F2D380012B4AD1C24A2D
:1006B800DFF81083079202EB0901FF2391F80DE0A0
:1006C80088F8743088F875304868C8F8847001F183
:1006D80008030989ADF868104FF0000B02218DF866
:1006E8006B1088F878B01AA98DF86AE0069388F834
:1006F80030B0C8F834B0C8F838B0C8F83CB0C8F85A
:1007080070B088F876B088F877B00DF0FBF8069BE3
:10071800079A997852F809005A460CF00BF93846AE
:100728000FF07AF9A54BC8F88830A54BC8F88C307B
:10073800C8F890B0384608F1880108F18C020DF02D
:10074800D7FC9CE0022B49D15FFA8AF21C2101FBFD
:1007580002FC9C4ACDF81CC002EB0C08964A88F8AB
:1007680079A0012188F8781002EB09014FF0000BFD
:1007780091F80DE0486888F87AB001F10802098913
:10078800ADF8681088F882B01AA9C8F884708DF896
:100798006AE006928DF86B300DF0B4F8864B069A35
:1007A80053F8090091785A460CF0C4F838460FF00F
:1007B80033F9844BDDF81CC0834AC8F8882003EB62
:1007C8000C01824AC8F88C208831C8F890B03846A5
:1007D8000A1D0DF08DFC0AF1010A50E0032B35D1FA
:1007E8009DF85330DFF8DC81DFF818923BB198F8B8
:1007F8002EB0384608214FF6FF7200231AE0BDF8E4
:100808005E2098F82EB0BDF86030B2F5FA7F0BD9AB
:100818006F49B1FBF2F23846082192B20DF09BF80D
:100828006C4B49F82B000AE06B49B1FBF2F23846F1
:10083800012192B20DF08FF8684B49F82B00C36084
:1008480098F82E30013388F82E3018E0042B16D192
:1008580096F82D80BDF858205F4B93FBF2F238468E
:10086800BDF85A30012192B20DF075F896F82D3086
:1008780006EB88080133C8F8580186F82D30039B29
:10088800059A93427FF485AE96F82D2086F8782154
:10089800534A544B92F800E0AEF117020027022A9F
:1008A8001F709C461AD8736A3B44D3ED007AF5EE64
:1008B800407AF1EE10FA02D1B36A63BB26E04A4AE5
:1008C80007EB02080FCB88E80F009CF800301037C0
:1008D8000133C02F8CF80030E5D1EDE7434B13F816
:1008E8003E908CF8009003EBCE03D3F804A0BAF145
:1008F800000FE1D04F45DFDA3B4A3B0103EB02082A
:1009080053440FCB013788E80F00F3E7384E3368BC
:10091800DF0424D41DE0374B374A13F83E0010702B
:1009280003EBCE035E68002EF0D000238342EDDA9D
:10093800C3EBC3017218DFF8D080D2F8009041F8F9
:10094800089001EB08079188B9809279BA71013350
:10095800ECE70EF0EF03082B284B20D122E09CF89F
:100968000020012AF5D9264B03EB0212103210336E
:100978009342EED053ED047AB6EE007A67EE877AAA
:1009880043ED047A53ED057A67EE877A43ED057AED
:1009980053ED037A67EE877A43ED037AE7E7BEF112
:1009A8000E0F33D11A7842F010021A70BEF1180FE8
:1009B80033D10AF017FE30E0B87D0108B9C300084A
:1009C80099C400089001002039CA000891C30008A2
:1009D80000127A00B9C4000840420F00A9C40008F8
:1009E80010090020601500204C08002090830108A1
:1009F800E81F0020B86C010884160020D4100020DD
:100A08005408002030150020851600201A7822F09E
:100A180010021A70BEF1190FCAE70AF0C7FD336851
:100A2800DFF834B3580358BFBC4BBD485CBF012244
:100A38001A70049B049A1B7843F0040313706269CC
:100A48004FF408534FF002094FF0010A42F4001224
:100A5800ADF8683029468DF86AA08DF86B90626110
:100A68000CF050FFAF4AB049116000200AF078FB43
:100A7800A26942F48052A261E26842F48052E260C4
:100A880062694FF0904642F400326261326A22F4A1
:100A980070023262326A42F4A0023262326A22F092
:100AA80070623262326A42F0A0623262326A22F0C6
:100AB80070423262326A42F0A0423262326A22F4F2
:100AC80070223262326A42F4A022002732624FF06A
:100AD8000308E022304629461A928DF86C908DF86A
:100AE8006D808DF86E708DF86F7005F01DFE102208
:100AF800304629461A9205928DF86CA08DF86D80C3
:100B08008DF86E708DF86F7005F00EFEE168874EF7
:100B180041F48051E160E16821F48051E160844949
:100B2800888820F480500004000C8880888880B26F
:100B380040F480508880088800F4415040F44570A3
:100B480040EA08000880888820F470600004000CDF
:100B580040F4E0608880888B20F40060000407235C
:100B6800000C88830B82088880B240F0400008801F
:100B780070490E60616941F480216161E16941F465
:100B88000011E161216B21F010012163216B41F01B
:100B980010012163DBF8201021F07061CBF82010E0
:100BA800DBF8201041F08061CBF82010DBF8201032
:100BB80021F07041CBF82010DBF8201041F0804183
:100BC800CBF82010402158461A9129468DF86E70AE
:100BD8008DF86F708DF86C908DF86D8005F0A4FD20
:100BE800802158461A91294605F09EFD3168524BDE
:100BF800059A21F0010131603068504901403160A7
:100C08004F493161316841EA0A013160B760F760E4
:100C1800B760B16841F40041B16031683160716812
:100C280021F0784121F400417160316841EA0A01FC
:100C380031601D68434E0493304605F4006339461D
:100C4800039305F4004B13F022FC049B8DF83D90B0
:100C580015EA09058DF83E708DF83F708DF83C80D7
:100C680005930DD03848CDF838A00EA905F05CFDE5
:100C78000622072332707770F37086F802A0554673
:100C8800BBF1000F0ED004232F480E930EA905F0D8
:100C98004BFD082333710723F371012375711D443C
:100CA800B371EDB2039B6BB1022327480E930EA9D3
:100CB80005F03AFD07233373F373012375731D445D
:100CC800B373EDB20EA908231F480E9305F02CFD4F
:100CD8000923337207237572F3720123B3721D441B
:100CE800E36A1A4823F4F873E362E36A43F4D873B7
:100CF800E362636943F0805343F00103636105F0E5
:100D0800E6FA1AA805F0B8FA114B1A93EDB2114B8E
:100D18001B93012D4FF0000320E000BF780D002049
:100D280000100048E02B002035AC000800540040BB
:100D380000300140DC0F0020E81F0020FFE0CF005A
:100D48007A25E000A81200200008004808000240A8
:100D580040000050B8120020000400480CBF1A469A
:100D680080221F924FF48072BD4C20924FF4806213
:100D780021922022204622921AA94FF400521C9355
:100D88001E9323922493ADF8745005F082FA2368D9
:100D980043F0010323604FF0A0440A20A36823F026
:100DA8004053A360A36843F08053A3600AF081F81E
:100DB800A36823F08043A360A368A360A36843F0FB
:100DC8000043A3604FF0A0418B68002BFADB8B68CF
:100DD800A44A23F040538B608B6843F000538B6028
:100DE8009068A14B034043F468339360CA689F4BF3
:100DF800134043F40053CB600A6B013D22F00F020D
:100E080015430D63002401233219917800296CD011
:100E18005D1C042B375DD078EDB24FF0A04E0ED894
:100E280003EB43035A00DEF830101F23934021EAF6
:100E3800030107FA02F30B43CEF8303031E0092BF7
:100E48000ED8053B06225A43DEF834101F23934080
:100E580021EA030107FA02F30B43CEF8343020E00D
:100E68000E2B4FF006010ED8A3F10A024A43DEF812
:100E780038C01F2393402CEA030107FA02F30B43FF
:100E8800CEF838300DE00F3B01FB03F2DEF83CC032
:100E98001F2393402CEA030107FA02F30B43CEF811
:100EA8003C30092F4FF0A0420FD99369A7F10A03EC
:100EB80003EB430397690721994027EA01019161F0
:100EC80091699840084390610EE053697B1E03EBDB
:100ED800430357693821994027EA01015161516953
:100EE80003339840084350612B460434102C8BD1AF
:100EF8004FF0A042936843F0010393604FF0A04382
:100F08001A68D107FAD5DA68594C22F00202DA6079
:100F1800DA6842F00202DA60DA6842F00102DA6066
:100F28009A6842F004029A60B4F85C31002B40F0F1
:100F3800DB85B4F95E21002A40F0D685B4F960213A
:100F4800002A40F0D185B4F864310393494B4A4EE6
:100F58001B684A48B3F85630049300210C2294F8D1
:100F6800635194F86B71B4F80CA094F80FB013F0B7
:100F78008EFA00211422304613F089FA404B336070
:100F8800404B41497360414B414A42483361022317
:100F98000B70052313700368069143F00103036087
:100FA80091463D4A0023092D137001D91D46F8E7E3
:100FB800012202FA05F140F2BA330B40002B40F04F
:100FC800878511F0450F00F08385192027211AAB7A
:100FD8000CF0AEFD002800F07B85284B2F4A1A60E4
:100FE8002F4A5A602B4A062389F80130136843F0C8
:100FF80002031360274D2B689A0702D51F4B1B6805
:101008009847DFF8A4802749BBF1000F4ED09DF820
:101018000C3013F0FF0F0AD12B6813F0020F4FF0BA
:101028007D0240F2712308BF4FF4FA7302E04FF4D7
:101038007A731A469A4505DBBAF57A6FA8BF4FF45A
:101048007A6A00E09A46531E5344B3FBF2F3013B1D
:10105800DBB203FB022288F879310A602AE000BF7C
:101068000800024000030050E010FCFF07C0FFFD2D
:1010780048200020201000203C280020B41F002019
:101088003FDE0008798F0008FA0D0020295C8F3DAB
:1010980018010020D0100020FA2B00208D8D0008A8
:1010A800398D0008782800209001002088F879B14F
:1010B800C1F800A0336898472B4A0023137017B172
:1010C800022F40F00B854FF0000A1E200A21012252
:1010D8001AAB8DF868A0C8F87CA10CF029FD88B17E
:1010E8009DF86830482B40F02785204B204A1A602D
:1010F800204A5A60022389F803302B6843F008031A
:101108002B6002E0824600F017BD94F858310BB10D
:10111800069A137094F859310BB1174A137094F862
:101128005A310BB1104A13702B68144913F0080F89
:1011380028D0BDF91000DFED126A642290FBF2F3AB
:1011480002FB130212B207EE902AB8EEE77A07EE16
:10115800903AF8EEE77AE7EE267AB2EE047A67EE8E
:10116800877AC1ED007A0FE0FB2B00209006002063
:10117800CD8D0008A58C0008FA2B0020041700204C
:101188008988883C00230B60B34F3B7843F0020307
:101198003B70B24B4FF488429A614FF488521A85DB
:1011A8004FF00A0ADFF8B492B9F814309BB283F40E
:1011B8008843A9F81430B9F814309BB283F48853E3
:1011C800A9F81430192009F074FE012009F0C8FFAD
:1011D800192009F06EFE0AF1FF3A002009F0C0FF5D
:1011E8001AF0FF0ADED14FF48853A9F828302B688B
:1011F8004FF4884A1B07A9F828A009D5984BC9F8C5
:1012080018A01B689847974BA9F828A001221A70C4
:10121800954B9FED968A1B68DFF894921B7B00EE36
:10122800103AB8EEC00A20EE080A05F0A3FEB9F895
:10123800003007EE903AF8EEE77A27EE800A13F0CE
:1012480035FB8B4B9FED8B7A1880B9F8003007EE91
:10125800903AF8EEE77A884BC7EE277AFF211A22F0
:101268009FED867AC7EE877A9FED857AC8ED607A1A
:10127800D6ED047A834E67EE887A304667EE877A31
:10128800C3ED007A13F003F9002232702A687E4B0E
:10129800012112F0020F19701FBF7170032119701C
:1012A800022118BFB1703046560741BF19784D1C4E
:1012B8001D70032548BF455412F00A0F0CD01A7848
:1012C80004218154511CC9B205254554D11C023250
:1012D800D2B2197006218154059A11688D0641BF52
:1012E8001A78551C1D70072548BF85540A0608D56D
:1012F8001A7809258554951C0132D2B21D700A2529
:1013080085546579082D01D00E2D04D11A78561C04
:101318001E700B2686541A7811F4803F4FF00C0E7D
:1013280000F802E002F101061CBFDFF85CE10232BE
:10133800F6B21E701FBF8EF80020524A4FF00E0EF4
:1013480002F806E04A0741BF1A78561C1E7010269C
:1013580048BF86541A78561CF6B24FF0120E11F494
:10136800806F1E7000F802E00ED094F80CE2BEF117
:10137800000F09D0DFF810E102328EF80020414A50
:101388004FF0130E02F806E01A7811F4007F4FF0C0
:10139800140E00F802E002F101061CBFDFF8E8E0D5
:1013A8000232F6B21E701FBF8EF80020354A4FF089
:1013B800150E02F806E0182D0DD11A781626865457
:1013C800561CF6B24FF0170E00F806E0D61C023293
:1013D800D2B21E7085540D0341BF1A78511C197082
:1013E800192348BF835400219822284813F04FF846
:1013F80004F0AFFC264B274A27491A6000234B808C
:101408000B7126490A60B4F8982190B2244921F852
:1014180013000133122BF9D1224E3368D8045CBF74
:10142800B4F89E0108801B0740F1F8801E4B93F822
:101438009231062B00F2EC80DFE803F004073E6DE2
:1014480088A7A70045F2F05201E042F6F822174BB0
:101458001A8004F034FDDAE0D42B00200010004894
:1014680090060020A80600205C07002035FA8E3C74
:10147800780700200AE81C415807002000401C4655
:10148800BD378635E90F0020E80F0020AC11002099
:10149800B40E0020D2210020040E0020C42B00200E
:1014A80024200020E81F002048200020C807002032
:1014B80012000020CDCCCC3F07EE902A5FED036AE6
:1014C8007C4BB8EEE77ADFED7C7AE7EE267A42F6D7
:1014D800F82119800023FCEEE77A784A17EE901A73
:1014E80042F823100133122BF7D1754A7549116060
:1014F800754A4020137009F0EDFB002800F0888041
:1015080001234FF0070990F90000704A8DE808029E
:1015180040216F4B76E0674B42F6F8221A80684B01
:101528006C4A1A60684B102240201A7009F0D2FBEE
:1015380000286DD001234FF0000C90F90000664A96
:101548008DE8081040214FF4E1335BE0594B42F637
:10155800F8221A805A4B614A1A605B4B08224020D5
:101568001A7009F0B7FB002852D001234FF0000E83
:1015780090F900005A4A8DE8084040214FF4E133C1
:1015880009F0A1FCC8F884013EE04A4ADFF88891D6
:10159800DFF888C1DFF888E1524D534C534842F6D2
:1015A800F821118048490C22062B0A700ED000231E
:1015B80089F800308CF800308EF800301B232B702F
:1015C8000523227003704FF4E1340BE0002189F801
:1015D80000108CF800108EF8001022702121444C65
:1015E80029700370364B434A1A60402009F072FB99
:1015F80070B101230025404A90F9000040218DE890
:101608002800234609F05FFC003018BF012028B9E4
:10161800082005F073FD2A4B384A1A6033682A4AB5
:1016280013F4804F1FBF082111702549344818BF93
:10163800086042F20101194003F0010003F400546C
:1016480079B11C4944F620650D8024B10821117038
:101658001B492C4C0C6020B10C21117018492A48E8
:101668000860117804395170190640F192800025FC
:10167800264CDFF8B090C8F88891294615222448EE
:10168800DFF8A48065706560A56012F000FFA9F11D
:1016980005032846C8F800300AF0CCFC1D4B022090
:1016A8001B68E36009F016FB00283FD1802005F095
:1016B80025FD66E0C80700200000B0C4CC2A002041
:1016C80018000020C90D0108481200204510010823
:1016D800A0860100B50D0108990F01089D0D0108AC
:1016E8004D0F0108362B0020592A0020372B0020E7
:1016F80090D00300C50C01082D0E0108290E010821
:10170800FD0D0108190E0108090E0108AC0600209C
:101718001C0300200C2000205A2A0020352B002012
:10172800342B002038220020CC060020637845792D
:10173800C3490C2202FB03125278AA4204D0013397
:10174800DBB2042BF4D900236370D8F80030627838
:101758001B7890F90000002B4FF00C0303FB0213D9
:1017680014BF0325012500225B7800950192022110
:1017780009F0A9FBB34B1860002897D001200AF0A4
:1017880059FCB14B1868B14B00F5C5721A600AF0E4
:10179800FFFCAF4AAF4B1360AF4AB04D80331360C4
:1017A80033680024DA032C7040F1AD800CF094FD0E
:1017B800DFF810C3DFF81093CDF810C040F22A3BD1
:1017C8004FF00108604621465A4685F8008012F01D
:1017D8005EFED9F81430A248A24D43F48023C9F81C
:1017E8001430436A23F00F034362436A43EA080351
:1017F8004362022203234FF4807A0CA98DF8342027
:1018080003928DF835308DF83640CDF830A08DF83C
:10181800378004F089FFD9F81830039A43F400336D
:10182800C9F818302B8823F440731B041B0C2B8039
:101838001D23EB620EA92A8560232C862846C5F84D
:1018480014800E93ADF83E401094ADF84440ADF8C6
:101858004640ADF84840ADF84A40ADF83C8004F049
:10186800AFFDAB6943F00803AB616B6C43F4004315
:101878006B64D9F8143043EA0803C9F81430A9F5A1
:101888007D69484604F023FD1AA804F0F5FC764B60
:101898001A9310231C938023DDF810C01F931AA9F4
:1018A8004FF400534846CDF86CC02393ADF874B09C
:1018B8001E94CDF880A021942294249404F0E9FC8D
:1018C800EB6843F40073EB60D9F8003043F002038F
:1018D800C9F800300BA80D238DF82C308DF82D8019
:1018E8008DF82E408DF82F800EF078F821465F4B4A
:1018F8001A685F4B43F8212001312029F7D10BF0FA
:1019080023FF0BF021FF33685B0556D5594D5A4B21
:10191800D5F8CC84C3F80080042009F0DBF9042151
:10192800C5F8D00409F0B2F9544B85F8D40408205E
:10193800C3F8008009F0CEF9514B524C18600821C9
:1019480009F0A4F9002185F8D5042C22204612F0CC
:101958009EFD8E2363704FF07C0AE0234FF07D09D3
:10196800E37084F800A084F82B90474C2C220021C7
:10197800204612F08CFD8A2363701020A023E370A8
:1019880084F800A084F82B90C5F8D88409F0A2F94F
:101998001021C5F8DC0409F079F985F8E004202065
:1019A800C5F8E48409F096F92021C5F8E80409F09F
:1019B8006DF985F8EC040FF05BFC3368334A13F4D7
:1019C800002318BF0123137009F04EFA304B18603A
:1019D800304B5A79052A194602BF2F4B4FF4C8726B
:1019E8001A802E4B4FF47A721A802D4A137843F0DE
:1019F800080313702B4A137823F00203137032681C
:101A080040F6020313406BB1274B284A1A60284B53
:101A180003221A70274B01221A70274A00231380C9
:101A2800264A13808B683360254B01221A703B7855
:101A380063F07F033B702FB0BDEC028BBDE8F08FE5
:101A4800345E0108E01C002020100020100F002048
:101A58008013002064220020181D0020790D00202A
:101A6800000400480044014034440140C45D0108BA
:101A78007A0D002090010020C41000201C110020C5
:101A880068110020EC10002021110020742800208B
:101A9800A807002048200020C60E0020F42B0020B4
:101AA800D4100020FD2B0020BC100020C4210020F1
:101AB8002011002010010020B00F0020B20F0020DC
:101AC800780D0020310300200010024035FA8E3CCA
:101AD800012D7FF68FAA0025FFF763BA012F7FF645
:101AE80014AB1F46FFF7E8BA1BB207EE903A5FED5A
:101AF800096AB4F95E31154AF8EEE77A07EE103A4A
:101B080067EEA67AB4F96031CDED1A7A07EE903A0D
:101B1800B8EEC77AF8EEE77A002127EE267A67EE64
:101B2800A67A11701AA80A498DED1B7ACDED1C7A98
:101B380005F028FAFFF707BA012F7FF6E6AA054B4A
:101B4800002783F800A0FFF7BEBA00BF7C00002082
:101B580084120020FB2B0020874A2DE9F04F1368E0
:101B6800864C03F59C4320332DED028B2360A3881C
:101B78000133A380824B196889B011F4804F059214
:101B8800019305D10FF0C2FA10B9237B01332373F7
:101B980000277C4BDFF804821E78FDB2AE4230D9B4
:101BA800D8F800307748072D98BF595D764B88BF25
:101BB80029461B689847032D1ED8D8F8002005F140
:101BC8000E0302EB83039988DA88A8B14FF47A737D
:101BD800401A5843531A90FBF3F040F6C90300F536
:101BE8007A70984205DC40F2EE239842B8BF184656
:101BF80001E040F6CA0080B204EB45050137E881F0
:101C0800C7E70F23277B84F83230032594F8333055
:101C1800B7FBF5F505EB45057D1B029394F83430C9
:101C28000393D8F800A0DFF87CB1EBB20493002549
:101C3800B54255DA5549029B31F815904FEA4508E7
:101C480053B90FF063FA28B1039B002B08BF4FF07C
:101C5800000901E0DDF80890BAF81400484503D8F7
:101C6800BAF8160048450ED2E8B20FF025FA032D4F
:101C78008146DFBF94F832E00120A8402EEA000038
:101C8800D8BF84F832000FF041FA18B1404828F85C
:101C9800009021E0049B94F87E002BF8139028B95B
:101CA800022F15D93549012081F87E00BBF80210B2
:101CB800BBF800000844BBF804100844354980B25A
:101CC80028F8010000B2032190FBF1F080B200E097
:101CD80048462F4928F8010001350BF1060BA7E704
:101CE80094F83250254BA5F10F0EDEF1000545EBB7
:101CF8000E0584F898503DB19A8811B21429CCBFCA
:101D0800143A00229A800BE083F83350B54207DA80
:101D1800E8B20FF0D1F91E4B23F815000135F5E7AD
:101D2800019B1B68DF0405D51B4B1B68DE0701D42C
:101D38000EF021FE059B1968184B1868837A9BB32F
:101D4800013B134D027B35F813301AB1C3F53B63E1
:101D580008339BB21BB2A3F57A73B3F57A7FA8BF99
:101D68004FF47A7323EAE37307EE903A9FED0C7A07
:101D7800F8EEE77A51E000BFDC2B0020000E0020CF
:101D8800E81F002048120020180000200E0E002036
:101D980024200020800E0020E40F0020C42B002007
:101DA80000007A44360E0020019A1268150440D5C6
:101DB800D4F89C20AD4E8A1A002A3ADB01F59C42E1
:101DC8002032C6F89C20AA4AC07A5579A94A32F826
:101DD800152096F8A050013592B292FBF0F205F06A
:101DE8000F0086F8A000304480F8A1201A46A248C7
:101DF800185C01330244102B92B2F8D112B292FB54
:101E0800F3F31BB2642BA8BF642323EAE37307EE42
:101E1800903A9FED9A7AF8EEE77AC7EE877A984A71
:101E28009FED987A67EE877AFCEEE77A17EE903A9C
:101E38001380019B944D1B68DFF8708213F4807F38
:101E48007AD0924B994204D9237A13B9874B01224D
:101E58001A72B4F904E098F80060844BBEF1140FCC
:101E6800CCBF4FF0000E4FF0010EC6F38006BEF156
:101E7800000F03D000279F725F7200E00327A07A4B
:101E8800D4F8B4B0D4F8B8C0B4F90490617AE3884F
:101E98002A88032848D8DFE800F0020E1B35BEF177
:101EA800000F02D02A8000222AE0002E40F0688627
:101EB8002A80A6723AE09CF8000000EB8000814579
:101EC80002DC2A8001221BE001206EB300F0BCBEB8
:101ED8003EB1BBF80E206A80AA80BCF80200E880F8
:101EE80002279CF800A09CF80100504400EB8000F9
:101EF800814500F34886002E00F045862A8002229C
:101F0800A27213E02A800322A2726172E3807EB17A
:101F180098F8003043F0020388F80030534B002251
:101F28005A720EF028FD03E02A80A0726172E380E5
:101F380017B1384609F032F9554EB6F852010DF08E
:101F4800C1FF834668B90EF083FB524BC3F800B05B
:101F5800C3F804B0C3F808B04F4B00221A605A60A7
:101F68009A6098F800305A0736D5019B1B68DB0643
:101F780032D54A4B1B78DF062ED4494B1B7893B1D8
:101F880096F8DE31BBF1000F15D17BB1454B1A68CD
:101F9800D4F8BC309B1A002B08DA0EF0ECFC334B5B
:101FA80083F8C0B018E0BBF1000F0DD1102009F084
:101FB800F5F801230EE03BB13A4A12684FF47A7102
:101FC80001FB0323C4F8BC3094F8C03023B109F0F6
:101FD800CDF8002384F8C030002396F8DCA196F8E9
:101FE800DD11B6F89A71B6F89CE1184635F9132058
:101FF8008008BA42C4BF60F07F00C0B201337245A6
:10200800B8BF40F04000042BF0D194F8C130174A13
:10201800834205D192F8C230F92B04D8013300E08D
:10202800002382F8C2301E4A84F8C10010780F4B92
:102038001D4F914600283ED13A68D00709D5BBF11B
:10204800000F38D198F80030D90734D50EF00EFBC0
:1020580031E098F8002052072DD593F8332052B379
:102068005B7A43BB21B30EF086FC24E0000E00200F
:10207800A8120020B8120020A10E00200000C842BB
:102088003C10002000C07F4424200020404B4C001E
:1020980048200020B01300206C140020D410002029
:1020A800100000200C200020E40F0020FD2B002051
:1020B800BBF1000FD7D094F8C230B64ADFF800B3AE
:1020C800142B40F08C8099F800301AF1000A18BFE0
:1020D8004FF0010A7BB392F8C1305F2B12D198F808
:1020E800003003F0040303F0FF0113B10EF043FCCA
:1020F80008E00B200391029209F050F8029A039924
:1021080082F8C210BAF1000F15D094F8C1307D2BB7
:1021180011D198F8003003F0040303F0FF0213B163
:102128000EF029FC07E00B20029209F037F8994BD2
:10213800029A83F8C22098F8003003F0040303F0F1
:10214800FF01002B4BD194F8C130924A572B11D183
:10215800914B4FF47A721A80019B1B681B0601D5BC
:102168000AF078F88D4B1B6813F0080337D18C4AB6
:10217800138034E001980068400717D55A2B15D111
:1021880092F8C3302BB1012382F8C31082F8C4300F
:1021980025E092F8C53083F0010382F8C5300BB111
:1021A8000C2000E00D2008F0F9FF18E05D2B00F08E
:1021B80020855B2B00F01F855E2B00F01E85562BBB
:1021C80001D105F017FA99F80030002B00F0E484EB
:1021D80094F8C1306F2B40F0D9840EF047FA019B78
:1021E8001B68580737D594F8C5306A4A93B198F8F0
:1021F800003059070ED5B5F90610B6F89A3199424C
:1022080008DD3B6813F0010302BF3221A2F8C810B1
:1022180082F8C5303B68DA030DD594F8CA205D4BC7
:102228002AB993F8C32012B93222A3F8C82001238F
:1022380084F8CA300FE094F8C330564A5BB198F876
:10224800003003F0040303F0FF0123B9012382F8EF
:10225800C31082F8C430DBF8009000233B6009F11A
:102268007B0609F1CB0A3278737816F8010C9A428A
:102278000BD2314608F098FD38B116F8022C01232C
:1022880003FA02F23B6813433B6004365645EAD131
:10229800444B1B7843B1444D404F2B68434E13F0D9
:1022A800020F40F035832DE309F1CA0609F5897755
:1022B8003278737816F8010C9A4225D2314608F024
:1022C80073FD08B3B37896F804E0394A96F803909A
:1022D80030480C21013B01FB0E4103EB430313443F
:1022E800D1F8D0209A420FD0C1F8D030002390F80E
:1022F800FC20C1F8D430012303FA0EF322EA0303C9
:1023080081F8CC9080F8FC300636BE42D0D1294BFB
:10231800DFF8B0B01E68284B1B68039394F833307D
:10232800049300230293DBF80030002B00F0E182D5
:1023380093F80090B9F1000F00F0DB82DBF804207D
:1023480003998A1A002A0CDB01F5FA720299CBF874
:10235800042001228A4094F8FC1021EA020284F841
:10236800FC20049A002A00F0C4821BF8042C597837
:102378000432D2B2002940F07E8235F912100F4A99
:10238800044FB2F8982102F1C800814222DD93F887
:1023980002A035E0000E0020F42B0020D010002011
:1023A800B0100020012C0020E40F0020981100201C
:1023B80014620108401000200C2000204820002052
:1023C80020100020D00E00200000C84200000000AD
:1023D80000007A44C83A914203DA9978C1F1000AB8
:1023E8000EE0029A0123934097F8FC2022EA0303A7
:1023F80087F8FC30039B03F5FA73CBF8043078E2D6
:1024080097F8FC30029A1341DB0700F17282BAF1A7
:10241800000FCCBF0220012008F0E6FE09F1FF33CF
:10242800132B00F25D82DFE813F0140021002F0067
:1024380043005C006300CA002D019401C401F4014B
:102448005B02430052006300CA002D019A00FF009E
:10245800640137785744FA2FA8BFFA2727EAE777A5
:102468003046377008F086FC01200BE07778574437
:10247800642FA8BF642727EAE7773046777008F00B
:1024880079FC02203946C1E196F80390D144B9F1AC
:10249800640FA8BF4FF0640929EAE97986F8039028
:1024A8003046D7F8001108F01BFC03204946ADE17F
:1024B800717951446429A8BF642121EAE1717171DD
:1024C8000D2008F0BDFCB9F10D0F00F0098231793B
:1024D80051446429A8BF642121EAE17131710E20B9
:1024E80094E1B179514481F30801B17105208DE17E
:1024F800D7F804311A78022A22D107EE90AAF8EE0A
:10250800E77AB2EE040A87EE800AD3ED097A30EE54
:10251800270AB5EEC00AF1EE10FA09D45FED567A33
:10252800B4EE670AF1EE10FAC8BFB0EE670A01E030
:102538001FED5A0A83ED090A0F2008F06CFC0AE027
:1025480099785144C829A8BFC82121EAE171997036
:102558000F2008F075FCB9F10F0F00F0C181D7F812
:1025680004311A78022A20D107EE90AAB8EEE78A39
:10257800B2EE040A88EE008A93ED080A38EE000AE3
:10258800B5EEC00AF1EE10FA09D45FED717AB4EE37
:10259800670AF1EE10FAC8BFB0EE670A01E01FED56
:1025A800750A83ED080A122058E159785144C82960
:1025B800A8BFC82121EAE1715970122026E1D7F895
:1025C80004311A78022A20D107EE90AAB8EEE70A59
:1025D8005FED837A93ED0C7A80EE270A30EE070AD6
:1025E800B5EEC00AF1EE10FA07D4B4EE670AF1EEC0
:1025F80010FAC8BFB0EE670A01E01FED8C0A83ED40
:102608000C0A102008F007FC0AE0197B5144C8297D
:10261800A8BFC82121EAE1711973102008F010FC45
:10262800B9F1100F00F05C81D7F804311A78022A4A
:102638001ED107EE90AAB8EEE78A5FED9D7A93ED7A
:102648000B0A88EE278A38EE000AB5EEC00AF1EECA
:1026580010FA07D4B4EE670AF1EE10FAC8BFB0EE6C
:10266800670A01E01FEDA70A83ED0B0A1320F5E0C6
:10267800D97A5144C829A8BFC82121EAE171D97281
:102688001320C3E0D7F804311A78022A22D107EEC2
:1026980090AA1FEDB10AF8EEE77A87EE800AD3ED2B
:1026A8000F7A30EE270AB5EEC00AF1EE10FA09D417
:1026B8005FEDBB7AB4EE670AF1EE10FAC8BFB0EE70
:1026C800670A01E01FEDBF0A83ED0F0A112008F029
:1026D800A2FB0AE0997D5144C829A8BFC82121EA74
:1026E800E1719975112008F0ABFBB9F1110F00F0F9
:1026F800F780D7F804311A78022A20D107EE90AA79
:102708001FEDCD0AB8EEE78A88EE008A93ED0E0A2F
:1027180038EE000AB5EEC00AF1EE10FA09D4DFED82
:10272800BC7AB4EE670AF1EE10FAC8BFB0EE670AD9
:1027380001E09FEDB80A83ED0E0A14208EE0597D62
:102748005144C829A8BFC82121EAE171597514204C
:102758005CE0D7F804311A78022A20D107EE90AA53
:10276800B8EEE78AB2EE040A88EE008A93ED0A0A08
:1027780038EE000AB5EEC00AF1EE10FA09D4DFED22
:10278800A47AB4EE670AF1EE10FAC8BFB0EE670A91
:1027980001E09FEDA00A83ED0A0A09205EE0D978DE
:1027A8005144C829A8BFC82121EAE171D97009207C
:1027B8002CE0D7F804311A78022A1ED107EE90AA25
:1027C800B8EEE78ADFED927A93ED0D0A88EE278A54
:1027D80038EE000AB5EEC00AF1EE10FA07D4B4EEEE
:1027E800670AF1EE10FAC8BFB0EE670A01E09FED84
:1027F800890A83ED0D0A0A2030E0597B5144C82923
:10280800A8BFC82121EAE17159730A2008F018FB12
:1028180066E0D7F804311A78022A22D107EE90AA86
:102828009FED7D0AB8EEE78A88EE008A93ED100ADC
:1028380038EE000AB5EEC00AF1EE10FA09D4DFED61
:10284800747AB4EE670AF1EE10FAC8BFB0EE670A00
:1028580001E09FED700A83ED100A0B2008F0DBFA07
:102868003EE0D97D5144C829A8BFC82121EAE171B9
:10287800D9750B20CAE7012932D1987835F9123079
:10288800B3F5617F05DB40F633029342A8BF1346D8
:1028980001E04FF46173B9F10C0F21D14FF4966246
:1028A80092FBF0F05D4AA3F5617393FBF0F3DFB29E
:1028B8001378BB4214D0042F34BF3B460223137055
:1028C800574A09FB0323574A0633136004F0DEFC1A
:1028D8004846394608F0B4FA781CC0B208F084FCBF
:1028E8005149029A0123934091F8FC20134381F83F
:1028F800FC30029B0133042B02930BF10C0B7FF489
:1029080012ADC8E4019B1B68D8050ED5637A63B184
:102918003B68990709D5338813F001090AD10DF0EE
:1029280097FE012004F0DAFB04E0012004F0C5FB67
:10293800012300E000232A6852070CD55BB101206F
:1029480004F0BBFB3388980708D40DF081FE022001
:1029580004F0C4FB02E0022004F0AFFB3388334AE2
:1029680013F0030F4FF4884114BF916111853A6841
:1029780012F00A0F23D02A68D10609D55A070AD4BB
:10298800042004F0ABFB2A4B1B88A4F8083102E0B2
:10299800042004F092FB2B689B0606D53388580662
:1029A80006D4402004F09AFB02E0402004F085FBA6
:1029B8002B68590642BF1E4B1B88A4F80A313B6896
:1029C8009A0608D42B681B0540F1A6804FF4807046
:1029D80004F084FBA4E0174B1B789F0768D5164BBF
:1029E8001B78042B64D92B680F4F13F4007927D078
:1029F8003388DC0650D4102004F070FB202004F04B
:102A08005CFB0E48011D09F079FB022340E000BF82
:102A18000000C8420000000000007A44941F002013
:102A2800E827002040100020000E00200010004879
:102A3800B0100020D4100020DA1000204810002028
:102A4800348804F01004A4B22CB1102004F035FB33
:102A5800012487F80C912B68580512D5D7F8103146
:102A680089495A89B1F90030002BB8BF5B429342BB
:102A780007DAB1F90230002BB8BF5B429342C0F2CB
:102A8800E9803388990608D5202004F016FB002336
:102A980087F80C31012400E0002497F81431B3B909
:102AA8000E2008F07BFB794B012283F814210EE0FD
:102AB800338803F03003002B84D0102004F0FDFA93
:102AC800202004F0FAFA002384F80C3102E0002CEC
:102AD8003FF478AF6E4B002003F1280603F1500451
:102AE8006C4A002122F810106B4A596022F8101025
:102AF8000432716022F8101000221A609A60326065
:102B0800B26022606160A260143314361434002865
:102B18007FF458AF0120E3E74FF4807004F0CDFA5A
:102B28005E4B5A79082A1C4601D00E2A02D1402051
:102B380004F0C3FA019B1B685A0540F1A08094F881
:102B48000C3223B998F8003013F0040F02E02B6818
:102B580013F4002F0BD0524B00221A703C2003F0C4
:102B6800F7F9002800F08B800CF08AF8F6E70EF0F1
:102B78007FFB09B0BDEC028BBDE8F04F03F0E9B86C
:102B88000120FFF786B90320FFF783B9BAF1000FD8
:102B980002D07E2B3FF421AB94F8C130972B06D19D
:102BA8003A4B4FF4C872A3F8C620FFF718BBA72BFF
:102BB80006D13C4A137843F004031370FFF70FBBA8
:102BC8000022BB2B079201D1022303E0B72B04D1CB
:102BD8004FF6FE73ADF81E301FE0BE2B01D1022365
:102BE80004E0BD2B7FF4FBAA4FF6FE73ADF81C3052
:102BF80013E0012002E0022000E003205FFA80F9E0
:102C080009F1FF3386F8A43704F0AAFA04F062FB4E
:102C1800484608F0E9FAFFF7E2BADBF80030BDF8F9
:102C28001C10B3F858200A44A3F85820BDF81E1009
:102C3800B3F85A200A44A3F85A2004F0DBFC002316
:102C480084F8C230FFF7CBBA013301469BB20220A9
:102C5800FFF71FB933889B063FF51FAF202004F00C
:102C68003DFA1148114B011D1A685B684360026008
:102C780009F044FA054B012483F80C410DE709B02B
:102C8800BDEC028BBDE8F08FB4100020000E0020D0
:102C9800180F0020F62B0020900F0020482000205D
:102CA8004D120020D410002050100020DC1000200D
:102CB8002DE9F04FC14BB3F90610C14B2DED028B36
:102CC8001F687A8989B0914201930EDBB1F5FA6FDA
:102CD800FC79BDBF8B1A6343A2F5FA64C4F164049E
:102CE800BCBF93FBF4F4643400E06424B54AB64BEB
:102CF800B2F898A192F962211868049092B20592EC
:102D0800054600220293AD4B33F912300393CAEB08
:102D1800030303F2F31640F2E63086424FEA420B11
:102D280003D8002BB8BF5B4201E04FF4FA73022AC4
:102D3800049E4FF064002FD096F811E1BEF1000F09
:102D480004D07345CCBFCEEB03030023DFF8C0E209
:102D580093FBF0FC6FF063093EF81C809B4E09FB67
:102D68000C390CF1010C3EF91CE00FFA88FCCCEB95
:102D78000E0E0EFB09FE9EFBF0FEC64426F80BE085
:102D8800BE1836797343924E93FBF6F364339BB2C5
:102D9800634393FBF0F02EE096F812E1BEF1000FCA
:102DA80004D07345CCBFCEEB03030023DFF84C827D
:102DB80093FBF0F06FF0630C0CFB003938F910E06E
:102DC8000130002B38F91000CEEB000000FB09F9A8
:102DD800BDF8140099FBFCF9CEEB090919FB00F9C1
:102DE8007A48A0F80490B879B8BF5B424343784862
:102DF80093FBF0F064306B78764E4FF0640E4343EB
:102E080093FBFEF3B354744EEB7A434393FBFEF308
:102E1800B3546B7D6D4E5843704B90FBFEF0022A05
:102E280098546F4B0FD183F802E0039B53450EDB98
:102E3800644CB4F89A21914215DBB1F5FA6FA8BF3A
:102E48004FF4FA6110E09C54039B534504DA36F8BA
:102E58000B305B4226F80B300132032A05F10105DD
:102E68007FF451AFE4E71146891A4FF47A73DFF81B
:102E7800A4E1564D59436FF06303C2F5FA62642723
:102E8800B1FBF2F191FBF7F23EF8120003FB0211DD
:102E9800013203B23EF91220D21A514391FBF7F3E3
:102EA8000344F3804F4B1B88580635D54E4B4F4A89
:102EB8001B881288DFED4E7A9B1A1BB208EE103A77
:102EC800B8EEC88A28EE278AB0EE480A04F052F80D
:102ED800F0EE408AB0EE480A03F0E9FFB5F9023097
:102EE80006EE903AB5F90030F8EEE66A07EE903A49
:102EF80020EE667AF8EEE77AA7EEA87A67EE807A8F
:102F0800BDEEC77AE6EEA87A17EE103AFDEEE77A3C
:102F18002B8017EE903A6B80364D2B68990740F15D
:102F2800A180354B354F1A687B6945F20721D31AC2
:102F38008B4240F397807A6103F0CEFC304BDFF888
:102F4800D8901A78032A9846B9F8003022D10A2B6B
:102F58002AD90023282088F8003007F0AAFF03F0B8
:102F6800BBFC284B18880EF091F8274B1A68D378C9
:102F780090FBF3F001300828244BA8BF08201870F4
:102F8800537980B213FB00F33B83137913FB00F0F2
:102F9800788309E00A2B07D803231C4A88F80030F5
:102FA800002313703B837B8398F80030144A012B6D
:102FB8003DD033D3022B4CD054E000BF2420002056
:102FC800401000204820002020100020B4100020CD
:102FD8000CFEFFFF2C140020A60F00204414002034
:102FE8009013002098110020B01000200A0F002034
:102FF80035FA8E3CE81F0020DC2B0020980F0020BB
:1030080020110020C0120020BC1000201001002058
:10301800B21400209A140020C01000203A8BB9F88E
:1030280000309A421EDD012388F800300FE0B9F81D
:1030380000107B8B8B4202DD022313700FE09E4B46
:103048001B8B0133994202DD002313700AE008202C
:1030580006E07B8BB9F8002001339A42E3DC0720B5
:1030680008F09CF82D682A0576D5944B924F1A687B
:10307800FB69C3EB020845F2072398456CDD904BCA
:10308800B6F906B0D3F80090FA6199F80A30B4F8A6
:1030980052018C4E012B4FF47A71ABF57A7B98FB79
:1030A800F1F803D041D3022B20D040E0864B386A98
:1030B8005A7B864B33F812204FF0080E92B290FBE1
:1030C800FEF3C01A8318BA843B6240F6E44293FBCD
:1030D800FEF39BB25343B9F80820C2EB13335943AC
:1030E800B9F9063091FBF3F1316020E0784BB9F87B
:1030F80008A01B78C6F800A05B0718D50CF0E2FE04
:1031080020B915F0100F18BF4FF0000B32220BFB3F
:103118000BF393FBF2F3B9F906205B445A434FF4DF
:103128007A7392FBF3F3534400E000233360D7E94A
:103138000A013368674A03FB08F84FF47A7398FB6F
:10314800F3F810EB080041EBE8710023C7E90A0126
:103158000EF0A8F9604B1860604E3368D90427D583
:103168002A0622D55E4B1B789B071ED55D4B187827
:1031780004281AD900225C4BD7180521951C4FF05A
:103188000A0E122AD154E9B287F801E004D0B0EB54
:10319800510F2A46EFD800E014215A18322002F8BD
:1031A800010CFF225A540F2000E00A2007F0F6FF16
:1031B8004E4D2A68002A50D04D4B4E4F186839683A
:1031C8008142984649D84C4BDFF8389119785268B3
:1031D800E1B94FF0010A83F800A0B9F80030D35CD8
:1031E80023B3504607F0BCFF444B83F800A00DF012
:1031F80099FFB9F80030CBB92B681B78053B5345CC
:1032080014D807F031FE3E4B18600FE04FF0000A6B
:1032180083F800A0B9F80030D35C3BB1504607F002
:103228009FFF364B83F800A00DF07CFF2A68B9F8A1
:10323800003052683348D25CFE2A01D100230BE0EB
:10324800FF2A02D107F092FF07E0D8F800500A21C0
:1032580011FB02523A60013303801D4D2B785F0742
:1032680004D5294B4FF488529A6163E03268D0073D
:103278005CBF43F001032B70194B1B7819075EBF25
:103288002B7823F001032B70D30242BF2B7823F055
:1032980001032B701D4B1A88184B1AB11C4A12686F
:1032A800970702D41B4A1288B2B302221A702B78ED
:1032B80023F001032B7034E0980F0020DC2B002052
:1032C800BC100020C8100020A8120020B81200204E
:1032D800FD2B0020407E0500CC100020E40F0020CC
:1032E800D4100020DA100020C01F00202C15002068
:1032F8000C2000202415002020150020C82B0020B9
:103308000C2A00202815002000100048C60E0020B6
:10331800D0100020F42B00202978CE0758BF0222B5
:103328001A7007F0A1FDB04B1B68C01A002801DB1A
:103338000DF0F8FEAD4F0DF09BFF3E78002E00F02B
:10334800AB80AB4B1A689846002A00F01B87D8F868
:10335800000007F0A4FF002800F01487A44BA54C38
:10336800186807F099FF092801D03F2852D14FF07B
:10337800000A2668DFF8B492554636B19E48D9F857
:103388000010324611F0D0F810B9CA4605B94D46BA
:103398009A4B09F110099945EFD3EDB1D5F800C062
:1033A800DAF8009023681CF803E019F80300704568
:1033B80012D15A1C904958B92D2B09D8DFF834E29C
:1033C800CEF800204FF0200E01F803E0885403E007
:1033D80001F803E02260E5E723680BB1554510D0FA
:1033E80087480BF047FD554507D855F8100B0BF0EB
:1033F80041FD09200BF036FDF5E782480BF03AFD58
:10340800002623689E42A2D27B4B985D0BF02AFDD2
:103418000136F6E72368002B40F09986042840F02F
:10342800D686754809F0D2FC00F0ACBED8F800008A
:10343800DFF8DCA107F033FF20B3DAF8000007F06B
:103448002BFFDBF8003093F848100246A1BB242874
:103458006BD1012283F84820DBF80030DFF8D0A1D7
:1034680093F84820062AE1D193F8490000F042FF7A
:10347800834600287BD00BF051FCD9F8003000229D
:1034880083F84820604B93F83530002B40F04D8688
:103498004C36982E00F076865C4BF21892F84A105B
:1034A8000129F5D1DFF88891F358C9F80020584A66
:1034B800CB4613609046B9E7012904D14D2814BFC3
:1034C80000220222C6E7022904D13C2814BF0022A8
:1034D8000322BFE703290CD140284FF0000102D98D
:1034E80083F84810B8E758711971D9719871042296
:1034F800B0E7042906D1997983F849004A409A71BE
:103508000522A7E70529A7D158791979884298791A
:1035180006D950409871481C18710B441A729BE7E1
:1035280090420CBF0622002294E72B78590793D4C7
:103538002328DAF800300DD1012139702C49039085
:103548000B60314933480B630BF094FC2D480BF0AA
:1035580091FC039A304B1B681B78934201BF2F4B99
:103568002F4A1A602F4B04BF2F4ADA6074E7DAF843
:10357800002092F849304C2B00F0888400F28580B6
:10358800332B00F0DB8421D8292B00F04B8409D899
:10359800252B00F02284272B00F02684232B40F0D3
:1035A800128609E22D2B00F04E8407D82B2B40F011
:1035B8000A860BF085FB607100F0B2BD2F2B00F07E
:1035C8002A85312B00F03C8500F0FDBD3E2B00F034
:1035D800E58044D8372B00F0E5842BD8352B00F054
:1035E800268200F0F0BD00BFCC2B0020012C00206B
:1035F800B01F0020141D0020E41C0020F86B0108F7
:10360800AE810108B3810108980F0020AC11002099
:103618007C110020E381010850120020FC9F00204B
:10362800EFBEADDE00ED00E00400FA05386A0108DF
:1036380078110020392B00F0E4833C2B40F0C3853F
:10364800DFF84C84D8F800A00BF03AFB8AF80000A9
:10365800D8F80030187808F061F800F061BD432B05
:1036680000F07D8406D8412B40F0AD854FF000086E
:1036780000F069BC442B00F018854A2B40F0A38564
:103688000BF028FBA08100F04BBDD12B00F0668326
:103698001FD8CC2B00F00C820ED8C82B61D004D8D0
:1036A8004E2B00F01D8400F08EBDC92B00F02F8337
:1036B800CA2B7DD000F087BDCE2B00F01B83C0F055
:1036C8001083CF2B00F04882D02B00F0FF8200F04F
:1036D8007ABDD82B00F001810BD8D32B3BD027D350
:1036E800D42B00F07D82D62B40F06D854FF000087A
:1036F8006BE2F22B00F0C28212D8EF2B40F0638508
:10370800DFF88C83D8F800A00BF0E4FAAAF85A0086
:10371800D8F800800BF0DEFAA8F8580000F000BDD9
:10372800F32B00F0C784FA2B00F0ED8200F04BBDBC
:103738002B7803F0040303F0FF08002B40F0F0841B
:103748000BF0BEFA022884F8A40740F2C582CC4BDD
:1037580083F8A487C0E20BF0BDFACA4B188000F0CA
:10376800DFBC92F805804FEA5808B8F1120F03D968
:1037780002F0EAFB00F0D4BC4FF0000AC24507D2C1
:103788000BF0A8FAC04B23F81A000AF1010AF5E772
:10379800BE4B012283F8342000F0C2BC0BF090FA33
:1037A80084F8DE010BF08CFA84F8DD0100F0B8BC77
:1037B800B74B1A681278022A4FF0000A984670D15F
:1037C800D8F800B00BF07CFA07EE900AF8EE677AAA
:1037D800B2EE048AC7EE887A0BEB8A0BCBED087A37
:1037E800D8F800B00BF06CFA07EE900A9FEDA97AB2
:1037F800F8EE677A0BEB8A0BC7EE877ACBED0B7A7C
:10380800D8F800B00BF05CFA07EE900A9FEDA27AA8
:10381800F8EE677A0BEB8A0BC7EE877A0AF1010A92
:10382800BAF1030FCBED0E7ACAD1BAF1070FD8F867
:1038380000B01CD10BF044FA07EE900AF8EE677A54
:10384800C7EE887ACBED117AD8F800B00BF038FAC9
:1038580007EE900AF8EE677AC7EE887ACBED127A0F
:10386800D8F800B00BF02CFA8BF84C0012E00BF0F3
:1038780027FAD3448BF80100D8F800B00BF020FAEF
:10388800D3448BF80B00D8F800B00BF019FAD344E6
:103898008BF815000AF1010ABAF10A0FC5D100F038
:1038A8003FBCD8F800B00BF00BFAD3448BF80100FA
:1038B800D8F800B00BF004FAD3448BF80B00D8F812
:1038C80000B00BF0FDF9D3440AF1010ABAF10A0F6E
:1038D8008BF81500E5D100F023BC8246DFF8B081F3
:1038E8009FED6D8AD8F800B00BF0F4F907EE900A56
:1038F800F8EE677A0BEB8A0BC7EE887ACBED087A7D
:10390800D8F800B00BF0E6F907EE900AF8EE677AFF
:103918000BEB8A0BC7EE887ACBED0B7AD8F800B0A0
:103928000BF0D8F907EE900AF8EE677A0BEB8A0BE2
:10393800C7EE887A0AF1010ABAF1030FCBED0E7AC5
:10394800CCD1BAF1070FD8F800B01CD10BF0C2F9EE
:1039580007EE900AF8EE677AC7EE887ACBED117A0F
:10396800D8F800B00BF0B6F907EE900AF8EE677ACF
:10397800C7EE887ACBED127AD8F800B00BF0AAF926
:103988008BF84C0012E00BF0A5F9D3448BF801003A
:10399800D8F800B00BF09EF9D3448BF80B00D8F898
:1039A80000B00BF097F9D3448BF815000AF1010A1F
:1039B800BAF10A0FC5D1B3E30BF082F91328834695
:1039C8003FF6D6AEDFF8C8A0DAF800800BF078F939
:1039D8000023324A0C2101FB0322117A814222D1B1
:1039E8000FFA8BFB08EB8B08137888F879300BF00B
:1039F80067F988F87A000BF063F988F87B000BF018
:103A08005FF9274B274A1A6088F87C00264BDAF8BA
:103A1800000018600021793007F0ECF9234B80F0A2
:103A2800010018707CE301331B2BD2D1A0E60BF008
:103A380047F90B2882463FF69BAE154BD3F800801A
:103A48000BF03EF903283FF693AE062303FB0A88E2
:103A580088F8CE000BF034F988F8C9000BF030F97B
:103A680088F8CA000BF02CF988F8CB000BF028F97D
:103A780088F8CC000BF024F988F8CD0050E300BF9B
:103A880048200020080F002024200020980F002044
:103A9800201000200000C84200007A44806201081B
:103AA800000F00208C210020040F002010000020AF
:103AB8005379092B7FF65CAE019BD3F800800BF09D
:103AC800FFF8019B88F80000D3F800800BF0F8F8A5
:103AD80088F801000BF0F4F8019B64281B68A8BF64
:103AE800642018710BF0ECF8019B64281B68A8BFD0
:103AF800642058710BF0E4F8019BFF281B68A8BFED
:103B0800FF2098710BF0DCF8019B6428D3F8008043
:103B180028BF642088F807000BF0D2F8019B88F8CA
:103B28000200D3F800800BF0CBF8019B88F8030063
:103B3800D3F800800BF0CEF8DAF80030A8F80A00C5
:103B48005B790A2B40F2EC82D74BD3F800800BF05C
:103B5800B7F888F80800E3E20BF0BCF86FF4AF623E
:103B680083189BB2C62B98BFA4F898010BF0B2F843
:103B7800A4F844010BF0AEF8A4F846010BF0AAF83B
:103B8800A4F848010BF0A6F8A4F8DA010BF098F8AD
:103B980084F8EB010BF094F80BF092F884F8EC0140
:103BA8000BF08EF884F887010BF08AF884F89401FA
:103BB8000BF086F8BD4BD3F800800BF08BF800EBC8
:103BC80080004000A8F856001BE10BF083F8B84BC2
:103BD80023F8180008F10108B8F1080FF5D19FE2A1
:103BE80053790F2B7FF4C4AD0BF06AF80728804691
:103BF8003FF6BEAD029BD3F800A00BF06BF80E2386
:103C080003FB08F8C244029BAAF81901D3F800A0E4
:103C18000BF060F8C244029BAAF81B01D3F800A07D
:103C28000BF058F8C244029BAAF81D01D3F800A073
:103C38000BF046F8C244029B8AF81F01D3F800A093
:103C48000BF03EF8C244029B8AF82001D3F800A08A
:103C58000BF036F8C244029B8AF82101D3F800A081
:103C68000BF02EF8C244029B8AF82201D3F800A078
:103C78000BF03AF8D044C8F8230151E20BF020F8D1
:103C88000F2880463FF674AD0BF01AF8C8EBC80849
:103C9800A04488F8D4000BF013F888F8D5000BF08E
:103CA8000FF888F8D6000BF00BF888F8D7000BF05F
:103CB80007F888F8D8000BF003F888F8D9000AF05C
:103CC800FFFF88F8DA0007F08DFC29E22B785B0704
:103CD80000F126820BF0D4FA03F042FA03F0FAFA64
:103CE8001EE22B78580700F11B82724B4FF4C87202
:103CF8001A8015E22B78590700F112826E4A137860
:103D080043F0040328E02B785A07E5D55BE20AF074
:103D1800D7FF694B1A7810B142F0020201E022F095
:103D280002021A700AF0CCFF644BDFF8B0811870F9
:103D38000AF0DAFFC8F800000AF0D6FFC8F8040055
:103D48000AF0C8FF5E4B18800AF0C4FF5D4B5E4A5C
:103D58001880137843F002031370E1E10AF0B0FF12
:103D680003900AF0C1FF83460AF0BEFF82460AF0BC
:103D7800BBFF80460AF0AEFF0AF0ACFF0AF0A0FFD6
:103D8800039BA3B9514B1020C3F800B0C3F804A09B
:103D980003F093F9484A137843F001031370B8F11C
:103DA800000F00F0BD814A4BC3F80080B8E1102B2A
:103DB80040F0B681474BC3F800B0C3F804A0B8F18F
:103DC800000F02D0424BC3F800804248424B022207
:103DD800011D1A7008F092F9A2E1A0600AF084FFB0
:103DE800A3681843A0609BE10AF074FFA4F85C0183
:103DF8000AF070FFA4F85E010AF06CFFA4F86001F5
:103E08008EE10AF05DFF84F87C010AF059FF84F81E
:103E180080010AF055FF84F87F010AF051FF84F809
:103E280081017DE10AF056FFA4F882010AF052FFF1
:103E3800A4F884010AF044FF84F886010AF04AFFD6
:103E4800A4F888016CE10AF03BFF84F892010AF0BB
:103E580041FFA4F89C010AF03DFFA4F898010AF07C
:103E680039FFA4F89A010AF02BFFDAF8003084F839
:103E780093015B79082B40F253810AF02BFFA4F8D9
:103E88009E010AF027FFA4F8A00149E10AF018FFF3
:103E980084F8D8010AF014FF84F8D9010AF01AFF4F
:103EA800A4F8DA013CE100BF4010002020100020F7
:103EB800961F0020C60E0020D4100020DA10002023
:103EC800D8100020D61000204610002048100020EE
:103ED80058100020501000200C0F0020DC1000208B
:103EE80092F805800323B8FBF3F8B8F1120F3FF6F8
:103EF8003FACDFF8FCA34FF0000BC34580F0108106
:103F08000AF0DEFE8AF8A2010AF0E4FE40F2ED2390
:103F1800984205DD40F6CA039842A8BF184601E05A
:103F280040F2EE20A0F2EE2019230BF1010B90FBDA
:103F3800F3F00AF1020A8AF8A101DEE70AF0C0FEEE
:103F480084F89401ECE00AF0BBFE04EB080308F1E6
:103F58000108B8F1080F83F88A01F4D1E0E00AF00B
:103F6800AFFEC4F808B060710AF0BEFEA36818433B
:103F7800A0600AF0A5FE84F892010AF0ABFEA4F84E
:103F88005C010AF0A7FEA4F85E010AF0A3FEA4F8FB
:103F980060010AF09FFEA4F882010AF09BFEA4F8D3
:103FA8008401BDE053794FF0070AB3FBFAF2C2EB84
:103FB800C2029A1A12F0FF0F7FF4DAABB3FBFAFAD7
:103FC8000AF1FF3A5FFA8AFABAF1FF0F00F0A88007
:103FD8000AF076FE5FFA80FB4FFA8BF006F03AFEA5
:103FE800804600283FF4C4AB80F800B00AF072FEA7
:103FF800A8F802000AF064FE88F804000AF060FEDF
:1040080088F805000AF05CFE88F807000AF058FEF8
:1040180088F80600D4E7DFF8D88208F1400A0AF0E9
:1040280059FEA8F89C020AF04BFE88F89E020AF096
:1040380047FE08F1040888F89B02D045EFD16FE0ED
:104048000AF03EFE1F2880463FF692ABD9F80030B2
:104058005B79082B7FF48CAB0AF03CFE08F18608EC
:1040680004EB880800F03F00A8F806000AF032FECA
:10407800B8F80630800100F4FE501843A8F806008E
:104088000AF01EFE000188F804000AF019FE98F8EC
:10409800043000F00F00184388F804000AF010FEFE
:1040A80088F805000AF018F93AE07D4B012283F8F8
:1040B800352035E00AF004FEFF2882461BD1002394
:1040C8008DF81F309DF81F30052B29D89DF81F004B
:1040D800744A9DF81F3052F8300002EBC3030121E7
:1040E8005B68994089B2042204F018FD9DF81F30DE
:1040F8000133DBB2E4E705283FF63AAB00200AF0CB
:1041080031FE0AF00BFED8F8000007F0BFF818B926
:10411800322006F0CEFEF6E74FFA8AF004F00CFDE6
:1041280000200AF01FFEFFF7A6B95F4B985907F069
:10413800ADF818B9322006F0BCFEF6E707F012FA1F
:1041480002F0E4FF594B5A4ADA60FFF7A1B90C288C
:104158003FD00A2841D1574D57480AF08BFE2846D0
:10416800232110F0CAF908B1401B20602368002BF6
:1041780036D1504823600021302210F088F93B786E
:10418800002B60D14D4B1B689B0615D54C4B444901
:104198001B688A6B9A1A002A0EDB4A4A1278042A8C
:1041A8000AD9494A03F5123303F5F8738B63938AE6
:1041B8009BB283F488439382444B9B68002B69D05D
:1041C8004348984766E001F0BFFEFFF754B90C2852
:1041D80047D140480AF04EFE35E00D2835D1BAE700
:1041E8005A1EA95C202901D11346C0E7314A236031
:1041F8000021D154384B394DD3F800A0D5F800B080
:10420800DFF8B090584610F086F906463246484620
:10421800594610F089F9324A28B919F8063053443A
:104228005B78580703D010359542E7D306E09542EE
:1042380004D2701CEB684844984702E029480AF009
:1042480019FE002395E7284807E07F280DD1013B98
:10425800184A264823600021D1540AF00BFEFFF7C4
:1042680076B87F2804D1FFF772B82F2B3FF66FA8D6
:10427800A0F12002D2B25E2A3FF669A813B920281D
:104288003FF465A85A1C22600A4AD0540AF0EAFD95
:10429800FFF75DB809B0BDEC028BBDE8F08F00BF39
:1042A800980F002084850108AC11002000ED00E083
:1042B8000400FA05E41C00204B8F0108D0100020F0
:1042C800DC2B0020DA100020001000483C280020D9
:1042D800B2100020B881010820010020386A0108C6
:1042E800F86B0108C3810108B3810108DF81010867
:1042F800482000202DE9F0474D282DED028B04467B
:1043080000F0598600F2B980302800F0C08651D8F4
:10431800222800F0978423D8032800F0018214D8BB
:10432800012800F0F181022840F0FF8604200AF0FD
:1043380019FD43200AF0E1FC4C200AF0DEFC46207F
:104348000AF0DBFC4C2000F05CBE042800F0F18190
:10435800052840F0EA861A200AF004FD0024F8E156
:10436800282800F0E78515D8242800F0CE852628CF
:1043780040F0DB86D84C06200AF0F4FCB4F85C0167
:104388000AF0F3FCB4F85E010AF0EFFCB4F860013F
:1043980000F0B8BD2C2800F0E0852E2800F06186DA
:1043A8002A2840F0C28601200AF0DCFCCA4B587962
:1043B80000F027BE3D2800F0F5821ED8362800F010
:1043C80031860BD8322800F01686342840F0AD86A6
:1043D80048200AF0C7FC002500F056BC3A2800F037
:1043E800B7823B2800F02784382840F09E860420B6
:1043F8000AF0B8FCB84C00F08EBD452800F0828663
:1044080027D8402800F00086422840F08E86B24C1B
:1044180010200AF0A7FC60790AF06FFCA0680AF087
:10442800ADFC94F892010AF068FCB4F85C010AF05B
:104438009CFCB4F85E010AF098FCB4F860010AF03C
:1044480094FCB4F882010AF090FCB4F8840100F0FE
:1044580059BD492800F0B1824B2800F09D854628B7
:1044680040F063860D200AF07DFC00200AF045FC30
:1044780000200AF083FC00F050BE702800F0F082A3
:1044880000F2DD80692800F0438200F2AF806628E0
:1044980000F09D8100F29F80642800F073816528F8
:1044A80040F043868D4C0B200AF05CFC20880AF013
:1044B8005CFC62688A4B9A420CBF2089608980B292
:1044C8000AF053FC874B1B68C3F3C000C3F3800298
:1044D800800040EA4200C3F340021043C3F3401295
:1044E80040EAC20003F0100318430AF03EFC7E4B7A
:1044F8001A88E36812F0010F14BF4FF0020C4FF056
:10450800000C12F0020F02F0080814BF4FF0040E5E
:104518004FF0000E03F4475912F0040F14BF102790
:10452800002749EA080912F0400F03F4804814BF35
:104538002026002649EA080912F0100F03F4004863
:1045480014BF4FF40075002549EA080912F0200F3E
:1045580003F4803814BF4FF48060002049EA08094A
:1045680012F4807F03F4003814BF4FF40061002177
:1045780049EA080912F4007F03F480285B4A49EAF3
:10458800080903F4002849EA0809127803F4801896
:1045980049EA080903F0007349EA0303C2F38002F9
:1045A80043EA020343EA0C0343EA0E0E4EEA070706
:1045B80046EA070645EA060540EA050041EA000121
:1045C80014BF4FF400184FF00008002041EA080813
:1045D8000346217CE6E0672800F02181682840F046
:1045E800A48510200AF0BEFB002488E16C2800F0A6
:1045F800A28117D86A2800F00B846B2840F09585B3
:1046080005200AF0AFFB3A4B18880AF0AEFB394B8D
:1046180018880AF0AAFB314B93F86E0000F00100ED
:1046280000F0EFBC6E2800F0978100F2CC810620E4
:104638000AF098FB00200AF0A1FB00F062BC782881
:1046480000F0FA8018D8742800F03F830AD872283E
:1046580000F09E83732840F0688508200AF082FBEA
:104668000124CEE3762800F0F38300F267832F203D
:104678000AF078FB204CD6E2A42800F00F8414D866
:104688007B2800F07682A02840F04F850C200AF0A5
:1046980069FB1A4B18680AF071FB194B18680AF085
:1046A8006DFB184B186800F03CBDF12800F0008144
:1046B800FE2800F01A84F02840F03785074C0420C3
:1046C8000AF050FBA36CB3F85A000AF04EFBA36C37
:1046D800B3F8580000F016BC48200020D80F00207E
:1046E80000540040D010002098110020FD2B00201D
:1046F8004E110020501100204F620108ACF7FF1F37
:10470800B0F7FF1FB4F7FF1F03200AF02BFB0020B0
:104718000AF0F3FA20460AF0F0FA0C2000F071BC17
:104728000AF020FB01200AF0E8FA0A200AF0E5FA6C
:10473800B2E306200AF016FB53200AF0DEFA442002
:104748000AF0DBFA46200AF0D8FA33200AF0D5FA44
:10475800D7E3B24B185D01340AF0CFFA0B2CF8D12D
:104768000024AF4B185D01340AF0C7FA082CF8D1C1
:104778000024AC4B185D01340AF0BFFA072CF8D1BD
:1047880000F0D1BC07200AF0EDFAE7200AF0B5FAEC
:10479800A54B58790AF0B1FA00200AF0AEFA0420C5
:1047A80000F0BFBC8B420BD2A04A9C5C012202FAEB
:1047B80004F414EA080F1CBF9A4010430133F1E7D0
:1047C8000AF0DCFA984B93F8A40700F01ABC122000
:1047D8000AF0C8FA964B1B88B3F5806F8CBF082582
:1047E80001250024934B33F9140090FBF5F00134B4
:1047F80080B20AF0BAFA032CF4D18F4CA08D0AF0DB
:10480800B4FAE08D0AF0B1FA208E0AF0AEFA608EA2
:104818000AF0ABFAA08E0AF0A8FAE08E72E3102034
:104828000AF0A0FA0024854B185D01340AF065FAF5
:10483800102CF8D100F077BC70200AF093FA00260B
:104848007D4D0E24AB6C744323440136B3F8190133
:104858000AF08BFAAB6C2344B3F81B010AF085FA13
:10486800AB6C2344B3F81D010AF07FFAAB6C234408
:1048780093F81F010AF041FAAB6C234493F8200126
:104888000AF03BFAAB6C234493F821010AF035FA9D
:10489800AB6C234493F822010AF02FFAAB6C1C444A
:1048A800D4F823010AF06AFA082EC9D100F03BBCFB
:1048B80070205D4C0AF056FA04F1700594F8D400A3
:1048C8000AF01BFA94F8D5000AF017FA94F8D60003
:1048D8000AF013FA94F8D7000AF00FFA94F8D800FF
:1048E8000AF00BFA94F8D9000AF007FA073494F89A
:1048F800D3000AF002FAAC42E0D100F014BC504BED
:10490800185D01340AF0F9F9102CF8D100F00BBC4D
:104918004C4D2878400000F0FE000AF023FA0024ED
:104928002B789C4280F0FF83474B33F814000AF041
:104938001CFA0134F4E7454C06200AF013FA2088E3
:104948000AF013FA60880AF010FA414B1888D9E285
:1049580004200AF007FAE3E307200AF003FA3D4BC4
:104968001888FF28A8BFFF20C0B20AF0C6F93A4B42
:10497800186880F3100080B20AF0F7F92E4BB3F8EC
:1049880064000AF0F2F9284B93F88721334B186832
:1049980022B10A23584380F3100001E000F30F000E
:1049A80080B2AFE2204C02200AF0DCF994F8DE0174
:1049B8000AF0A3F994F8DD0123E302200AF0D2F902
:1049C800194B98899EE21C4C0B200AF0CBF9A36E78
:1049D80018780AF092F9A36E58780AF08EF9002632
:1049E8002546AB6E144C3344013618790AF085F924
:1049F800032EF6D1A36ED8790AF07FF9A36E9878C2
:104A08000AF07BF9A36ED8780AF077F9A36E588973
:104A18000AF0ABF9A36E187AF3E200BFF07E010842
:104A2800FC7E0108D17E010848200020E90F002003
:104A380012000020AA100020D80F0020101000201B
:104A4800241000204812002024200020E01F00200D
:104A5800B0100020C0100020CC100020C81000208A
:104A6800C64C1E200AF07EF9A36C1B78022B4FF06F
:104A780000056BD1A36C03EB850393ED080AB2EE36
:104A8800048A20EE080A0FF011FF80F30800C0B274
:104A98000AF033F9A36CDFEDBA7A03EB850393EDE3
:104AA8000B0A20EE270A0FF001FF80F30800C0B2BE
:104AB8000AF023F9A36CDFEDB37A03EB850393EDDA
:104AC8000E0A20EE270A0FF0F1FE80F30800C0B2AC
:104AD80001350AF012F9032DCCD1072DA36C23D18F
:104AE80093ED110A20EE080A0FF0E0FE80F30800AB
:104AF800C0B20AF002F9A36C93ED120A20EE080A7C
:104B08000FF0D4FE80F30800C0B20AF0F6F8A36CE8
:104B180093F84C3000EE103AB8EE400A0FF0C6FE9B
:104B280080F30800C0B20BE02B4458780AF0E5F88F
:104B3800A36C2B44D87A0AF0E0F8A36C2B44587D78
:104B480001350AF0DAF80A2DC7D1ECE2A36C2B4440
:104B580058780AF0D2F8A36C2B44D87A0AF0CDF82A
:104B6800A36C2B440135587D0AF0C7F80A2DEDD106
:104B7800D9E23C200AF0F6F80024804D9FED818AA6
:104B8800AB6C03EB840393ED080A20EE080A0FF0E0
:104B98008DFE80B20AF0E9F8AB6C03EB840393ED69
:104BA8000B0A20EE080A0FF081FE80B20AF0DDF849
:104BB800AB6C03EB840393ED0E0A20EE080A0FF0AA
:104BC80075FE013480B20AF0D0F8032CD5D1072C39
:104BD800AB6C16D193ED110A20EE080A0FF066FEB1
:104BE80080B20AF0C2F8AB6C93ED120A20EE080A04
:104BF8000FF05CFE80B20AF0B8F8AB6C93F84C008A
:104C08000BE0234458780AF0B0F8AB6C2344D87A08
:104C18000AF0ABF8AB6C2344587D01340AF0A5F8D0
:104C28000A2CD4D17FE214F8010F002800F07B820F
:104C38000AF063F8F7E701200AF094F84F4B9B6CF1
:104C48001878DEE150200AF08DF800254B4B9C6C5B
:104C58004D4B04EB85040C2194F8792001FB0233B9
:104C6800013593F838000AF048F894F87A000AF009
:104C780044F894F87B000AF040F894F87C000AF0B5
:104C88003CF8142DE2D14EE23C4B9C6C062303FB0E
:104C98000544013594F8CE000AF02FF894F8C900BD
:104CA8000AF02BF894F8CA000AF027F894F8CB0019
:104CB8000AF023F894F8CC000AF01FF894F8CD0015
:104CC8000AF01BF80C2DDFD12DE24FF00008012669
:104CD80000272A4B1A7C974227DA11330024FA5C02
:104CE800294D0C2305F130016343595C914207D1EA
:104CF8002B44586B0FF00FFC82462EB9B14605E0E5
:104D080001341B2CECD10EE080440CE0D1450ADACA
:104D18000C2303FB04535B6B13F8090009F0EDFF48
:104D280009F10109F2E70137D3E7002E00F0FB8112
:104D38005FFA88F00AF016F80026C9E70F4D287CBC
:104D48000AF010F800242B7C9C4280F0EC810F4B79
:104D5800E65C00210C480C2200F1300702FB01F34D
:104D6800DA5DB24205D1034493F8380009F0C5FF73
:104D780002E001311B29EDD10134E4E7D80F00200E
:104D88000000C84200007A4450620108E90F002080
:104D9800D14C162009F0E6FFB4F8980109F0E5FFB8
:104DA800B4F8440109F0E1FFB4F8460109F0DDFF69
:104DB800B4F8480109F0D9FFB4F8DA0109F0D5FFD1
:104DC80094F8EB0109F099FF002009F096FF94F898
:104DD800EC0109F092FF94F8870109F08EFF94F82E
:104DE800940109F08AFF002009F087FFBB4B9B6CF8
:104DF8000A20B3F9563093FBF0F080B209F0B5FF02
:104E080089E0E0B2013409F078FF092CF9D18AE190
:104E1800102009F0A7FFB24BB24C187800F002003E
:104E280009F06BFFB04B187809F067FF206809F0AC
:104E3800A5FF606809F0A2FFAC4B188809F095FF40
:104E4800AB4B188809F091FFA44BB3F86C0059E0FC
:104E580009F036FF0746122009F084FF9F4C17B966
:104E6800266F656F05E0102F13BF0025A66FE56F4D
:104E78002E46384609F041FF304609F07FFF2846A4
:104E880009F07CFFD4F8800009F078FF002009F0D1
:104E98006CFF002009F069FF0020B2E08F4D95F803
:104EA800840080000130C0B209F05CFF95F88400EE
:104EB80009F023FF00242E4696F884309C4280F0A7
:104EC80032818C4D285D09F018FF05F11003185D3B
:104ED80009F013FF05F120033035185D09F00DFFC7
:104EE800285D09F00AFF0134E6E7082009F03AFFD7
:104EF800002009F03AFF002009F037FF002009F0F0
:104F080034FF002009F031FF0DE1042009F02AFFE9
:104F1800714B986805E194F87C0109F0EEFE94F86D
:104F2800800109F0EAFE94F87F0109F0E6FE94F8A2
:104F3800810166E0684C072009F014FFB4F882018B
:104F480009F013FFB4F8840109F00FFF94F8860103
:104F580009F0D3FEB4F88801D4E75F4C0C2009F0BF
:104F680001FF94F8920109F0C8FEB4F89C0109F019
:104F7800FCFEB4F8980109F0F8FEB4F89A0109F0BB
:104F8800F4FE94F8930109F0B8FEB4F89E0109F014
:104F9800ECFEB4F8A001B5E74F4C042009F0E2FE9E
:104FA80094F8D80109F0A9FE94F8D90109F0A5FEF2
:104FB800B4F8DA01A6E7504C504D207800EB4000D9
:104FC800C0B209F0CFFE002623789E4205F1020503
:104FD80080F0A98015F8020C09F08FFE15F8010C75
:104FE80000EB800000EB800000F2EE2080B209F0B8
:104FF800BCFE0136E8E7012009F0B4FE364B93F811
:10500800940109F07AFE8EE0082009F0ABFE002436
:10501800314B2344013493F88A0109F06EFE082CC1
:10502800F6D180E02D4B2C4C93F8C500C0EBC000A6
:10503800C0B209F097FE04F11805314A94F8F2015C
:1050480092F9001043B2994271D092F90C1099422A
:105058006DD092F918209A4269D00834AC42ECD14C
:1050680061E040201C4C09F07DFE04F14005B4F8D5
:105078009C0209F07AFE94F89E0209F03EFE043480
:1050880094F89B0209F039FEAC42F0D14BE0E020E5
:10509800114C09F067FE04F18005B4F81E0200F017
:1050A8003F0009F062FEB4F81E02C0F3861009F052
:1050B8005CFE94F81C02000909F01FFE94F81C021B
:1050C80000F00F0009F019FE043494F8190209F0F1
:1050D80014FEAC42E1D126E048200020D80F002081
:1050E800D4100020DC100020DA100020D810002096
:1050F800D61000205D10002048120020EA21002070
:1051080054120020132009F02DFE0024154B185DC1
:10511800013409F0F2FD0B2CF8D1002009F02EFE25
:10512800002009F02BFE012018E0002016E009F00D
:10513800E4FDB4F8F40109F018FE94F8F60109F05A
:10514800DCFD94F8F70109F0D8FD94F8F90109F0AD
:10515800D4FD94F8F80109F0D0FD7EE7BDEC028B90
:10516800BDE8F087F07E01082DE9F047B94CBA4E4A
:10517800237886B00746002B00F0F2813268636816
:10518800D31A7C2B40F2EC81237A626001332372BC
:10519800002505F12400DFF8BC82C0B20CF058F8F5
:1051A80008F10A0333F9153007EE903AAB4B1B8828
:1051B800B8EEE77A07EE903AF8EEE77A0135C7EEEF
:1051C800277A9FEDA77A67EE877AFDEEE77ACDED2D
:1051D800037ABDF90C000CF029F8032DD9D1302041
:1051E8000CF036F800200CF021F80CF029F898F8AB
:1051F800085015F0030520D1D8F8042041F288336F
:105208009A420BD910200CF023F828460CF00EF81F
:1052180021200CF01DF828460CF008F814200CF09A
:1052280017F8B4F910000CF001F81C200CF010F875
:1052380000200BF0FBFF0CF003F8237ADFF8148250
:105248005B0740F06A8102200CF002F80A23B8F9E3
:10525800120090FBF3F00BF0E9FF0320B8F91A50A5
:10526800DFF810920BF0F4FF7E4B1B7813F0040F5D
:105278004FF0050A95FBFAF5ADB20BD038460AF0A7
:1052880021FE28B9D9F8003013F0100F18BF0025F7
:1052980028B205E0D8F81C309889B0FBFAF000B2C3
:1052A8000BF0C4FFD9F800309F0740F18180DFF888
:1052B800C891678C99F80030228C664D3F014FF0F9
:1052C8006408BFB208FB02325B00B2FBF3F347EAA3
:1052D8000327BFB2C3F303231F4306200BF0B8FF15
:1052E80038B20BF0A3FF638C99F8001001339BB21E
:1052F80093FBF1F201FB12336384636A9B7B012BFE
:1053080005D139200BF0A4FFB5F9200019E02D8C48
:105318006E233A205D4315270BF09AFF95FBF7F5AE
:10532800AFB2B7FBF8F528B20BF080FF08FB157594
:105338003B200BF08DFFA8B2451D0A2095FBF0F02D
:1053480000B20BF073FF28200BF082FFA36A414DD7
:105358000A2093FBF0F000B20BF068FF04200BF07A
:1053680077FFE369E86A9A894FF6FF739842A8BF06
:105378001846C2B10028ACBF131A134607EE903A7C
:105388009FED397AF8EEE77A67EE877A07EE102A0A
:10539800B8EEC77AC7EE877AFDEEE77A17EE900A7D
:1053A8006428A8BF642020EAE07000B20BF03EFF3A
:1053B800236B284F9D0640F1A58097F83430980755
:1053C8001BD511200BF044FFF88E284B4FF4F365E2
:1053D800684390FBF3F000B20BF028FF19200BF0A4
:1053E80037FFF88E4543642095FBF0F595FBF0F305
:1053F80000FB135000B20BF019FF94F83430258FDE
:1054080013F0020F08BF002501200BF021FF28B27E
:105418000BF00CFF09200BF01BFF00200BF006FF20
:10542800134B94F83A501A88B2F5967F0AD9094B6B
:105438001B7A03F00F03072B04D842F20F7595422D
:1054480028BF154605200BF003FF636A5B7BBBB9D9
:1054580028B232E0A01000200C200020120000200A
:1054680000007A44FD2B00200000C842A0860100FD
:1054780012010020E81F0020100100206666E63FA8
:10548800A5F1200307EE903A1FED047AF8EEE77ACB
:10549800F6EE006AC7EE877ABEEE007AF5EEC07ABD
:1054A800F1EE10FA58BFB0EE667A77EE877AFDEE25
:1054B800E77ACDED037ABDF90C000BF0B7FE94F84E
:1054C8003420C34B910703D493F83B20012A04D11D
:1054D800012384F83B30BF481BE05B6ADFEDBE6AFE
:1054E80093ED017AD3ED027A27EE267A67EEA67A53
:1054F800BDEEC77AFDEEE77A8DED047ACDED057A3B
:1055080004A806E0B54A92E8030004AB83E8030068
:10551800184602F0B5FD0BF093FE237A282B1FD115
:10552800AB4B00221A723C2733684FF47A70B3FBF6
:10553800F0F817200BF08CFEB8FBF7F5B5FBF7F089
:1055480007FB1050000200B20BF070FE18200BF0A1
:105558007FFE07FB158000B20BF068FE0BF070FEB3
:1055680094F844309A4D002B00F0578105F07CFCEC
:10557800AB6C9B4AC31A9342074640F2BC80002397
:1055880085F84E3085F850302B8CDAB21B0A85F836
:105598006A2085F86B3085F8602085F86130AA6F3D
:1055A80033689A1AEB6FD97B4FF47A734B439A425C
:1055B8000DD38C4B1B68AB6795F88030013B012BF2
:1055C8009FBF102385F84E30022385F850300A20FB
:1055D800A26A92FBF0F284F86820121284F869201B
:1055E80094F83420E36A93FBF0F384F86C301B12D0
:1055F80084F86D30920794F83A30754984F89B30F6
:1056080003D42D2381F89C3074E0042BD4F83C900B
:10561800266CDFF8E081744A8CBF3323322381F88B
:105628009C304FF0060C714B99FBF3F096FBF3F3AB
:1056380008FB009108FB036803EB83030CFB01F1F3
:1056480003EB830391FBF2FE642502FB1E119B0012
:1056580091FBF5F184F88D1009120CFB08FC84F815
:105668008E109CFBF2F143FA81F39BB202FB11C24C
:1056780092FBF5F284F89220121284F8903084F8A4
:1056880093201B0AE28E84F891302423534393FB22
:10569800F5F5B4F8AE3084F8943000EB80001B0ABE
:1056A80000EB8000800084F895300A22238FB3FB3A
:1056B800F2F303F5FA739BB240FA8EF080B284F8E5
:1056C80096301B0A4FEAD97984F88B00F60F000A46
:1056D80084F8885084F89730C5F30725B4F8B030BB
:1056E80084F88A9084F88C0084F88F6084F8895054
:1056F80084F89D30A76494F8B280354DB8F1000F56
:105708000DD1D5F8B80005F0CAFD012807D902283F
:10571800374E00F0458202F0A5FC0123B370D4F89F
:10572800BC202B4D002A78D095F8B2603EB1D5F850
:10573800C43040F6B731FB1A8B4219D86DE001230B
:10574800D5F8B80085F8B23003F08DFAD5F8C8302E
:1057580093F9000002238DE84800082132464FF4EF
:10576800964305F0B0FB85F8CC60C5F8B80052E068
:1057780095F8C060CEB9D5F8B800C5F8BC6085F812
:10578800B26003F070FAD5F8C83093F9000001232D
:105798008DE84800082132464FF4964305F093FB04
:1057A800C5F8B80002F05EFC35E0013EF6B285F8B7
:1057B800C06095F8CC1095F8CD30EEB94A1C01338D
:1057C80085F8CC2085F8CD30D5F8B80021E000BFA9
:1057D800A0100020DC1000208096184BD063010830
:1057E8003F0D03000C20002040420F0080969800D7
:1057F80012000020806967FF12F8016BC5F8BC2011
:10580800701885F8CC000133D5F8B80085F8CD308C
:10581800314605F047FDC4F8C47094F8CE30954D74
:10582800DBB1D5F8D030C3B1D5F8D430ABB1C5F8B9
:10583800D8301B68904AC5F8DC30D5F8E0301344FE
:10584800187AFEF757FD09F069FAD5F8E030013308
:10585800092B88BF0023C5F8E030884D94F8E42070
:105868002E68844B002A00F0D581D3F8E820002A5E
:1058780000F0D08193F8EC30013B012B00F2CA8193
:10588800D4F8E8007B4F05F00AFDE0B1D7F8E8004E
:1058980005F002FD97F8ED30D5F800907E2B804694
:1058A8000ED102231B2887F8EC3009D1D7F8E8007D
:1058B80005F0F5FC20B90123C7F8F09087F8F4301B
:1058C80084F8ED80DCE7D7F8F0202B689B1A41F6C6
:1058D800583293421DD9032387F8EC309AE1684A7D
:1058E80032F8130010B903464FF403600133B0F5E2
:1058F800C06FDBB269D01DD9B0F5006F6ED030D95A
:10590800B0F5036F3BD184F8F530236B594F9A06F5
:105918003CD494F8F41094F8F530002900F03D8157
:105928002A68921B012ADAD984F8F530002384F812
:10593800F4306FE1B0F5007F3ED006D8B0F5807F37
:105948007CD0B0F5887F79D0E7E7B0F5806F00F0BC
:105958009B80B0F5826F00F0E080B0F5047FDCD169
:1059680020E0B0F5E26F78D0B0F5E46F7AD0B0F50A
:10597800E06FD2D184F8F530B4F90A1076E0B0F5CA
:10598800046F63D0B0F5026FC7D1F1E097F83430F7
:105998009B07BED5F98E24234B431233642193FB16
:1059A800F1F1F4E084F8F530364B324F1B68990773
:1059B800AFD53B8C0A21E9E084F8F530314B2D4F07
:1059C8001B681A05A5D5B96AE1E084F8F5302D4BB6
:1059D800284F1B681B059CD5F96AD8E0216B254A1E
:1059E80084F8F530880694D592F83410890790D554
:1059F800DB0711D5136C83EAE371002BA1EBE3718C
:105A080001EB51014FF01902B1FBF2F1ACBF41F0CB
:105A1800004141F040410EE0D36B83EAE371A1EB12
:105A2800E371002B01EB51014FF01902B1FBF2F1C8
:105A3800B8BF41F080414FF4006088E084F8F53049
:105A4800236B5F077FF565AF00215FE0B4F91010A5
:105A580084F8F5306423594379E084F8F530B4F9D3
:105A68000C1003E0B4F90E1084F8F5302C2391FBE8
:105A7800F3F16CE0A0100020D06301080C20002096
:105A8800F6820108E81F002084F8F53094F8F63013
:105A9800624A0133DBB2032B88BF012382F8F63058
:105AA80094F8F61042F2107359435D4B1B78D807EF
:105AB80048BF01319A0748BF02315F07B4F8F83090
:105AC80048BF0431D80748BF0A319A0748BF143184
:105AD8001F0648BF2831D80548BF28315A0748BF94
:105AE80064311F0748BFC831980548BF01F5C87120
:105AF8009A0648BF01F57A71DF0648BF01F5FA61D9
:105B0800580648BF01F57A614FF4806002F076FAD2
:105B1800424B002283F8F420FBE6216BDFF8FC807F
:105B280084F8F53011F0200717D098F8342012F0D7
:105B3800020F14BF4FF47A71002112F0010F14BF45
:105B48004FF4FA6300230B4494F83A10194402F016
:105B580055FA002384F8F430DBE6324B1B6819064B
:105B68007FF5D7AE394602F049FA88F8F470D0E6E6
:105B780084F8F530236B294F9A067FF5CAAE97F85B
:105B880034309B077FF5C5AE3B8F6421594302F043
:105B980035FA002387F8F430BBE684F8F53039E0AD
:105BA800B37823B1C5F8B47086F80280B7E5D5F8A4
:105BB800B430FB1AB3F57A6FFFF4B1AD0123D5F811
:105BC800B800B37005F068FB0646D5F8B80005F0D4
:105BD80063FB76067FF4A3AD8A2802D08E280CD00A
:105BE8009DE52B6B99067FF59AAD95F8B230002BA1
:105BF8007FF495AD05F1810306E095F8B230002BEE
:105C08007FF48DAD05F14C03C5F8BC302D2385F824
:105C1800C03084E506B0BDE8F08700BFA0100020C2
:105C2800FD2B0020E81F0020704708B51F4A18B94F
:105C3800536802221A8208BD0020516810800B7830
:105C480013F07F030DD14B7A990644BF02211170DE
:105C580013F0400F137814BF43F0010323F001033E
:105C680015E0012B1FD0022B1ED14B7913F0800FAA
:105C780003F00F034FEA830303F1804303F5B843AE
:105C88001B6806D003F03003102B07D101231370D3
:105C980004E003F44053B3F5805FF6E793681B69AB
:105CA8009847024808BD104608BD00BFA011002053
:105CB80010B5064C18B9636801221A8210BDA36892
:105CC8009B68984760680C3010BD00BFA011002089
:105CD80010B5064C18B9636801221A8210BDA36872
:105CE8001B68984760680A3010BD00BFA0110020EB
:105CF800084BDA68D10709D4DA68D20608D4DB6819
:105D080013F0040F14BF03200420704701207047CC
:105D1800022070470020024010B50446B0F9000088
:105D280009F02DFEB4F9020009F029FEB4F90400C7
:105D3800BDE8104009F023BE10B50446006809F01C
:105D48001EFE606809F01BFEA068BDE8104009F05F
:105D580016BE2DE9F74F012004F0BCFF002488B3DC
:105D6800012C2FD8194E4FF04C0909FB04FA06EB09
:105D78000A0808F15407BD7815B10134E4B2EEE71A
:105D880090F9003090F804E01846114B03228DE892
:105D9800240001212A4653F82E3005F094F8834652
:105DA80060B106F10C00504429464A460EF06FFBDC
:105DB80001231C44C8F80CB0BB70E4B2012004F005
:105DC8006FFFCCE703B0BDE8F08F00BFA011002043
:105DD800E863010810B5184C002120461A220EF07D
:105DE80056FBA4F5F870142380F8F231052300223D
:105DF800042180F8F63180F8F83180F8FE3180F817
:105E0800003280F8063280F808325223012480F8E4
:105E1800F71180F8F92180F8FF1180F8012280F845
:105E2800071280F8092280F8F03180F8FA2180F80A
:105E38000242A0F8F44110BD3822002010B5FFF747
:105E480057FF4FF43024012806D11CB1FFF750FF4B
:105E5800013CF8E7052010BD002C08BF052010BD47
:105E680070B50646441E14F8011F89B1094D28462D
:105E78000EF043FB0028F6D005F1080398423FBF17
:105E8800054B401BC018A31B38BF80F88A31EAE7CE
:105E980070BD00BF1683010848200020031EB8BF4C
:105EA8002D2210B5B8BF58420C46B8BF01F8012BD7
:105EB8000A2200F0CDFE00230370204610BD07B56E
:105EC8001C4B03F1A802C3F8A4201B4A92F89221A4
:105ED8005AB1012A14D1032183F8AA10072183F8A3
:105EE800AC2083F8AB100C2208E0022183F8AA103A
:105EF800032183F8AC2083F8AB10072283F8A8208D
:105F08000E4B0F4A1A60402004F0E4FE70B10122E3
:105F1800002390F9000040218DE80C00094A4FF455
:105F2800E13304F0D0FF003018BF012003B05DF862
:105F380004FB00BFA011002048200020180000200A
:105F4800710D0108010F01080120002108F0ECBEC5
:105F5800F0B51C4A92F8AD30D2F8B05092F8B4704F
:105F680092F8C06092F8CCE0022B0ED805EBC3047F
:105F7800591CA31CC9B206D02346A48814F0010FEB
:105F880001D0204205D10B46EEE782F8AD30002063
:105F9800F0BD93F902307CB29C4201D1002307E0A6
:105FA80074B29C420CD04FFA8EF49C42EBD102237F
:105FB80082F8AD100C2101FB0322D2F8B800F0BD25
:105FC8000123F5E7A011002030B5002202F180532B
:105FD80003F5B8539B0042F400441D6840F60F7166
:105FE80044F08004294001322143042A1960EDD18C
:105FF800024B40F08000186030BD00BF4C5C004090
:106008002DE9F843324D6E68328A377ABAB9042FCF
:1060180015D130480378012B0CD12F4B19682F4B21
:1060280089B20B445B0019681A603023A5F8D83090
:10603800027049E01023A5F8D830072744E0B48A55
:10604800B369A24294BF04270227944228BF14468A
:106058001FFA84F8404698471F4A13689BB203F119
:10606800005303F540535B0004F1010E1B689BB21B
:1060780003F1005303F540534FEA6E0E5B00002115
:10608800714500F1020009D010F8019C10F802CC0B
:106098004CEA092C23F821C00131F1E712680F4BB3
:1060A80092B213445B001A681C60338AC8EB03037E
:1060B8003382738A98443023A5F8D8304FF440537C
:1060C800A6F81280A5F8DA306B681F72BDE8F8836D
:1060D800A0110020FE2B0020505C00400230002060
:1060E8000E4B0F4A1B689BB203EBC00002443E29CB
:1060F8004FEA420209D94B09C80604BF03F1FF332E
:106108009BB29B0243F4004304E04B08C90748BF15
:1061180001339B0211681360704700BF505C004058
:106128000630002008B50B4B002093F83010FFF71D
:10613800D7FF094B5A68107A082801BF4FF48052DC
:10614800A3F8DA201022A3F8D820A0F109035842B6
:10615800584108BD18000020A011002038B5444D52
:106168006A68107810F07F0004D1537A23F0200376
:10617800537238BD022879D15388002B77D113790F
:10618800002B74D1537923F08000840004F18041FE
:1061980001F5B84113F0800F096814BF01F0300110
:1061A80001F44051032861D800295FD0927A002A6F
:1061B8005CD004F1804404F5B8441906226825D55A
:1061C80002F03002102A4CD103F07F039B0003F148
:1061D800804303F5B8431A68510641BF196840F671
:1061E8000F720A4042F4004244BF42F0C0021A60F3
:1061F8001A6822F4E04222F0400292B282F03002A1
:1062080042F4004242F080021A602AE002F440524E
:10621800B2F5805F25D128B9164B93F83010FFF7F7
:106228005FFF11E09B0003F1804303F5B8431A6850
:10623800520441BF196840F60F720A4042F44042C6
:1062480044BF42F080021A60236823F4804323F09D
:1062580070039BB283F4405343F4004343F080033C
:106268002360AB685B699847002038BD022038BDC1
:10627800A011002018000020002303604360836001
:106288008381036143618361C36103624362836203
:1062980070478A68036810B50C6A14430A69144386
:1062A8004A6914438A691443CA6914434A6A1443FD
:1062B8008A6A23F4FF4323F07003224313430360E5
:1062C8008B8943600B6883604B68C36010BD0268AC
:1062D8004FF6FE731340036000230360436083603E
:1062E800C360294B984201D1284A27E0284B98429D
:1062F80001D1264A2AE0274B984201D1234A2DE0B2
:10630800254B984201D1214A30E0244B984201D1D3
:106318001E4A33E0224B984204D11C4A536843F486
:1063280070032EE01F4B984204D1184A536843F07B
:10633800706326E01C4B984204D11C4A536843F012
:106348000F031EE01A4B984204D1184A536843F0D1
:10635800F00316E0174B984204D1144A536843F4EB
:1063680070630EE0144B984204D1104A536843F40A
:10637800704306E0114B984204D10C4A536843F429
:1063880070235360704700BF0800024000000240BD
:106398001C00024030000240440002405800024005
:1063A8006C000240800002400804024000040240E1
:1063B8001C040240300402404404024058040240D5
:1063C800036A23F001030362036A70B544688269B3
:1063D8000D6822F4803222F0730215438A8923F073
:1063E800020313438A881343134A90420FD002F5DD
:1063F800006290420BD002F54062904207D002F54D
:106408008062904203D002F5806290420DD1CA8921
:10641800CE8823F0080313430A8A24F440741443F3
:106428004A8A23F00403334314438A68446085612D
:106438004263036270BD00BF002C01409D4A53684F
:1064480003F00C03042B2DE9F04105D0082B06D0EE
:1064580099490160B3B916E0974B036012E053689D
:106468005468C3F38343991CE30349BFD36A934B2E
:10647800914C03F00F0344BF0133B4FBF3F34B43D8
:10648800036000E0002351688D4FC1F303113944C4
:1064980091F834500168EDB221FA05F44460566869
:1064A800C6F302263E4496F8346024FA06FEC0F885
:1064B80008E05668C6F3C2263E4496F83460F6B241
:1064C800F440C460D2F82C80C8F3041808F00F0C0C
:1064D80007EB4C0C18F0100FBCF844C01FFA8CFCEA
:1064E80007D0BCF1000F04D0B3FBFCFCC0F810C00F
:1064F80000E00161D2F82CC0CCF3442C0CF00F085A
:1065080007EB48071CF0100FB7F84470BFB204D06F
:106518001FB1B3FBF7F7476100E04161176BFF0656
:106528005ABF654F87618161176BBF065ABF624FBB
:10653800C761C161176B7F065ABF5F4F076201626F
:10654800176BFF0506D5994204D1AE4202D14F0020
:10655800476200E04462176BFF0406D5994204D1F4
:10656800AE4202D14F00876200E08462176BBF051C
:1065780006D5994204D1AE4202D14F00C76200E06D
:10658800C462176B7F0506D5994204D1AE4202D189
:106598004F00476400E04464176B3F0506D59942F5
:1065A80004D1AE4202D14F00876400E08464176BC7
:1065B800BF0406D5994204D1AE4202D14B00C36450
:1065C80000E08464156B3B4BAD0701D1046315E013
:1065D8001C6B04F00304012C01D101630EE01C6B59
:1065E80004F00304022C02D14FF4004305E01B6BB6
:1065F80003F00303032B01D12F4B0363146B2D4BC3
:1066080014F4403F02D1C0F834E018E01C6B04F4E5
:106618004034B4F5803F01D1416310E01C6B04F4B1
:106628004034B4F5003F02D14FF4004306E01B6B41
:1066380003F44033B3F5403F01D11F4B4363146B60
:106648001C4B14F4402F02D1C0F838E018E01C6B42
:1066580004F44024B4F5802F01D1816310E01C6B51
:1066680004F44024B4F5002F02D14FF4004306E0AF
:106678001B6B03F44023B3F5402F01D10E4B83630A
:10668800146B0C4B14F4401F02D1C0F83CE021E01D
:106698001C6B04F44014B4F5801F01D1C16319E0E8
:1066A8001C6B04F44014B4F5001F0BD14FF40043E5
:1066B8000FE000BF0010024000127A0000093D0000
:1066C800180000201B6B03F44013B3F5401F01D1E1
:1066D800134BC363126B134B12F4400F03D1C0F872
:1066E80040E0BDE8F0811A6B02F44002B2F5800F79
:1066F80002D10164BDE8F0811A6B02F44002B2F5E0
:10670800000F02D14FF4004306E01B6B03F4400373
:10671800B3F5400F01D1024B0364BDE8F08100BF1F
:1067280000127A0000100240F0B500230E681C46E3
:106738000125A54005EA060EAE452BD10F797A1E34
:10674800012A15D8856803229A4025EA0202826048
:106758004D7982689D4015438560828892B222EA0D
:106768000E0282808A798588A2402A4392B282806A
:10677800032205689A40D2431540056005689F408A
:106788002F430760C7681740CA7902FA03F547EA3A
:106798000502C2600134102C03F10203C8D1F0BD18
:1067A80038B52DED048B4A4C0368C4F8DC30838877
:1067B800A4F8E030013A0D46072A42D8DFE802F093
:1067C800040A101822292F35B4F8DC300B80B4F8ED
:1067D800DE3013E0B4F8DE300B80B4F8DC3005E0CE
:1067E800B4F8DC305B420B80B4F8DE305B4205E085
:1067F800B4F8DE305B420B80B4F8DC306B80B4F860
:10680800E0301DE0B4F8DC305B420B80B4F8DE30D9
:1068180012E0B4F8DE300B80B4F8DC300CE0B4F8E9
:10682800DC300B80B4F8DE3005E0B4F8DE305B42D3
:106838000B80B4F8DC305B426B80B4F8E0305B422C
:10684800AB80244B93F86430002B3ED1B5F900306F
:1068580094ED3C0AD4ED397A09EE103AB5F90230D4
:1068680008EE103AB8EEC88AB5F90430B8EEC99AFD
:1068780028EE000A08EE903AA7EE890AF8EEE88AB0
:10688800D4ED3F7AA7EEA80A0EF010F894ED3D0A71
:10689800D4ED3A7A288028EE000AA7EE890AD4EDCA
:1068A800407AA7EEA80A0EF001F894ED3E0AD4ED5E
:1068B8003B7A688028EE000AA7EE890AD4ED417A6F
:1068C800A7EEA80A0DF0F2FFA880BDEC048B38BD36
:1068D800A01100201800002008B50A4890F80931D6
:1068E80000EB43030A22B3F8181189B2A0F820116B
:1068F80000F5947004F0D9FC80B20AF0C7FB024B93
:10690800188008BDA0110020C0100020F0B5012497
:10691800B0FBF4F58D4201D34C43F9E70026D4B11E
:10692800B0FBF4F504FB1500B4FBF1F41EB9002D1F
:1069380001DC002CF3D1092D03F1010EEFB204DDC7
:10694800002A14BF3725572500E030253D441D7027
:1069580001367346E3E71C70F0BDF0B50124B0FBC7
:10696800F4F58D4201D34C43F9E70026D4B1B0FBCE
:10697800F4F504FB1500B4FBF1F41EB9002D01DC9D
:10698800002CF3D1092D03F1010EEFB204DD002A2A
:1069980014BF3725572500E030253D441D700136CA
:1069A8007346E3E71C70F0BD03685A1C0260197057
:1069B80070472DE9F843089E002B07468846144681
:1069C80014BF4FF030094FF02009334613F8012B5C
:1069D8000AB9254603E0002CFBDD013CF6E7002D53
:1069E80004DD38464946C047013DF8E724EAE47427
:1069F8003546A01B284415F8011B11B13846C0477D
:106A0800F7E7BDE8F883024B186804F04BBC00BFF9
:106A1800C80F002090ED017A07EE901AB5EE407A83
:106A2800F1EE10FA01BFF8EEE77A9FED0E7A67EE05
:106A3800877AB7EE007A04BFC7EE277AC0ED017AED
:106A480090ED017AD0ED007A30EE877A30EE670A61
:106A5800C0EE870AE0EE807AB0EE670AC0ED007AF1
:106A6800704700BFDB0FC94010B50278202A0346E3
:106A780000F10100F9D0092AF7D02D2A03D10346E5
:106A8800BFEE000A04E02B2A08BF0346B7EE000A4F
:106A9800DFED387A1A46134612F8010BA0F13001DF
:106AA800CCB2092C0AD807EE101AB8EEC77AF2EE63
:106AB800046AA7EEA67AF0EE477AECE72E2816D1FC
:106AC800F2EE046A1146B0EE666A0B4611F8012B25
:106AD800303AD0B209280AD807EE102AB8EEC77A99
:106AE80087EE267A66EE866A77EE877AEDE71A7879
:106AF80002F0DF02452A35D15A782D2A02D1023315
:106B0800012004E02B2A14BF013302330020013B8B
:106B1800002213F8011F3039CCB2092C03D80A24FB
:106B280004FB0212F5E7B2F59A7F28BF4FF49A7278
:106B38001346B7EE007A072B05D9DFED0F6A083B3D
:106B480027EE267AF7E702F007032BB1F2EE046A84
:106B580027EE267A013BF8E7F0EE476A20B1C7EE48
:106B6800877A03E0F7EE006A67EEA67A20EE270A36
:106B780010BD00BF0000000020BCBE4C30B52DED9C
:106B8800028B87B0B0EE408A0C220021054603A88C
:106B98000DF07DFCB5EEC08ADFED2A7AF1EE10FA31
:106BA800CCBF38EE278A38EE678ADFED277A28EEE1
:106BB800278A6946FDEEC87A17EE904A84EAE4709F
:106BC800A0EBE470FFF76AF9002CACBF20232D235B
:106BD80068468DF80C300DF09EFC012807D1302353
:106BE8008DF80D308DF80E308DF80F300CE002283E
:106BF80005D130238DF80D308DF80E3004E00328D0
:106C080004BF30238DF80D30694603A80DF066FCEB
:106C180003A80DF080FC0338C4B2224603A9284615
:106C28000DF0A6FC00232B55284608490DF056FC0C
:106C380003AB284619190DF051FC284607B0BDECE6
:106C4800028B30BD6F12033A00007A442B8301088F
:106C580070B5064615460846B6FBF2F414B1204650
:106C6800FFF7F6FF05FB1464024B1B5D00F8013BC0
:106C780070BD00BF2D8301082DE9F04F814689B012
:106C88008A4616461C4600253178002900F0DD802A
:106C9800252902D00136484675E07278302A08BFA7
:106CA800B278A2F1300319BFB71C4FF0000BF71CE4
:106CB8004FF0010B092B4FF0000819D8A2F130034F
:106CC800D9B2092905D80A2202FB083817F8012B7E
:106CD800F4E7A2F16103052B02D8A2F1570305E0FE
:106CE800A2F14103052B03D8A2F137030A2BEADDF1
:106CF8006C2A31D13A78642A07F1010600F08380C2
:106D08000BD8252A3DD003D8002A00F09E80BBE787
:106D1800582A0CD0632A19D0B6E7732A22D002D891
:106D28006E2A37D0B0E7752A5CD0782AACD1271DF7
:106D38002068A2F1580462424FF01001624155E008
:106D48002CD9582A32D0632A2AD13E46484621787F
:106D5800271DD04701350FE0642A64D00ED9732A65
:106D680014D13E46236800934846514642460023C4
:106D7800FFF71FFE271D05443C4685E7252ADFD17E
:106D88003E4648462521D04701357DE70AD86E2A78
:106D980006D13E46236804341D6075E7002A54D0A6
:106DA8003E4671E7752A26D0782AF9D1A2F1580310
:106DB80004F1040C5A422068CDF80CC04FF01001C1
:106DC8005A4105ABFFF7A2FDDDF80CC03E4664460C
:106DD80005AB00934846514642465B46FFF7E9FD3E
:106DE800054451E72068271D0A21002205ABFFF75B
:106DF800B4FD3C46ECE704F1040CCDF80CC0206867
:106E08000A210022DDE72068002804F1040708DAD7
:106E18002D238DF8143040420DF115030A2100226C
:106E2800E5E705ABFAE72068002804F1040C0ADA64
:106E38002D238DF8143040420DF11503CDF80CC008
:106E48000A210022BEE705ABF8E7284609B0BDE8ED
:106E5800F08F0FB413B50B4904AB08680A4953F80F
:106E6800042B09680193FFF707FF0446074B1868CE
:106E780004F00CFA0028F9D0204602B0BDE8104012
:106E880004B070479401002090010020C80F002032
:106E980080EAE073A3EBE0738B4206DB002801DD98
:106EA800401A704702D00844704700207047FDEE32
:106EB800C07A17EE903A2033402B43D8DFED237A7F
:106EC800B4EEE70AF1EE10FA04DDDFED217A30EED8
:106ED800670AF3E7DFED1F7AB4EEE70AF1EE10FA7E
:106EE80004D5DFED1B7A30EE270AF3E7DFED1A7AD7
:106EF800B4EEE70AF1EE10FA04DD30EE670A37EE79
:106F0800C00A0AE09FED157AB4EEC70AF1EE10FA4E
:106F180044BF30EE270A37EE400A60EE007ADFED14
:106F2800106A9FED107AA7EEA67ADFED0F6AE7EEFA
:106F3800876A9FED0E7AA7EEA67A20EE276AA6EE5C
:106F4800070A70479FED0A0A704700BFDB0F4940E8
:106F5800DB0FC940DB0F49C0DB0FC93FDB0FC9BFDF
:106F68009A7C2E36FAAF4FB93587083CA4AA2ABEB8
:106F780000000000DFED027A30EE270A97E700BF35
:106F8800DB0FC93F38B52DED068B90ED008AB0EECA
:106F9800480A0C460546FFF7EDFFB0EE40AAB0EEF2
:106FA800480AFFF784FFD5ED018AB0EE409AB0EEAB
:106FB800680AFFF7DFFFB0EE408AB0EE680AFFF715
:106FC80076FFD5ED02AAF0EE408AB0EE6A0AFFF726
:106FD800D1FFF0EE409AB0EE6A0AFFF768FF60EE64
:106FE8000A6A69EE297AF0EE665AE7EEA85A29EE9F
:106FF8008A6A29EE007A69EE889A29EE489A28EE7C
:10700800400A28EE0A8AC4ED035AF0EE465AE7EE23
:10701800685AE6EEA87AA6EE687AC4ED009AC4ED3E
:10702800028A84ED059A84ED088ABDEC068B84ED0E
:10703800010AC4ED045A84ED067AC4ED077A38BD16
:1070480010B52DED048B8AB090ED009AD0ED028A30
:1070580090ED018A0446084601A9FFF793FFDDED8C
:10706800047A9DED017A68EE277AE9EE077A9DEDBC
:10707800077AE8EE877A9DED027AC4ED007ADDEDB5
:10708800057A68EE277AE9EE077A9DED087AE8EE48
:10709800877AC4ED017ADDED067A28EE278ADDEDE0
:1070A800037AA9EE278ADDED097AA8EEA78A84ED8E
:1070B800028A0AB0BDEC048B10BD074B1A8822EA7D
:1070C8000000904210B518801C4602D0012004F040
:1070D8008BF8208810BD00BF98110020064B1A8835
:1070E8001043904210B518801C4602D0012004F0CD
:1070F8007BF8208810BD00BF98110020024A9368D1
:1071080023EA0000906070474820002008B5104B23
:107118001A780023D9B2914207D20E4951F82310A8
:107128000968002008600133F4E7322003F0C1FE4B
:10713800094B1B685A0309D5084B9B685B0305D4A8
:1071480040F2DC50BDE8084003F0B3BE08BD00BF04
:107158006015002030150020E81F0020482000207E
:10716800454A69232DE9F34113704FF4FA635380BC
:10717800BE231371EF2382F8CD37002382F8CE3770
:1071880019461646F25C0133B3F5FA6F81EA02013B
:10719800F8D1394B83F8CE17384B1A69120604D543
:1071A800374A5A6002F188325A6004270020013FAA
:1071B80017F0FF074FD0314B3422DA60002444B176
:1071C800002356F804800193FEF738FE0428EED118
:1071D80017E0FEF733FE0428E9D1284D2B6943F068
:1071E80002032B61274B6B612B6943F040032B6132
:1071F800FEF724FE2B69042823F002032B61DFD05D
:10720800D5E71E4D2B6943F001032B6104F10063A0
:1072180003F57E331FFA88F21A80FEF70FFE042862
:1072280010D1194B23440193019B4FEA1848A3F846
:107238000080FEF703FE2B69042823F001032B616D
:1072480005D0B4E72B6923F001032B61AFE70434C1
:10725800B4F5FA6FB3D1094A1369042843F08003DF
:10726800136102D107F0EAFF10B90A2003F0D4FF36
:1072780002B0BDE8F08100BF482000200020024095
:107288002301674500F8030802F8030810B50E4CFF
:10729800206803F06FFD2068047A002202FB02F3E5
:1072A800193B634303F6C4135343192193FBF1F3CA
:1072B800064921F812300132072AEFD10449BDE806
:1072C800104003F00DBD00BF40100020980F0020B3
:1072D8008C2100202DE9F04107F0B0FF10B90A20F9
:1072E80003F09AFFA34CA449A44D4FF4FA62204638
:1072F8000DF0C2F894F8A437022B84BF002384F859
:10730800A43794F8A4274FF4CC7101FB02F3E018DA
:10731800234400F53770286093F8300303F54A7367
:10732800022801FB024284BF0020187292F8303311
:10733800934A13700C2202FB0343924A03F2A6738A
:107348001360A36846F209021A401AB9894A43F43D
:1073580000539360A368D80703D54FF40050FFF794
:10736800CDFEA368590409D50820FFF7C7FE4FF4DE
:107378000050FFF7C3FE0120FFF7C0FEA3681A07FD
:1073880006D54FF40050FFF7B9FE0120FFF7B6FE0F
:10739800A3689B0406D54FF48030FFF7AFFE40206A
:1073A800FFF7ACFE94F8DC21724B2AB193F8E02188
:1073B80012B1002283F8E021734B744E1E604FF027
:1073C800000C674604EB0C03B3F8F4E14FEA5E01E6
:1073D80001F077314FEA9E0303F03333C1EB0E001F
:1073E800C11A4FEADE0303F01133CB1A03EB231360
:1073F8001EF0010803F00F324FF0FF0392FBF3F386
:10740800C3EB032318BF0137A2EB030318BFFFB276
:10741800012B0ADD022B40F0AA80B8F1000F00F022
:10742800A6801EF0BC0F00F0A2800CF1080CBCF185
:10743800180FC7D1013F012F00F29980FFF726FFEF
:10744800302200215248534F0DF021F8524BD5F805
:1074580000801F60514B002108F17900C3F80080BB
:1074680003F0C8FC4E4B80F0010018704D4B07F13B
:1074780026021A604C4B07F1C8021A6098F80000FF
:1074880004F04CF92868494B00F5C5721A6004F0FD
:107498007FFE474BDFED476A07F194021A60464BBF
:1074A80000221A809A71454B07F12C021A602B684A
:1074B800434A93ED187A03F219111160414A03F215
:1074C80089111160404A07F1080111603F4A1760AD
:1074D8003F4A07F19C0111603E4A07F1A60111607D
:1074E8003D4953610E6067EE266AB4F866119361F0
:1074F800B6EE007A07EE901A87EE267AB4F868118D
:107508005762101DF8EE677AC2ED027A07EE901AFC
:1075180093F85C10117193F87810517194F8DF1199
:107528001174F8EE677AB3F81611C2ED037A07EE14
:10753800901A2A4908602A4903F164000860294919
:10754800F8EEE77A81ED007A9FED277A2749C7EEB2
:10755800277A9FED277A67EE877AC1ED007A03F1E3
:10756800680103F21113D1611362BDE8F081FEF7DF
:1075780031FC63E74820002000F8030820100020B1
:10758800941F002040100020C42B0020D22100208E
:10759800CC0E00208C210020000F0020040F0020BA
:1075A80010000020D40600205C060020100F0020E8
:1075B800B80E0020DB0F4940040E00202C070020E5
:1075C8001C1D0020340900207C1600208016002095
:1075D80048080020501300200C0900205C070020F8
:1075E8009407002090070020000061444408002010
:1075F8004C3D0F4408B5FFF7B3FDFFF76BFE0120C4
:10760800BDE8084003F0F0BD2D4B2E4A1B681268F8
:1076180010B51A602C4A1168596051689268DA608E
:107628002A4A996011681961516892689A61284AD2
:1076380059611168D961516892685A62254A19627C
:1076480011881985518859859188D288DA85224A06
:107658009985118819865188598692889A861F4A71
:107668001188D986518819871946928821F83A2FA6
:107678001B4A10780022824206DA1A4C34F812406B
:1076880021F8024F0132F6E7174A1288A3F864205E
:10769800164A1288A3F86620154A1188A3F86810BC
:1076A80051889288A3F86C20124AA3F86A101288AD
:1076B800A3F86E20104A5289A3F85E2010BD00BFBF
:1076C80098280020DC2B0020001400200C14002037
:1076D80018140020B410002004100020AA10002064
:1076E8006015002024100020C0120020BC0F0020CC
:1076F8000A1000203C100020101000202DE9F8434B
:107708000E4B93E8800305460E460024B44213DA74
:107718007B1933F9140008EB050333F9142009EB3E
:10772800050333F914301344022293FBF2F3C01A11
:1077380008F025F90134E9E7BDE8F8839828002026
:1077480070B5472008F06AF8174B1B681B0307D56C
:10775800164B174A5B6810681B68C01A08F000F9D6
:10776800144E154C154D307808F0FAF8236828683F
:10777800C01A08F004F963686868C01A08F0FFF8CE
:107788000F4B188808F0ECF80E4B188808F0E8F84A
:107798000D4B188808F0E4F8337823742B68A3603D
:1077A8006B68E36070BD00BFF829002098280020AE
:1077B800DC2B0020DA10002084280020DC100020B8
:1077C800D8100020D6100020441000207FB5254C8A
:1077D800254E264D2649274A274B20B127480088A1
:1077E800B0F5805F30D23088ADF8040028781D4DA0
:1077F800897912788DF806008DF807108DF8082021
:107808001B788DF8093001A8294606220CF024FEC1
:1078180028B30198BDF808302860AB80532007F0E2
:10782800FDFF208808F09CF8A07808F099F8E37824
:1078380001932379029301A86379039307F0F6FF74
:107848000E4B00221A800AE0308820808979287837
:1078580012781B78A070E17022716371DEE704B0C2
:1078680070BD00BF7813002098110020D4100020AC
:10787800040E0020330E0020980E0020182A002045
:10788800A0F17D03012B70B504460D460A4E05D8BC
:1078980030687D2103F006FD84F02004306821461D
:1078A80003F000FD35B12B881C4404EB142404F0CC
:1078B800FF042C8070BD00BF881100200A4A13887D
:1078C80001331380094A136801331360084A138887
:1078D80001339BB2202B01BF00231380054A138874
:1078E80008BF013313807047182A0020002A00209F
:1078F800042A0020062A002038B53A4B1B78083B9A
:10790800012B05460C466BD8452007F087FF284613
:1079180007F084FF0C2D23D004D80A2D0AD014D8E0
:1079280035B138BD0E2D4BD02ED3FF2D50D038BDDC
:10793800206849E0207807F071FF62796378002AAF
:1079480014BF80200020184300E0207807F066FF6D
:10795800A07807F063FFE07807F060FF20793BE04C
:10796800B4F9000007F0F2FFA07807F057FFE078BD
:1079780007F054FFB4F9040007F0E8FFB4F9060073
:10798800BDE8384007F0E2BF637820788BB180F01B
:10799800800007F043FFA468E0B207F03FFFC4F39C
:1079A800072007F03BFFC4F3074007F037FF200E1E
:1079B80012E007F033FF6068BDE8384007F0DFBF2A
:1079C800206807F0CDFF6068BDE8384007F0C8BF01
:1079D800054807F001FF0020BDE8384007F01EBF4A
:1079E80038BD00BF74280020528301082DE9F04FEC
:1079F800B84BB94F1A888BB00193002A40F09D808C
:107A0800B7F8CA07B54E42F20103C41A6042604192
:107A1800FFF7DCFEFFF7F8FD3468492007F0FEFEAB
:107A2800AF4B2546186807F09BFF55F8040B07F085
:107A380097FF2846FEF780F904F11000FEF77CF95D
:107A480004F11C094FF01008A64D01232A6803FA17
:107A580008F3134203D0D9F8000007F090FF08F1AB
:107A68000108B8F1130F09F10409EDD104F1280058
:107A7800FEF752F9B7F84431B4F92E00C01A07F0EE
:107A88006FFF2B68D90408D5974BB4F864001B889E
:107A9800181AC0F30D0007F063FF2B689A0403D58A
:107AA800B4F8660007F05CFF2B685B0503D504F1AA
:107AB8006800FEF731F92B68180403D5B4F86E0096
:107AC80007F04EFF04F13000A046FEF725F904F157
:107AD8003600FEF721F9B7F8443138F93C0FC01ADF
:107AE80007F03EFF0127814B1B789F4208DA38F9DF
:107AF800020FB4F93C30C01A07F041FF0137F2E732
:107B08002B68990505D5B4F95E00A0F2DC5007F0A2
:107B180036FF326876487260B260121A1111754ADF
:107B28004A43531C032293FBF2F202EB42029A1AD5
:107B3800702303FB02033360C0E16F4B6F4A1B687D
:107B480011688B4206D00AA9002041F8203D136035
:107B5800FFF7D2FE019B97F8CA171B8897F8CB0747
:107B68000B44013BB3FBF0F200FB12338B4280F075
:107B780070815A4F0120FFF729FEFFF745FD50207D
:107B88003E687D6807F04AFEBA683B6810681B6863
:107B98007A6803441068A3EB400007F0F0FE6A68B7
:107BA80073689B1A0293AA68B3689B1A0393EA68DE
:107BB800F36802A89B1A0493FEF7BEF82A69336992
:107BC8009B1A02936A6973699B1A0393B369AA693A
:107BD80002A89B1A049307F029FE06F11C0B05F175
:107BE8001C0810243F4901220B68A2401A428A4609
:107BF80006D0DBF80000D8F80030C01A07F0BFFE46
:107C08000134132C0BF1040B08F10408EAD106F136
:107C1800260005F12601002331F9024F30F9022F21
:107C2800121B02AC44F823200133042BF4D10321A6
:107C38004FF000094FEA89035FFA83F902AB53F862
:107C480021206AB102F108000F2802D849F0010981
:107C580006E08032FF2A94BF49F0020949F003097F
:107C680011F1FF31E6D2484607F0D8FD00240DF1A6
:107C7800080BA04609F00302022A16D0032A1DD0D9
:107C8800012A4ED1B8F1000F05D1DBF800402401DC
:107C9800E4B2904645E0DBF8000000F00F00204316
:107CA80007F0BCFD4FF000083BE0B8F1000F0CD026
:107CB800DBF80000C0F3031020432CE0B8F1000FFC
:107CC8001ED19BF8010007F0A9FD9BF8000007F002
:107CD800A5FD26E0042A002048200020982800203E
:107CE800002A0020F8290020F4290020601500202F
:107CF800A4280020B76DDBB60C2A0020082A002033
:107D0800DBF80000C0F30330204307F087FDDBF801
:107D18000000C0F3071007F081FDDBF800402401E4
:107D2800E4B20BF1040B06AB9B454FEA9909A1D1CC
:107D3800B8F1010F02D1204607F070FDDAF8001003
:107D480011F480541FBFB6F86430B5F864209B1A4C
:107D5800029318BF01248A040AD50AAB03EB8402F4
:107D6800B5F86600B6F866301B1A42F8203C0134B4
:107D78004B0513D502AB03EB840C06F1660E05F137
:107D8800660000233EF9022F30F9028FC8EB020289
:107D98004CF823200133032BF4D1033408040BD50A
:107DA8000AAB03EB8402B5F86E10B6F86E305B1AB6
:107DB80042F8203C013400E0FCB1012C03D10298C8
:107DC80007F0DDFD19E0631E002002AA400052F80A
:107DD8002320C0B20AB140F00100013BF5D507F0FD
:107DE8001DFD4FF0000802AB53F8280008B107F05A
:107DF800C6FD08F10108A045F5DB30200321FFF797
:107E08007DFC36200321FFF779FC2F4B3C201978A5
:107E1800FFF774FCDAF80030990506D5B6F95E006C
:107E2800B5F95E30C01A07F0AAFD3A6827487B68A2
:107E38007A60121A1111264ABB604A43531C032266
:107E480093FBF2F202EB42029A1A702303FB02033D
:107E58003B60204B1B681A0630D51F4C1F4D22680B
:107E68002B689A420BD162686B689A4207D1019BD2
:107E78001B88102B11D11A4B1B885B060DD148208B
:107E880007F0CCFC206807F07AFD606807F077FD02
:107E980023682B6063686B600EE0124A0F4B117801
:107EA8002A7C914208D1104A99681068884203D107
:107EB8005268DB689A4201D0FFF742FC07F07EFC6B
:107EC8000BB0BDE8F08F00BF60150020A42800208B
:107ED800B76DDBB6E81F002048100020842800207A
:107EE800062A0020DA100020DC1000202DE9F84FC7
:107EF8000C9E3A4CC2EB030B0B9BF61A63680029E5
:107F080014BF4FF0060A4FF0040A013305469046A5
:107F180013D1236853455ED2314A324852F82320A0
:107F2800032B98BF294607F067FC63680133636039
:107F38002D4B002205469A7113E0002511E02B4ACB
:107F48001278954240DA0B9BE3B109FB06F2995C83
:107F580001228A40264909680A4213D1636801331D
:107F68006360D4F804900A9B1C4F9945E7DB2BD13A
:107F78000A2007F053FC3B6801333B604FF0FF33A6
:107F88007B6021E0184A917921B12C2007F046FC4A
:107F9800013501E001219171226809FB0BF308EB1F
:107FA800030752B958F8030007F016FC97F90410B4
:107FB8004B1C0544D2D00F4802E03A440E481179D0
:107FC80007F01AFC0544C9E7206850452CBF00207B
:107FD8000120BDE8F88F0020BDE8F88F102A0020A6
:107FE8000C6401085D830108781300201C0100203F
:107FF800F82900206C830108078E010830B585B088
:1080080004AC002524F8025D0091ADF80600214675
:108018001020FFF735FC9DF806002146FFF730FCDD
:108028009DF807002146FFF72BFC9DF8000021462C
:10803800FFF726FC9DF801002146FFF721FC9DF87B
:1080480002002146FFF71CFC9DF803002146FFF7BC
:1080580017FC9DF80E00C043C0B22946FFF710FC7C
:1080680005B030BD10B5054C206803F018F918B1FB
:10807800206803F011F9F6E710BD00BF5811002081
:1080880013B5044601A9006809F0A6F8132009F001
:10809800DFF8BDF9040009F0C9F81B2009F0D8F889
:1080A800BDF9060009F0C2F8232009F0D1F82368C9
:1080B800002BB4BF53204E2009F0B8F801A960681E
:1080C80009F08AF8122009F0C3F8BDF9040009F094
:1080D800ADF81A2009F0BCF8BDF9060009F0A6F8B9
:1080E800222009F0B5F86368002BB4BF572045205B
:1080F80009F09CF802B010BDF8B504460E461746C4
:108108000025204620210CF0F8F90446D0B10134AE
:1081180020460CF057FAB0F5617F05DB40F63403D2
:108128009842A8BF184601E04FF46170A0F561704D
:10813800192390FBF3F00DB9307000E070703B78B4
:1081480001333B700DB90125DBE72046F8BD30B59A
:1081580005460C461346294622460248BDE83040EB
:10816800FEF777BE608401087FB504780646E4B957
:10817800354B1B6803EB8403192193F87B0093F8B4
:108188007C6093F8792093F87A304FF4617511FB8D
:10819800005011FB0651009001912C4821460134F2
:1081A800FEF757FE142CE3D14BE00CF00BFA132822
:1081B800054641DC244B701C1C68202100238DF8E7
:1081C8000F300CF09AF91E35064670B1013630466C
:1081D8000CF0F8F919289FBF04EB850358709DF837
:1081E8000F30013398BF8DF80F30304620210CF046
:1081F80084F9064670B1013630460CF0E3F90D28D3
:108208009FBF04EB850398709DF80F30013398BF2A
:108218008DF80F3004EB85043046E11C0DF10F0298
:10822800FFF76AFF9DF80F30042B0AD0601C00216D
:1082380004220CF02CF904E0054800211322FFF772
:1082480086FF04B070BD00BF201000207F840108A5
:1082580094840108014806F00DBE00BF9A84010805
:108268002DE9F04304788FB00546002C59D17B4B9B
:108278000021142209A807AED3F800800CF007F9F2
:108288000722304600210CF002F905A80023A700B8
:10829800059308EB070583801A467149B5F802E093
:1082A80031F813C01CEA0E0F0AD00DF1380C0E314C
:1082B80002F1010E6244595C02F81C1C5FFA8EF24E
:1082C8000133072BE9D100210B46664AB5F802E0D5
:1082D80011F802C01CEA0E0F0AD00DF1380C063254
:1082E80003F1010E63448A5C03F8242C5FFA8EF3D1
:1082F80001310629E9D118F807305B498DE84100BA
:108308006A78029209A81A0903F00F0307F0C4FD5E
:108318002146564809AA0134FEF79BFD202CA6D118
:1083280098E00CF04FF91F28044600F38680284691
:108338002021E4B20CF0E1F81F2C02D9FFF78AFFE4
:1083480088E0464B1B6803EB8404451C002120464B
:1083580004220CF09CF80027454B09AE304600215A
:108368000A2217F803905FFA87F80CF090F80023B8
:1083780015F8012B32B10A2B04D04A4502D0F25429
:108388000133F5E74A455ED108F1FF33032B09D8DD
:10839800DFE803F01005023F0DF1230134E00DF191
:1083A80023011EE030460CF00DF92378C0B243EAF1
:1083B800001006E030460CF005F9237800F00F00B5
:1083C8001843207031E00133062B0AD0244800F10D
:1083D8001B069E5D9642F6D103445A7D638813437B
:1083E800638011F8012F02B30023EFE70133072B55
:1083F8000AD01B4800F10E069E5D9642F6D130F871
:10840800132063881343638011F8012F6AB1002396
:10841800EFE730460CF0D6F80F2804DC30460CF0B5
:10842800D1F8607001E0002363700137052F93D104
:10843800012405F051FF6CB980E70E4800211F2286
:10844800FFF785FE06E02046002104220CF01FF805
:108458000024EEE70FB0BDE8F08300BF80130020D2
:108468002464010839640108A8840108B784010854
:108478004564010894840108F8B50478064674B97F
:10848800304DB5F8C621B5F8C8312F48214601341A
:10849800FEF7DFFC042C05F10405F2D1F8BD2B49E9
:1084A8000BF0FEFFA8B9274B4FF47A714FF4FA622C
:1084B800A3F8C611A3F8C821A3F8CA11A3F8CC21C0
:1084C800A3F8CE11A3F8D021A3F8D211A3F8D42190
:1084D800F8BD30460CF076F8032805462BD8304610
:1084E80020210CF00AF8044630B1013420460CF083
:1084F80069F80126074600E00646204620210BF0D1
:10850800FCFF10B9BDE8F840A4E601300CF05AF8B9
:10851800012EF7D1A7F2EE2240F2DC539A42F1D8AD
:10852800A0F2EE229A42EDD8064B703503EB850394
:10853800DF801881F8BD064800210322BDE8F84015
:1085480005E600BF48200020C3840108D68401083E
:10855800999001082DE9FF4104780546002C39D18E
:108568007348744D06F086FCD5ED057AF5EE407A31
:10857800F1EE10FA00F0D88021466F48FEF769FC4A
:1085880095ED050A6846FEF7F9FA01466B48FEF7CD
:1085980060FC95ED060A6846FEF7F0FA0146674862
:1085A800FEF757FC95ED070A6846FEF7E7FA01461D
:1085B8006248FEF74EFC95ED080A6846FEF7DEFABB
:1085C800013401465E48FEF744FC0C2C05F1100509
:1085D800CAD1A9E05B4905220BF0A6FF40B9554B6B
:1085E80003F1C0020021596110339342FAD19BE094
:1085F8002846554904220BF097FF04462846002CCC
:1086080040D120210BF079FF002800F08D80451C17
:1086180028460BF080FF07464C4B53F824601EB9E0
:108628004B4806F027FC7FE028463146FAB20BF0AB
:108638007BFF01340028EFD13E4B03F1C0029E4678
:108648000021596110339342FAD1424B03EBC40223
:108658009846D2F804C0BCF1000F04D131463E4818
:10866800FEF7F7FB57E0002718F834309F42F5DA99
:108678003B010EEB030563440FCB143585E80F006F
:108688000137F1E70BF09EFF0B28064647DC28462A
:1086980020210BF032FF054650B101352846FEF780
:1086A800E3F9244B03EB061383ED050A012400E0EC
:1086B8000446284620210BF020FF054648B1013525
:1086C8002846FEF7D1F91B4B03EB061383ED060A88
:1086D8000134284620210BF010FF054648B101352A
:1086E8002846FEF7C1F9134B03EB061383ED070A7F
:1086F8000134284620210BF000FF10B9FFF7AAFD2E
:1087080012E00130FEF7B0F90A4B032C03EB061612
:1087180086ED080AF2D11148FFF71CFF04E0104863
:1087280001210C22FFF713FD04B0BDE8F08100BF62
:10873800DC84010848200020F7840108FD84010832
:10874800EF8D0108D684010801850108F86B01083E
:10875800068501089083010815850108E281010852
:1087680094840108F0B5047887B006461CBB514BC9
:108778001968062303FB0411192091F8CA5091F8CF
:10878800CB7091F8CE2091F8C9304FF4617610FB88
:10879800056510FB07600095019091F8CC000290E8
:1087A800C83145484979039121460134FEF751FB08
:1087B8000C2CDCD17CE00BF005FF0B28044672DCA6
:1087C8003C4B701C1D68202100238DF817300BF0DE
:1087D80094FE064680B1013630460BF0F3FE0328BE
:1087E8009FBF062303FB045383F8CE009DF8173080
:1087F8009CBF01338DF81730304620210BF07DFEE9
:10880800074680B1013738460BF0DCFE0D289FBFC4
:10881800062303FB045383F8C9009DF817309CBF57
:1088280001338DF8173006266643A9193846CA3130
:108838000DF11702FFF760FC20210BF05EFE0746E2
:1088480070B1013738460BF0BDFE14289FBF9DF864
:1088580017307619013386F8CC0098BF8DF8173099
:10886800384620210BF049FE78B101300BF0AAFE02
:108878000D289FBF062303FB045383F8CD009DF802
:1088880017309CBF01338DF817309DF81730062B31
:108898000ED0062202FB04500021C9300BF0F7FD70
:1088A800FFF7D8FC04E0054800210B22FFF74FFC36
:1088B80007B0F0BD2010002021850108948401082C
:1088C800F0B5027887B0AAB94C4C04F118064C4BA5
:1088D80094F9F21193F900208A4272D093F90C208E
:1088E8008A426ED093F918308B426AD00834B44269
:1088F800EDD180E0002204920592451C0BF062FE47
:10890800C4B260B202F0A6F9074618B18DF810405B
:10891800012400E00446284620210BF0EEFD054620
:1089280038B1013528460BF04DFE0134ADF8120080
:10893800E4B20026284620210BF0DFFDB0B3451C29
:1089480028460BF03FFE00222E4951F82230834280
:108958005FFA82FE04D00132082AF5D1002300E034
:10896800734651F82320824220D1022E0FD0032EC5
:1089780012D05A1E012ED2B204D0042A13D88DF870
:1089880014300EE0042A0ED88DF8153009E0052BB6
:1089980009D88DF8173004E09A1E052A03D88DF8F7
:1089A80016300134E4B20136042EC3D1052C03D8A5
:1089B80007B0BDE8F0404DE404AB03CB3860796004
:1089C80019E094F8F7010F4B94F8F65153F820008A
:1089D800B4F8F421009094F8F90153F820000190BC
:1089E80094F8F80153F82000029053F8253006480F
:1089F800FEF72FFA7AE707B0F0BD00BF4820002045
:108A080054120020E8630108418501082DE9F3416B
:108A1800047880464CB9204601A9FDF73FFA013495
:108A2800FFF7F4FF122CF6D16BE00BF0CBFDC6B2CA
:108A3800112E61D8344C06F1D00704EB470308F136
:108A4800010020219D780BF058FD18B9AA1E554247
:108A5800554139E04378682B06D0732B07D0612B3A
:108A680013D14FF0000804E04FF0010801E04FF087
:108A78000208A8F102035D4200F101004FF0200155
:108A88005D410BF03AFDD8B115B9FFF7E3FB38E0CB
:108A980001300BF097FD40F2ED2380B2984205DDDE
:108AA80040F6CA039842A8BF184601E040F2EE20FB
:108AB80004EB4703A0F2EE20192290FBF2F0D870E5
:108AC80004EB470383F8028004EB47040F4AA378BA
:108AD800134493F8262055B1E3780D4840F2EE246C
:108AE8001925314605FB0343FEF7B3F909E0314682
:108AF8000848FEF7AEF904E0074800211122FFF705
:108B080026FB02B0BDE8F08148200020246401085B
:108B180060850108728501089990010807B501234D
:108B2800ADF8041001A98DF806208DF8073004F07F
:108B3800E9FE03B05DF804FB2DE9F843404B414CD6
:108B48009A6A42F400129A629A6A22F400129A62AD
:108B58005A6942F400125A6106464FF4A061204651
:108B68000122FFF7DBFF4FF4A063238572B6364D71
:108B780002214FF00809298528460422A5F82890E3
:108B8800FFF7CCFF284601224946FFF7C7FF2F48C9
:108B980050F8364000EBC6002368426801265700AB
:108BA80006FA07F848EA030396402360A661C5F869
:108BB80018902B8A9B07FCD4236848EA0303236098
:108BC800214B0822B1B221851A854FF48072A3F88F
:108BD80028284FF48062C3F8182840F605531A482D
:108BE800028A950711D4013BF9D122680323BB40BF
:108BF80022EA0303236008210222FFF78FFF62B6EF
:108C08003220BDE8F84302F054B90422A661204698
:108C1800FFF784FF0B4B4FF480621A850A4B1A8AC0
:108C28009207C9D5228A92B21642064A4FF0080026
:108C38004FF4807115BF9861188511859161EDE732
:108C48000010024000100048000800488485010810
:108C580010B50446204602F019FB18B90A2002F0A4
:108C680028F9F7E710BD0C4B5A6882421A4607D01C
:108C78001B69834206D0D36983420BD1022302E0E9
:108C8800002300E001230021C1620C2000FB032324
:108C980019725960704700BF5412002013B506229C
:108CA80004466B4603211E2004F042FF9DF8002075
:108CB8009DF801309DF8021043EA02231BB21B4ABB
:108CC80007EE903A92ED007AF8EEE77A67EE877A47
:108CD80092ED027AFDEEE77A17EE903A23809DF83E
:108CE800033043EA01231BB207EE903AF8EEE77A25
:108CF8009DF8041067EE877A92ED017AFDEEE77A27
:108D080017EE903AA3809DF8053043EA01231BB281
:108D180007EE903AF8EEE77A67EE877AFDEEE77AA3
:108D280017EE903A638002B010BD00BF80000020AB
:108D380013B506220446A82119206B4604F0F8FE54
:108D4800F0B19DF800309DF8012043EA022202218B
:108D58009DF8033012B292FBF1F222809DF80220B6
:108D680042EA032212B29DF8053092FBF1F26280CA
:108D78009DF8042042EA03231BB293FBF1F3A3807E
:108D880002B010BD08B524218022192004F04CFF40
:108D9800642002F08EF820219722192004F044FF65
:108DA8000A2002F086F810222321192004F03CFF43
:108DB800642002F07EF8024B4FF480521A8008BDFE
:108DC800120000202DE9FF41634B1B6893B11A681C
:108DD8001AB16249486902434A619A88ADF8042089
:108DE80002228DF807209868002201A98DF8062034
:108DF80004F088FD322002F05CF8002111221E20C8
:108E080004F012FF012160221E2004F00DFF6420EF
:108E180002F04FF802A8FFF741FF00240A27264670
:108E28002546022101221E2004F0FEFE322002F017
:108E380040F802A8FFF732FFBDF90820BDF90A1073
:108E4800BDF90C308A421444A8BF0A4693421D4417
:108E5800A8BF134613F5805F0E440ADD404A938A83
:108E68009BB283F48843013F9382DAD14FF0010823
:108E780001E04FF000081E200021122204F0D4FE69
:108E88000A27022101221E2004F0CEFE322002F021
:108E980010F802A8FFF702FFBDF90820BDF90A1073
:108EA800BDF90C308A42A4EB0204A8BF0A469342DB
:108EB800A5EB0305A8BF134613F5805FA6EB0106D3
:108EC80008DD274A938A9BB283F48843013F938243
:108ED800D7D101E04FF0000807EE904A9FED217AC4
:108EE800214FF8EEE77A0021C7EE277A70221E207C
:108EF800F0EEE77AC7ED007A07EE906AF8EEE77AC7
:108F0800C7EE277A9FED197AF0EEE77AC7ED017A76
:108F180007EE905AF8EEE77AC7EE277AF0EEE77A8E
:108F2800C7ED027A04F080FE012120221E2004F001
:108F38007BFE1E200221002204F076FE642001F050
:108F4800B8FFB8F1000F04D14FF07E533B607B604F
:108F5800BB6004B0BDE8F0810C03002000100240A3
:108F68000010004800406F468000002001C05E46A7
:108F7800154B37B5082205461A85E82006F006FD88
:108F88000024002006F002FD0DF804000134062C30
:108F9800F7D10D4B08229A619DF800209DF8013009
:108FA80043EA02232B809DF802209DF8033043EA10
:108FB80002236B809DF804209DF8053043EA0223C4
:108FC800AB8003B030BD00BF001000482DE9F04F62
:108FD800944D954C2B68954E9BB2238022883188FE
:108FE8000A40900585B007D54FF6FF53904A2B608D
:108FF80013780133DBB2137023880B40190440F156
:1090080043830023ADF80A302B6887499AB21804C5
:10901800228040F139830B8803F00F038B70002BFB
:1090280040F00483834A844F136884489BB23B8092
:109038003B8803F0300303803B8803F440533B80B4
:10904800D2F800E04BF6BF730EEA030383F4005333
:1090580083F0200343F4004343F0800313600B883C
:1090680013F0100F804626D1116848F60F730B4095
:10907800734913600B681A7A022A894601D0042AB8
:1090880005D1FCF7BDFFD9F800301B7A3FE1062A6D
:109098006ED15A78052A09D11A78520606D1D8789D
:1090A800FCF792FF674B1B681B6A9847664B1B6867
:1090B8009B6898475CE013689BB2ADF80A30BDF82E
:1090C8000A301B0540F1F38111685D4840F68F7343
:1090D8000B405E4913600A685D4B92B213445B0013
:1090E80081461A68036893F808E0BEF1090F8A46BA
:1090F80017D092B2520002F1804202F5C0421178B4
:109108001970517859709188C8B2090A41EA00214A
:1091180059801189C8B2090A41EA002199809289C7
:10912800DA8001221A72DA8893F801B0002A40F036
:10913800F1801A7812F07F0250D1BBF1090F10D1DB
:10914800DA78012A00F2CA809978002940F0C680AE
:109158009988002940F0C2809A723A4B1B685B6874
:10916800BAE0BBF1050F10D193F90320002A01DA08
:109178000823CCE09A78002AFAD19A88002AF7D1F5
:109188009B7A002B00F0B480F2E7BBF1030F0FD1FC
:10919800DA78012A40F0A2809A88002A40F09E805E
:1091A8005A7A42F020025A72264B1B68DB6993E018
:1091B800BBF1010F40F09280DA78012A40F08E80EE
:1091C8009A88002A40F08A805B7A980640F1868067
:1091D800FCF7C4FF002800F08B807FE0012A39D11A
:1091E800BBF10B0F7AD1184A58791268D97892696D
:1091F8009047D9F800309A7A002A6FD000286DD1AC
:109208001A79002A6AD19B78002B67D10D4B1B680D
:10921800DB6898470A4B1B685A79DA72DA781A734E
:1092280066E000BF445C0040841300201C2A002034
:10923800FF2B0020005C00407A12002078120020EA
:10924800A4110020A811002018150020505C00402F
:1092580004300020022A41D1BBF1010FB8D0BBF184
:10926800030F3BD1587920F0800E4FEA8E0202F1AD
:10927800804101F5B84110F0800F096814BF01F072
:10928800300101F44051BEF1030F27D8B3F802E0D2
:10929800BEF1000F22D109B39B7AFBB102F18042E3
:1092A80002F5B842010613684BBF23F4E04323F4E8
:1092B800804323F0400323F070034BBF9BB29BB263
:1092C80083F0100383F4805343F4004343F0800396
:1092D8001360A94B1B689B69984709E0A74B1B685B
:1092E80058465B699847032810D000287FF440AFA0
:1092F800DAF80020A24B92B213445B001A680022ED
:109308001A603023A8F80030062300E00923D9F8B2
:10931800002065E1BBF1060F13D11A7850067DD104
:109328009A78964B012A02D11B68DB696AE0022A07
:1093380002D11B681B6A65E0032A6FD11B685B6A50
:1093480060E0BBF1000F3AD15988002966D15A680C
:1093580022F47F42B2F5003F60D11A7812F07F0202
:1093680004D19B88002B00F0F48157E0012A0AD130
:10937800824A587912689269904700284ED1D9F8E4
:1093880000309B7A17E0022A48D15A7902F00F017F
:109398000BB29B0003F1804303F5B84312F0800F32
:1093A8001B6814BF03F0300303F44053032935D876
:1093B80012F0700F32D1002B40F0CB812EE0BBF1C0
:1093C800080F04D11B78590600F0C58126E0BBF1CF
:1093D8000A0F23D11A7802F07F02012A1ED19A7A45
:1093E800E2B15988D1B95A6822F47F42B2F5803F78
:1093F80014D1624A5879126892699047002800F09F
:10940800AC810BE053B1D9F800204FF0000AA2F864
:1094180012A093615046984750460BE0574BD9F835
:1094280000201B6850781B699847032802D1554BC8
:109438001B6806E0D9F800301A8A4FF6FF718A4295
:1094480001D1092203E0022800D012B908221A72B9
:10945800C7E093F90010002923DAD988039103980B
:10946800DFF818E1824202D9039A1A8211E08A428F
:109478000FD2DEF8001091F82C00824201D20021B0
:1094880005E092FBF0F100FB112212B901213E4ADE
:109498001170DEF8002092F82C209A82FCF7B0FDBB
:1094A8009FE003221A724FF440533B8099E0BDF8C5
:1094B8000A301BB2002BBFF6A7AD116840F68F73B8
:1094C8000B4013602F4AD2F8009099F80830022B0D
:1094D800934600F08280042B7FD0032B01D0052B0C
:1094E80075D1D9F81830B9F810209BB9B9F81020FF
:1094F800002A4FD04FF440533B80244B1968204B2F
:1095080089B20B445B001968002119603023A8F860
:1095180000303FE0002AE9D0B9F814A0924528BFEE
:1095280092461FFA8AF2104601929847019AB9F8B2
:1095380010309B1AA9F81030B9F812301344A9F862
:109548001230124B1A68124B92B213445B000AF1A4
:10955800010A1B689BB203F1005303F540534FEA1D
:109568006A0A5B0000215145C0D053F8212020F839
:1095780011200131F7E700BFA811002018150020BD
:1095880002300020A4110020FE2B0020505C004077
:1095980004300020B9F814309342DBF8003001D8C9
:1095A800032201E012B105221A720CE00621197299
:1095B8006C4B19686C4B89B20B445B0019681A60D4
:1095C8003023A8F80030DBF800301B7A06E0072BC0
:1095D80003D1664B1B68DB6898470823DBF800203B
:1095E8001372FCF79FFD624B1A684BF6BF7313406A
:1095F8003A88D2043A8848BF83F480539004B8F874
:10960800002048BF83F40053D106B8F8002048BFB3
:1096180083F01003920648BF83F0200343F400430D
:1096280043F08003524A9BB213602DE09A0002F186
:10963800804202F5B842116889B2ADF80A10BDF847
:109648000A1009B2002909DA106840F68F71014042
:109658001160013B474A52F823309847BDF80A3059
:109668001F067FF5D1ACA1788B0003F1804303F589
:10967800B84348F60F72186802401A603D4B03EB76
:1096880081039B699847BFE42288338813405905B2
:1096980005D54FF6FF332B60374B5B689847228818
:1096A80031880A40920444BF4DF6FF732B6023882B
:1096B800324A0B40DB0452D54EF6FF732B60002371
:1096C800D370D378052B41D8DFE803F0030D1418C5
:1096D800222DA368294D1BB902F03AFE062300E0AB
:1096E8000523EB703BE002F033FE0423E370012313
:1096F800A36034E002232371032328E02379013B8C
:10970800DBB22371237953BB1C4B0422DA7026E0A9
:109718001B4A13689BB243F0100313600523E370E0
:109728000A2323711BE02379144A013BDBB223711E
:10973800237903F0FF0093B911490C684FF6EF73D2
:1097480023400B600623D370906008E00623E37083
:1097580005E00C4B57E60C4B55E60C4B53E605B0B1
:10976800BDE8F08F505C0040023000201815002042
:10977800005C0040106901081C00002084130020D0
:10978800405C0040335C0008D95C0008B95C000804
:10979800704770477047FEE7FEE7FEE7704730B551
:1097A8000024E3B293420DD2030F092B94BF303348
:1097B800373301F8143001EB4403002500015D70D4
:1097C8000134EEE730BD00BF2DE9F04F2DED028BDF
:1097D80085B007460293A04B1B889807934636D559
:1097E800109B9E48DC89B0F900301B1B03F2F3156F
:1097F80040F2E632954203D8002BB8BF5B4201E045
:109808004FF4FA73B0F90220121B02F2F31440F27B
:10981800E630844203D8002AB8BF524201E04FF430
:10982800FA729342B8BF1346C3F5FA73052293FB45
:10983800F2F30A22643B53433A7FD2105343642223
:1098480093FBF2F3134423EAE373DBB200E06423EF
:109858000093CB1C0193B8460024019BDFF824A297
:1098680013F8016F0193022C4FEA440905D1BAF9A4
:1098780004301B365E43761146E079493AF81420E5
:1098880031F91410022012FB0011CBF100029142B1
:1098980003DB59450A46A8BF5A467249029B31F96B
:1098A8000950551B33F91420154406F025FB88B1DF
:1098B80007EE905A6C4AB8EEE70AB2EE048A105DD9
:1098C80080EE080A06F0D4F820EE080AFDEEC07A09
:1098D80017EE905A604A1288D10712D43AF9093023
:1098E8001B365E4393074FEA26160DD5BB7C5D43B6
:1098F8009DF900305D43642395FBF3F506EB2516CF
:1099080002E03E7A75432E11584B042533F909308D
:1099180093FBF5F5564BE25C924698F80120751BCF
:1099280051466A434A43642192FBF1F297F8511079
:10993800D21108EE102AA9B1022CB8EEC80A08D133
:109948004A0803D09142A8BF114600E001214948C6
:1099580002E0181D00EBC400D3ED070AFDF75AF822
:10996800BDEEC08ADFF808E1434B98F80B60188811
:109978000EF1200300FB05F253F82410D21206FB67
:109988000216B6F5001F3D4AA8BF4FF400169642CE
:10999800B8BF16460EF12C0243F8246052F8243062
:1099A80042F82450EB1A0EF138014FF6FF72000905
:1099B800B2FBF0F043430EF1440051F8245050F844
:1099C800242040F824509B112A4441F8243097F869
:1099D80050101A444FEA840C761300EE102A79B11D
:1099E8000EF15000B8EEC00A00EBC400DEED070A25
:1099F800CDF80CC0FDF70EF8DDF80CC0BDEEC00ABE
:109A080098F8153010EE102A18EE101A5A435346DB
:109A180053431A463144642392FBF3F3184A1B124A
:109A2800194422F8091018EE100A02F1080101344D
:109A38004CF8010002F114012032032C4CF80160AB
:109A48004CF8023008F101087FF407AF05B0BDEC0F
:109A5800028BBDE8F08F00BF981100202420002061
:109A6800F62B0020E01F00204869010804100020A0
:109A780090130020A4130020D80F00200000E0FF5E
:109A8800F8130020B41000202DE9F04F2DED028BC3
:109A980087B000260593C54B0491B3F90280B3F94A
:109AA80000300392B8F1000FB8BFC8F10008002BCE
:109AB800B8BF5B429845B8BF9846B8F5FA7F0746E5
:109AC800A8BF4FF4FA780090B1460196B3463446E1
:109AD800B74D2B88990758D0B44BB64A33F8143091
:109AE80032F91420022013FB0022039B5B429A42A6
:109AF8004FEA440103DB039B9342A8BF1346AE4AD7
:109B080031F902A0059A32F91420CAEB030303EBDA
:109B1800020A06F0F1F988B107EE90AAA74BB8EE51
:109B2800E70AB2EE048A185D80EE080A05F0A0FF85
:109B380020EE080AFDEEC07A17EE90AA3B7A64225E
:109B480003FB0AF393FBF2F33A7F6FF0040101FB86
:109B580002FB5B4505DB02EB82029342A8BF13467A
:109B68009B46974A52F824100AEB010342F21071FF
:109B78008B42A8BF0B4693498B42B8BF0B4642F8AD
:109B88002430BA7C53431B1301932D8805F003033B
:109B9800012B38D0854B8C4933F91490009B51F830
:109BA80024E093F801C0894B33F9140080EAE0738C
:109BB800A3EBE073B3F5206F4FEA840616DC09EBDC
:109BC80089031A0192FBFCF3042290FBF2F0181AA5
:109BD8008644BEF57A5FA8BF4FF47A5E7C4B9E45FB
:109BE800ACBF41F824E041F8243002E0002341F8FA
:109BF80024308B597D2693FBF6F6009BDB7A734362
:109C0800402693FBF6F6AA0711D5019BC8F5FA7210
:109C180008FB09F008FB06F54FF4FA7102FB0B008C
:109C280002FB035590FBF1F095FBF1F505E0EB071E
:109C38004DBF019D354648465846644B33F91420BC
:109C4800042392FBF3F3634A02F19C014FEA440AAE
:109C5800615C4B436FF04F0193FBF1F397F85110A0
:109C6800C31808EE103A51B1101DB8EEC80A00EB3F
:109C7800C400D2ED070AFCF7CDFEBDEEC08ADFF8BE
:109C880054E1524B0EF1A0013AF803003AF90130C1
:109C98002AF8010002B20EF1A4010EF1AC00D31AA9
:109CA800042293FBF2F2A30051F824C0029350F867
:109CB800243041F82420634497F8501040F824C019
:109CC800134400EE103A59B10EF15000B8EEC00A34
:109CD80000EBC400DEED070AFCF79CFEBDEEC00AEF
:109CE8003C4A02F1B40110EE103A095D01FB03FE93
:109CF80018EE101A02F1680029444FF0200C9EFB60
:109D0800FCF3C91A2AF80010029902F1700E0846ED
:109D180018EE101A40F80E1002F17C015B42455013
:109D280002F188014350009B013300930CB90124D0
:109D3800CEE61E4B946AB3F90410049B9B790F334B
:109D48005B004B435B112149002BB1F904104FF024
:109D5800040091FBF0F0A3EB0000B8BF5B42322B8C
:109D6800797B0BDC1C4B01FB00418B42A8BF0B46E7
:109D78001A498B42ACBF9362916201E0002393625F
:109D8800F97801FB00F31649097803294FEAA31370
:109D980029D9B7F84E10B1F5FA7F24D24842834248
:109DA80020DB8B42A8BF0B461DE000BFB41000208B
:109DB80098110020F62B0020E01F002048690108B8
:109DC80024140020F0D8FFFFB01300200410002056
:109DD80080C1FFFF90130020FEFFFF0F020000F07C
:109DE800601500200346916A936741F34F31B1F53E
:109DF800807FA8BF4FF480716FF0FF008142B8BF29
:109E0800014658180023A2F86C00C2F88410C2F862
:109E1800903007B0BDEC028BBDE8F08F2DE9F04F14
:109E28002DED028B85B080460393BC4B02911C88B4
:109E3800019204F00204A4B294B1B94BB3F9024000
:109E4800B3F90030002CB8BF6442002BB8BF5B42A6
:109E58009C42B8BF1C46B4F5007FA8BF4FF40074FD
:109E6800C2460025AF4AAE4B32F9152033F815101B
:109E7800AD4882EAE27EAEEBE27E0BB2BEF5206F21
:109E88004FEA45094FEA43034FEA850750F8256032
:109E980012DC4FF0040E92FBFEF29A1A1644B6F545
:109EA8007A5FA8BF4FF47A56A04A9642ACBF40F8F2
:109EB800256040F8252002E0002240F82520C659F8
:109EC8009AF80B20F61156439AF801205343934A07
:109ED80012884FEAA31B93074FEAA61654D0944A58
:109EE800019B32F90920022011FB00215A429142BC
:109EF80003DB8B42A8BF0B461A468E49039B39F9F0
:109F08000110511A33F915208B1808EE103A05F094
:109F1800F3FF68B1B8EEC80A874AB2EE048A80EE49
:109F2800080A505D05F0A4FD20EE080ABDEEC08ABF
:109F3800824883493A5818EE103A42F2107E1A4481
:109F48007245A8BF72468A42B8BF0A463A5098F886
:109F5800081098F81C00594300EB8000C911C0F1A3
:109F6800000E714503DB8142A8BF01468E4698F872
:109F780012104A431213CEEB0B03B61A664363431F
:109F880002EB66260EEB632B664A39F902100422AF
:109F980091FBF2F16B4A02F19C00405D4143ABEB4F
:109FA800A11398F8511008EE103A51B1101DB8EEEF
:109FB800C80A00EBC500D2ED070AFCF72BFDBDEE81
:109FC800C08ADFF880E1574B0EF1B80139F8030079
:109FD80039F9012029F801000FFA80FC0EF1BC01C3
:109FE8000EF1C400C2EB0C023B584FF0040C92FB7C
:109FF800FCF257F801C07A50634498F8501047F8BB
:10A0080000C0134400EE103A59B10EF15000B8EEFA
:10A01800C00A00EBC500DEED070AFCF7FBFCBDEE4D
:10A02800C00A484901F1B40210EE103A525D534398
:10A038005A1118EE103A01F1680E9819801A01F1B8
:10A04800700329F80E0018EE100AF85001F17C038D
:10A058005242FE5001F188030AF1010AFA500B46F8
:10A068000DB90125FEE62E4A9C6AB2F90410029A3F
:10A0780092790F3252004A4352112A49002AB1F903
:10A0880004104FF0040091FBF0F0A2EB0000B8BF01
:10A098005242322A98F80D100BDC2B4A01FB004182
:10A0A8008A42A8BF0A4629498A42ACBF9A62996285
:10A0B80001E000229A6298F8031001FB00F224499B
:10A0C800097803294FEAA2120CD9B8F84E10B1F555
:10A0D800FA7F07D24842824203DB8A42A8BF0A4677
:10A0E80000E00246996A9A6741F34F31B1F5807FE3
:10A0F800A8BF4FF480716FF0FF008142B8BF0146DE
:10A1080050180022A3F86C00C3F88410C3F89020FC
:10A1180005B0BDEC028BBDE8F08F00BF98110020A0
:10A12800B410002004100020B013002080C1FFFFED
:10A13800F62B0020E01F00204869010824140020A5
:10A14800F0D8FFFF90130020FEFFFF0F020000F081
:10A15800601500202DE9F04F2DED0A8B85B0834660
:10A16800039390F85030029101921BB1322BA8BF93
:10A17800322300E0012307EE903AF8EEE7BADFED6C
:10A18800DE7ADE4B9FEDDECA1B88C7EEABBA002B2A
:10A1980008BF012307EE903AB8EEE7AAD94B2AEE9A
:10A1A8000CCA1B887BEE8CBA9807CCEE2BBA27D545
:10A1B800D54AB2F90030B2F9022083EAE37182EAA3
:10A1C800E270A1EBE371A0EBE27088420446B8BFED
:10A1D8000C46B4F5E17F16DA88429FEDCCBA05DD6E
:10A1E800002AD8BF524207EE902A04E0002BD8BFBD
:10A1F8005B4207EE903AF8EEE77A87EE8BBA04E016
:10A208009FEDC3BA01E0B7EE00BAC24EDFEDC09AC7
:10A21800CDF800B006F1080806F1100906F11C0592
:10A228000024F0EE69AABC49DFF8D8A231F914304D
:10A23800B54909EE103AB8EEC99AF5EE047A29EE56
:10A24800279A31F91430BAF80010BDEEC99A08EE11
:10A25800103AF8EEC97A9FEDB19A89074FEA440798
:10A2680027EE899AB8EEC88A00F08180AC4931F9A6
:10A27800143007EE903AF8EEE77AB0EE007AE8EE9E
:10A28800077A019B5842FDEEE77A17EE901A814251
:10A2980003DB8B42A8BF0B461846A249039B795E95
:10A2A800401A33F91410084407EE900AF8EEE78ACA
:10A2B80005F022FE48B19C49F2EE049A88EEA90AFC
:10A2C800085D05F0D5FB60EE298A9BF81C30DFEDB0
:10A2D800976A0AEE903A9BF8083007EE903AF8EE43
:10A2E800677AF8EE6AAA68EEA77AB1EE047A67EEA2
:10A2F800A67A2AEE877AFDEEE77A17EE901AF1EE43
:10A30800477AFDEEE7AA1AEE903A994208DBFDEE8D
:10A31800C7AA1AEE903A8B42A8BF0B460AEE903AAB
:10A32800D5ED007AE8EE8C7ABBEE0E7AF4EEC77AB9
:10A33800F1EE10FAF8EEEAAA09D4B3EE0E7AF4EECA
:10A34800477AF1EE10FAC8BFF0EE477A01E0F0EE76
:10A35800477AC5ED007A9BF8123009EE903AF8EE8C
:10A36800699A67EEA97ADFED729A67EEA99ABAF848
:10A378000010CA0753D46848385E0028B8BF404266
:10A38800B0F5206F03DD0020C9F8000026E0009B2F
:10A398009FED687A5B7868EE077A07EE103AB8EEB8
:10A3A800477A87EE877AD9ED007A37EE497AE7EE71
:10A3B8000C7A9FED617AF4EEC77AF1EE10FA09D4BF
:10A3C8009FED5E7AF4EE477AF1EE10FAC8BFF0EE30
:10A3D800477A01E0F0EE477AC9ED007A009BD9EDA3
:10A3E800007ADB7A08EE903AF8EE688A8B0768EE16
:10A3F800A77ADFED538A67EEA88A14D538EE6A8A01
:10A40800F0EE6A7AEBEE087A78EEE98AB0EE678ABF
:10A41800F0EE697AEBEE287AF0EE678A03E0F0EE68
:10A42800698AB0EE6A8A474B9FED477A03F19C012F
:10A43800625C9BF8511007EE902AF8EEE77A67EE17
:10A44800C97AA7EE878A51B1181DB0EE480A00EB09
:10A45800C400D3ED070AFCF7DDFAB0EE408A96EDAA
:10A46800007ADFF8E0A0D8ED007AA6EC019A39EE80
:10A47800477A0AF1B40187EE0C7A635C09F10409A2
:10A48800043509EE103A37EE677AB8EEC99AEBEE62
:10A49800877A38EE280AE8EC017A67EE897A9FED28
:10A4A8002B9A27EE899A30EE490A0AF0FFF90AF149
:10A4B8006801BDEEC88AC85318EE103A0AF1700157
:10A4C800FDEEE88AB1EE499A41F82430BDEEC99A0A
:10A4D8000AF17C0118EE903A41F8243019EE103A4E
:10A4E8000AF18801574641F82430009B0133009354
:10A4F80074BB012497E600BF83F9223ED80F0020E1
:10A50800BD37863598110020B41000200000E143C3
:10A51800000000005C14002004100020CDCC4C404A
:10A52800F62B0020E01F0020486901086F12033C49
:10A538000AD7A33D0000A043000040C300004043E9
:10A548000AD7233C90130020A69B443BF7CC9238B3
:10A55800029A584B9479B3F90430640028345C4368
:10A56800554BB3F9043000EE103ABAEECF0A0AF0B0
:10A578009DF96411201A002C07EE900AB8BF6442B6
:10A58800322CF8EEE76A03DD0023CAF8283029E008
:10A59800BDEECAAA1AEE103A23F0030307EE903A6A
:10A5A800B8EEE7AADFED457A9BF80D30CAEE277AB8
:10A5B80007EE103AB8EE477ADAF8283026EE877AAE
:10A5C80067EE277AFDEEE77A17EE902A13443C4AA5
:10A5D8009342A8BF13463B4A9342ACBFCAF82830FF
:10A5E800CAF82820BB6A5B13B3F5807FA8BF4FF475
:10A5F80080736FF0FF029342B8BF134607EE903A9C
:10A60800F8EEE78AFDEEE67A9BF8032017EE903A1B
:10A6180053439B1107EE903A2B4B1B78032BB8EE54
:10A62800E78A14D9BBF84E20B2F5FA7F0FD2FDEEB7
:10A63800C87A534217EE901A994204DB914217EEFA
:10A64800903AA8BF134607EE903AB8EEE78A9BF80F
:10A65800511079B14B0803D09942A8BF194600E0C0
:10A668000121B0EE480A1948D7ED070AFCF7D2F9DC
:10A67800B0EE408A38EE280ABDEEC00A8DED000A19
:10A68800BDF9003000EE103AB8EEC00A0AF00EF933
:10A69800BDEEC88AFDEEE88A0023A7F86C0087EDB6
:10A6A8001E8AC7ED218AC7F8903005B0BDEC0A8B29
:10A6B800BDE8F08FB41000200410002000803B4556
:10A6C800FEFFFF0F020000F060150020A413002019
:10A6D8002DE9F74FA44C00F0C7FB26686568A7680A
:10A6E800861BF643451BC71BED43FF43F60F804609
:10A6F800ED0FFF0F2EB93FB9002D00F07E82B9464D
:10A708002CE04FF0000929E0B14627E003EB8A0B63
:10A71800BBF8023019050ED413F4805F1DBF934AAD
:10A728009BF801101268924A924B14BF52F82120EC
:10A73800126843F82A20BBF80230DA0516D49B05C4
:10A748000AD58D4B1B7813F0040F0CBF8B4A8C4A2B
:10A75800884B126843F82A2009F10109207B8949AE
:10A768005FFA89FA82450B68D0D320E050465946F3
:10A77800854A03F041FD854B1B88580603D5504692
:10A788005946834A10E0590703D550465946814A2D
:10A798000AE09A0703D5504659467F4A04E0DB078A
:10A7A800DAD57E4A5046594603F026FDD4E7DFF84D
:10A7B80004E20093BEF906307822A3F57A73534376
:10A7C8004FF47A7293FBF2F303F22B1301930022F6
:10A7D800F3465FFA82FE864517D2009B03EB820E92
:10A7E800BEF802E01EF4806F0DD0DFF88891019B5F
:10A7F80039F822E040F2671A9E449EFBFAFC0AFBF5
:10A808001CEE29F822E00132E3E74DB308F5C33323
:10A81800A0336360637B544A13BB9373604B1B681C
:10A8280013F0020F0AD0DFF890E19EF800E0BEF1C5
:10A83800000F03D04FF0010E82F80EE0DA0506D5BE
:10A84800584B5B791BB1A37B43F00203A3734A4BBC
:10A858001B7813F0050F02BFA37B43F00403A37317
:10A8680094F80EE0BEF1000F03D13F4B5B7B002B49
:10A878004FD094F80DC01CF0010FACF10C031DD1A2
:10A88800BCF1030F07D8DFF8E8903C4A1EF0040F2C
:10A8980008BF4A4600E0364AACF1040CBCF1070F89
:10A8A80005D8DFF818C11EF0010F18BF6246DBB2E9
:10A8B800032B0ED81EF0020F3B4B06E0DBB2032B36
:10A8C80006D82F4B2A4A1EF0020F18BF1A4600E07E
:10A8D800274A4FF0000C5FFA8CF383420DD20B68C5
:10A8E80003EB8C035B881B0642BF224BD2F8009017
:10A8F80043F82C900CF1010CEDE785B1BEF1000F87
:10A9080008D0637B184A0133DBB2142B06D100232D
:10A9180004E025B1637B002BF3D100E05373002ED4
:10A9280050D0224AB2F90250B2F90020002DB8BF27
:10A938006D42002A4FF03203B8BF524295FBF3F53F
:10A9480092FBF3F2EDB2D3B2AB4238BF2B46184AB2
:10A9580013B192FBF3F300E0134643442360E37B17
:10A96800014A6BBB01232CE080140020181D002035
:10A97800987E01087A0D0020FD2B0020A07D01089B
:10A98800907D0108801300204A6901089811002071
:10A9980050690108566901085C6901086269010883
:10A9A800E81F0020040E0020A87D0108B410002034
:10A9B800400D03002420002020110020B07D010854
:10A9C8000023D3738E4D8F4B2D78E27BADB9002FCA
:10A9D80000F00E818C4B267B1A788C4B8C4D93F8AB
:10A9E80000C08C4BD3F800E00B6802F00402002191
:10A9F800D2B203EB86060F46B5E01AB9864A1A6149
:10AA0800002508E0854AFAE70A68AB00D618768878
:10AA1800760604D40135EBB28342F5D3D7E7804EEE
:10AA2800B6F90060192E25DD12F803E094F814C079
:10AA380026690EF00F09E1450CDCDFF8C8C19CF867
:10AA480015C0BCEB1E1FDEBFDFF8D8E1D6F800C08A
:10AA580043F80EC012F803E094F816C00EF00F0980
:10AA6800E14533DBDFF89CC19CF815C0BCEB1E1F29
:10AA78002CDC26E0193629DA12F803E094F814C021
:10AA880026690EF00F09E1450CDCDFF878C19CF867
:10AA980017C0BCEB1E1FA2BFDFF888E1D6F800C0C4
:10AAA80043F80EC012F803E094F816C00EF00F0930
:10AAB800E1450BDBDFF84CC19CF817C0BCEB1E1F4F
:10AAC80004DBD6F800E0574E43F806E0544EB6F9DA
:10AAD8000260192E1BDD12F803C094F814E02669F1
:10AAE8000CF00F09F1450CDCDFF8189199F8159076
:10AAF800B9EB1C1FDEBFDFF82CC1D6F8009043F875
:10AB08000C90D25C02F00F0CF4451EDD82E719367A
:10AB180080DA12F803C094F816E026690CF00F09E1
:10AB2800F1450CDBDFF8DC9099F81590B9EB1C1FA8
:10AB3800DEBFDFF8F0C0D6F8009043F80C90D25C86
:10AB480002F00F0CF445FFF665AF94F817E0BEEB82
:10AB5800121FA2BF334A36689E505BE7588800052B
:10AB680004D404330435B342F8D122E04AB101EBEE
:10AB78000C0A06209AFBF0F900FB19A001280DDC4D
:10AB880001E057B9012793F801900EEB89003EF8D0
:10AB980029A090F80290C07803E01746002081466B
:10ABA8008246013125F802AC85F800906870C9B278
:10ABB800D7E7164A1378013B13F0FF0308BF0623B3
:10ABC8001370114B1B785B0741BFBBF90630A3F527
:10ABD8007A7303EBC3034FF47A7243BF93FBF2F328
:10ABE8000133DBB20123104A92FBF3F34344A36021
:10ABF80003B0BDE8F04F02F0A7BD03B0BDE8F08F89
:10AC0800330E002080140020FD2B00208C00002033
:10AC18007C0D0020181D0020AC7D0108987E0108DD
:10AC2800B41000207A0D0020400D0300034B4FF4B0
:10AC3800085208B19A6170471A8570470010004899
:10AC4800034B4FF4085208B11A8570479A61704750
:10AC5800001000480C4B1B6893F90220824209D06F
:10AC680093F90A20824207D093F91220824208D130
:10AC7800022002E0002000E0012003EBC0000230C7
:10AC880070470020704700BF5012002038B1438839
:10AC980011EA030003D08B420CBF01200220704749
:10ACA80030B50A4B0A491C680A78022A0AD81346A2
:10ACB80004EBC303551CEAB29D882842F5D00A70FC
:10ACC800981C30BD0A70002030BD00BF5012002013
:10ACD80098140020014B00221A70E1E79814002014
:10ACE8002DE9F047877890F803C0214DBBB2C7F132
:10ACF800640E03EB83065C42C3F178005FFA8EFEB4
:10AD08007600CCF16408A4B280B2A3B20FFA83F93A
:10AD1800B9F1000F05DC002B14BFBA464FF0010A49
:10AD280000E0F24613FB03F303FB0CF21AFB0AF3F1
:10AD380092FBF3F3434403FB09F30A2293FBF2F378
:10AD480033449BB225F8023FB1F800904A880A3490
:10AD5800C9EB020AA4B21AB202FB0AF24FF47A73E0
:10AD6800844292FBF3F34B442B80CED1BDE8F087AD
:10AD78009814002010B544780078002202FB02F3F2
:10AD8800193B634303F6C413534340F6C4114343CA
:10AD980093FBF1F3034921F812300132072AEDD170
:10ADA80010BD00BFB21400200430114B33F910005D
:10ADB800B0F5617F10B506DB40F6330398420246D2
:10ADC800A8BF1A4601E04FF461720C78192340F2CB
:10ADD800833013FB0404944207DA497813FB010318
:10ADE8009342B4BF0020012010BD002010BD00BF59
:10ADF8002420002010B500F1500302788A4203D1C4
:10AE08008478C278944204D304309842F5D1002063
:10AE180010BD012010BD1FB5084B1B681B030AD5C8
:10AE28008DF8040001230D2001A98DED030A8DF88A
:10AE38000530FCF761FD05B05DF804FBE81F002054
:10AE48001FB5084B1B681B0309D58DF80400029138
:10AE580000230D2001A98DF80530FCF74DFD05B044
:10AE68005DF804FBE81F002010B5094A094B11687A
:10AE78009B6812689142F8D1074A946A4FF47A7035
:10AE880000FB04F2D31AB3FBF4F300FB013010BD4E
:10AE98000C20002010E000E09814002038B504468B
:10AEA800FFF7E2FF0546FFF7DFFF401BA042FAD39A
:10AEB80038BD10B504462CB14FF47A70FFF7EEFF99
:10AEC800013CF8E710BD2DE9F04F06468A4890F995
:10AED800004087B0B44288469DF8445011461A464F
:10AEE8009DF8403009D090F90C40B44207D090F951
:10AEF8001840B44209D1022702E0002700E00127E8
:10AF08000C2404FB0700047A0CB10020F0E0012EA9
:10AF180000F0DD80142E05D0002E40F0E88000956A
:10AF28007648D6E0DFF814A2DAF8183043F00103C7
:10AF3800CAF81830DAF814304FF0904543F400336B
:10AF4800CAF814304FF0010903224FF4805B04A9BA
:10AF58004FF090408DF815200392CDF810B08DF881
:10AF680014908DF816908DF81740FBF7DDFBA5F8C7
:10AF780028B0C820FFF79DFFC5F818B0DAF81430DC
:10AF8800039A43F40033CAF8143028464FF4C053E8
:10AF98004FF0020B04A904938DF815208DF814B016
:10AFA8008DF816408DF81740FBF7BEFB6B6A23F44B
:10AFB80070436B626B6A43F460436B626B6A23F4A1
:10AFC80070236B626B6A43F460236B624C4B4D4D8C
:10AFD8004FF480221A6002F18042A2F53F32122318
:10AFE800EB65082385F86130136885F8629023F4CF
:10AFF80080231360536823F48023536095F86030EE
:10B0080003F1804303F582331A6842F480221A6000
:10B01800EA6D3D4B22F01F0002F01F02C15809FAE9
:10B0280002F221EA0202C250EA6D384922F01F00FA
:10B0380002F01F0250F801E009FA02F22EEA0202B9
:10B048004250EA6D22F01F0102F01F02C85809FAA7
:10B0580002F20243CA502E4B2E4A1C60DAF81C300A
:10B0680043F40003CAF81C302B4B04A8DA608DF8AF
:10B0780010608DF811B08DF812408DF8139004F01F
:10B08800ADFC2A238DF810309DF813308DF81190FF
:10B098008DF812401BB104A804F0A0FC04E01F4B7B
:10B0A8004FF48062C3F884201D4B1E4C1C600223A1
:10B0B80085F86C301C4A1D4B1D49C5F8803011605D
:10B0C8001B6898471B4BEB62A4F1380006E01A484E
:10B0D800009501F091FA00283FF417AF064B06716E
:10B0E8000C2202FB073787F80880786000E02046CA
:10B0F80007B0BDE8F08F00BF5412002000380140AF
:10B108001404014098140020080401400C04014074
:10B11800D80042420005FA0500ED00E000E100E039
:10B12800A4110020FC140020A81100201C000020FD
:10B1380090000020686901080044004000100240A7
:10B14800024A136801331360704700BF0C200020C7
:10B15800024BD3F8843003B1184770479814002085
:10B16800014B1B68184700BFE02B002010B50020DA
:10B17800FFF7F6FF074B00241C7005F0D3FF064BC2
:10B1880083F88840C3F88C40A3F89040C3F89440F3
:10B1980010BD00BFC82B00209814002010B510B9AE
:10B1A800BDE81040E2E700230C225A430C4C111969
:10B1B800125D824203D00133102BF5D110BD094B2B
:10B1C800D3F8940018B14A784078824206D2002217
:10B1D800C3F89410A3F89020C3F88C2010BD00BFCA
:10B1E800486E01089814002010B540001428A8BF24
:10B1F80014200023074A022199540B449918142457
:10B20800834201F8014CF5DBFF21D1540F20BDE842
:10B218001040C3E7C01F002038B5174B4FF48842D1
:10B2280040F2DB159A6168434FF488521A85851EEF
:10B238000B24013C14F0FF0417D00F4A938A9BB2E9
:10B2480083F488439382938A9BB283F488539382CE
:10B258002846FFF72EFE0120FFF782FF1920FFF78F
:10B2680028FE0020FFF77CFFE3E7044B044A1A603E
:10B27800044B054ADA6038BD00100048FC9F0020E6
:10B28800EFBEADDE00ED00E00400FA0503681B69BF
:10B2980018470368DB68184703689B681847036802
:10B2A8005B68184703681B6818472DE9F84FB0F921
:10B2B8000230934218BF00232DED028B18BF037094
:10B2C800057804460E469146002D40F08B8007EE27
:10B2D800902A9FED770AF8EEE77AB6EE008A27EE15
:10B2E800800ADFED747A20EE270AA04620EE080ACD
:10B2F80009F052FBDFED706A60EE266AB7EE006A6D
:10B30800B0EE667AA0EE007A40F2DC536365D0EEC8
:10B31800006A1023A4F8523037EE067A76EE866A71
:10B32800C6EE077A1823A4F85030274684ED046A3D
:10B3380027EE807A27EE007A77EE075A84ED017AB5
:10B34800C4ED025A70EE005A84ED037AB8EE007A22
:10B35800A5EE807A27EE877A67EEA67A84ED057ADD
:10B36800C4ED067ADFED557A98ED047A27EE277A50
:10B37800F0EE678AB5EEC07AF1EE10FA4CBF77EEC0
:10B38800487A77EE087A013517EE900A06F0A6F8A3
:10B39800D8ED017A67EEA87AC7E90E01F5EEC07A12
:10B3A800F1EE10FA4CBF77EEC87A77EE887A08F19A
:10B3B800040817EE900A06F091F8032DC7E9080172
:10B3C80007F10807CED1A6F2DC531B042367E36715
:10B3D8006367C4F88030A367C4F884300123A4F8F5
:10B3E80002902370D4F85490B4F95280636A276AA3
:10B3F800206FE26FD4F840C0D4F88010C4F88020E1
:10B40800C9EB060606FA08F64FEAE67B734307FB24
:10B418000B332667A7FB06671F44636C656F60677D
:10B428004FEAE27B53430CFB0B3EACFB0223734415
:10B43800B61A67EB0307E36AA26AC4F884104FEAF6
:10B44800E07B434302FB0B3EA2FB00237344B61888
:10B458005F41E36CA06CB4F95020A5674FEAE17B2B
:10B468004B4300FB0B33A0FB01011944636B361AF5
:10B47800206B4FEAE57B05FB03F300FB0B3367EB1F
:10B488000107A0FB050119448019794105F0FCFF6B
:10B4980008F1FF3201239340E067C01841EBE371E4
:10B4A800424605F0F1FFBDEC028B4844BDE8F88F39
:10B4B8006F12833ADB0F4940F404B53F0000804B1C
:10B4C8002DE9F8430024244B93F8C860E0B2B04259
:10B4D8000DD203EB8003214AD3F8983032F81010CC
:10B4E8001BB10B2801D8DB6898470134EBE71C4BEC
:10B4F8001B685B032DD500242346E2B2B24228D252
:10B50800DFF8549009F198074FEA840857F8242087
:10B5180055689D4215D0284602F0BEFDEFF3128310
:10B52800502282F3128828216A6A01FB00900132B6
:10B53800C0F8F0206A6942F001026A61DBB283F365
:10B54800118857F808301B6800221A6001342B460E
:10B55800D3E7BDE8F88300BF98140020241000202A
:10B56800E81F002008B50E4B1B6813F4805F0D4BD5
:10B5780014BFD3F8E421D3F8E82193F8C8109288CF
:10B588000023D8B2884204D2074820F81320013398
:10B59800F7E7FFF795FF3220BDE8084089E400BFD0
:10B5A800E81F002098140020241000200A4B1A6875
:10B5B8000A4B30B502F48052D3F8E441D3F8E8518D
:10B5C80000230AB1A18800E0A988054820F81310D3
:10B5D80001330C2BF5D130BDE81F00209814002052
:10B5E800961F002070B5124D0024214605F2ED107B
:10B5F800702285F8EC4108F04AFF2146D5F8603200
:10B608000B4A0B4493F9020080B102F2ED141E6854
:10B618000E5108199C8884809B79837192F8EC31CB
:10B6280007310133702982F8EC31E7D170BD00BFD2
:10B6380098140020094B1A680E2303FB0020437A54
:10B64800FF2B07D0064A12789A4203D9054A32F8E6
:10B65800130000E0808800B2704700BF1C1D002066
:10B66800481200202420002038B5294C2DED048BE9
:10B6780094ED998AB0EE480A0546FBF77BFCF0EE9C
:10B68800408AB0EE480AFBF712FC94ED9A9AB0EEA5
:10B69800408AB0EE490AFBF76DFCF0EE409AB0EE36
:10B6A800490AFBF704FC95ED017AD5ED027A95ED90
:10B6B800006A68EE676A27EE088AE7EE286A68EE8D
:10B6C800000A67EE807AE6EE290AB0EE660AE7EE2F
:10B6D800A80A09F0EDF9DFED0F7A20EE270ADFED71
:10B6E8000E7A80EE270AD4ED9B7A30EE270AF2EE26
:10B6F800047A80EE270A09F0D9F8BDEC048B83B2EE
:10B708001A0444BF00F5B47083B218B238BD00BF44
:10B71800981400200000E144DB0F494001380A4B2F
:10B72800042804D8DFE800F00507090B0D00074AD4
:10B7380008E0074A06E0074A04E0074A02E0074A29
:10B7480000E0074A1A6070471401002025FF00082E
:10B75800D197000851020108259E0008919A000817
:10B768005DA1000882B01B4B1B4A8DF807101968B1
:10B77800106860B31268052A29D1184A106810BBEE
:10B788009DF808109DF8073043EA012314490B80FF
:10B79800144B1968144B89B20B445B0019680121DA
:10B7A800196013680B441360104A136823F4E043CC
:10B7B80023F040039BB283F0300343F4004343F08B
:10B7C8008003136003E01A68521A312AD5D902B0EF
:10B7D800704700BF0C200020E42B00200817002031
:10B7E80080610040505C00400A300020045C00404A
:10B7F800014B5868C0B270470817002001207047F5
:10B808007047704720B9034B1B6808221A8270479B
:10B8180001487047A4110020B400002020B9034B50
:10B828001B6808221A82704701487047A41100203B
:10B83800B400002021B901288CBF022000207047E5
:10B848000220704710B5094B1A68D378042B0BD81F
:10B85800074C518ADB00234418B99B895B1A138271
:10B8680010BD9B68581810BD002010BDA411002001
:10B87800B4000020054B1968054B4A8A18B99B8DFE
:10B888009B1A0B827047986A10447047A4110020D5
:10B89800B4000020054B1968054B4A8A18B99B8EDD
:10B8A8009B1A0B827047186B10447047A411002034
:10B8B800B4000020074B1B681B7803F07F03212B83
:10B8C80006D100F0DF00022814BF022000207047D4
:10B8D80002207047A4110020212810B508D1114B6F
:10B8E8001B681B7803F07F03212B10D0022010BDAA
:10B8F8002028FBD10B4B0C4A1B681B78107003F0F7
:10B908007F03212B094B18BF00230BB9EEE7084B27
:10B91800044A1268002493615482204698472046BE
:10B9280010BD00BFA4110020002C00200DB8000895
:10B9380025B80008704707EE900AF8EEE77ADFEDC1
:10B948000C6A9FED0C0AF5EEC07AF1EE10FAD4BF3E
:10B95800B1EE677AC7EEA67A08B5D8BFC7EE267AE1
:10B9680027EE800AFBF706FB034B83ED000A08BDB0
:10B978008096184B35FA8E3C08010020F7B51C4B11
:10B988005A681D460AB95C6800E00124187A00214B
:10B99800CAB2A24201F1010107D202AE2F18164421
:10B9A8003A44527A06F8042CF2E75A68121B5A6095
:10B9B8001A7A5D6822441A729DB903204021FAF769
:10B9C8008FFB0C4A136823F4804323F070039BB267
:10B9D80083F4405343F4004343F080031360044B63
:10B9E8001D72002CCBD09DF8040003B0F0BD00BF41
:10B9F800081700200C5C0040F8B5A84B1B680546EA
:10BA0800187818B1012800F0838106E3242DA44C8E
:10BA18000CD006D80A2D00F0EC800D2D00F0E9803E
:10BA28005CE12A2D09D02C2D07D057E184F8490074
:10BA380084F84A0084F84B0066E19A4B94F84A105F
:10BA480094F84970964A0020585447BB197882F8F0
:10BA58004C70472923D15978502920D19978472902
:10BA680008D1D978472905D11979412902D101216D
:10BA780082F84C1099788B4A522903D1D1784D29F4
:10BA880000F0CD829978874A472908D1D17853297F
:10BA980005D11279562A04BF032284F84C2094F861
:10BAA8004C207F4E022A3BD0032A50D0012A40F076
:10BAB8008A80BA1E072A00F28680DFE802F00408AE
:10BAC8000F131A25842B04F061F920657BE01B789D
:10BAD800532B78D1236D5B42236574E004F056F94B
:10BAE800606570E01B78572B6DD1636D5B426365B1
:10BAF80069E01B78302B6C4B1A788CBF42F002023D
:10BB080022F002021A705EE0002004F09FF984F827
:10BB1800580058E0002004F099F9A4F85A0052E0BF
:10BB2800072F07D0082F4ED1012004F08FF9A6F86F
:10BB38005E0048E0012004F089F941F218435843B7
:10BB48004FF47A73B0FBF3F0A6F85C003BE0022FE9
:10BB580007D0032F0BD1002004F078F9534B18704D
:10BB680031E0002004F072F986F860002BE02AD951
:10BB78003A1F921096F860300132D2B2013B02EBC4
:10BB88008303DBB2102B1ED8F91EC2F1010201EBB0
:10BB98008202D2B2012A0BD0042A11D100205E1EE3
:10BBA80004F054F9424B9855424B00229A5507E04D
:10BBB8005E1E414A0020935504F048F93F4B9855C2
:10BBC800636E01336366364B2A2D18BF93F84B20FA
:10BBD80007F101074FF000000CBF0122554084F81F
:10BBE800497084F84A000CBF83F8682083F84B50EA
:10BBF8008AE094F8680000284CD0314B13F8012DE6
:10BC080030495A708B42F9D1264A254D137852781B
:10BC1800402B85BF373B1B011B01DBB298BF03F0EC
:10BC2800F003402A8CBF373A303AD2B2134494F822
:10BC38004B20DBB29A422AD121230B7095F84C0095
:10BC4800EB6E204A01330128EB660CD0022820D184
:10BC5800722313701C4BB5F85C201A801B4BB5F887
:10BC68005E201A8015E0672313700F4B1B789F071F
:10BC780010D5174B2A6D1A606A6D5A60154B95F8E6
:10BC880058201A70144BB5F85A201A8002E03F2346
:10BC98000B700020002384F8683035E0CC060020C3
:10BCA8000817002014200020D41000205C10002069
:10BCB8008D1000207D1000205D1000206D100020E8
:10BCC800300300201C030020D61000204410002060
:10BCD800DC100020DA100020D810002094F84A3038
:10BCE80094F868000E2B9FBFB14A591C82F84A107D
:10BCF800B04A98BFD554AE4A28B992F84B305D4047
:10BD080082F84B5000E00020003018BF0120F8BD39
:10BD1800A74B93F870100022082900F27E81DFE813
:10BD280001F0050C101A2B3C63828F00B52D40F0F2
:10BD3800748183F87120012253E0622D08BF02222A
:10BD48004FE0032283F8702083F8725083F8735011
:10BD580083F8745061E1042283F8702093F873200B
:10BD680093F8741083F875502A44D2B283F873207C
:10BD78000A4483F8742050E1052283F8702093F870
:10BD8800732093F87410A3F876502A44D2B283F83B
:10BD980073200A4483F874203FE1062283F8702058
:10BDA80093F8732093F874102A44D2B283F873205E
:10BDB8000A4483F87420B3F8762002EB0525ADB267
:10BDC800B5F5AC7F88BF7A4AA3F8765084BF0121C5
:10BDD80082F871100022A3F87820002D40F01D8110
:10BDE800072283F8702018E193F8732093F87410F1
:10BDF8002A44D2B283F873200A4483F87420B3F833
:10BE08007820B2F5AC7F3CBF6949891802F101027C
:10BE180038BF81F87C50B3F8761092B29142A3F8FB
:10BE28007820DDD9F9E0082283F8702093F8733080
:10BE3800AB4200F0F2805E4B012283F871200FE0E4
:10BE48005D4C83F8702014F8012D62705B4A9442AF
:10BE5800F9D193F87410564AA94206D03F232370AB
:10BE6800574A536801335360D7E0D16E92F8710096
:10BE78000131D16610B13E232370CEE0212121701B
:10BE880092F87510062944D004D8022907D003294E
:10BE980026D0F8BD12295CD030296CD0F8BD5021CD
:10BEA80021704849D2F880404C60D2F884400C6038
:10BEB800D2F88C104FF47A7491FBF4F1424C218043
:10BEC80092F8D411414A19B1117841F0020102E007
:10BED800117821F002011170012283F8D5218EE03A
:10BEE8005321217092F88110CE0705D592F8802051
:10BEF800D51E6A426A4100E0024602F0010183F859
:10BF0800D411002A7BD131490A7822F002020A7042
:10BF180075E04F21217092F88710CC0705D592F86B
:10BF28008620D11E4A424A4100E0024602F0010141
:10BF380083F8D41122B925490A7822F002020A703E
:10BF4800234A93F8AB101170224AB3F8A810118055
:10BF580055E0562121702049D2F890400C8042F2D9
:10BF68001074D2F8941091FBF4F11C4C218001213B
:10BF780082F8D61143E04921217092F88010184ABE
:10BF8800102988BF10211170164914780022A24286
:10BF980032D2154D0E7A5655144D4E7A5655144DCB
:10BFA800CE7A5655134D11F80C6F56550132EEE7FF
:10BFB8000817002014200020300300201C03002054
:10BFC800AC060020DC100020D8100020D41000207F
:10BFD800DA10002012010020D610002044100020A2
:10BFE8005C100020841700205D1000206D100020D8
:10BFF8007D1000208D1000205A6E01325A6693F889
:10C00800D5310B4A9BB192F8D63183B1002182F821
:10C01800D51182F8D6111846F8BD0020F8BD12795E
:10C02800432A7FF42FAD022284F84C202AE5F8BD7C
:10C03800081700200449054B0968187000225A6146
:10C0480099611A77704700BF0C200020AC060020C9
:10C0580010B5121A07EE902A5B1A2DED028BF8EE36
:10C06800E78A07EE903A184B059CB8EEE78AD3EDBD
:10C07800007A28EE278A28EE080AA8EEA80A08F00F
:10C0880019FDDFED127A049B20EE270AF0EE480A2C
:10C09800BCEEC00A83ED000AB1EE680A08F008FD9C
:10C0A800DFED0B7A9FED0B7AE0EE077ABDEC028BA1
:10C0B800FDEEE77A17EE903A002BBCBF03F50C4370
:10C0C800A033236010BD00BF080100202C7D8E3FE7
:10C0D80000A00C46A00CB34544F25063984203DD1F
:10C0E800A0F50C40A0387047034B9842BCBF00F540
:10C0F8000C40A030704700BFB0B9FFFF73B51A4CB1
:10C10800036823600B686360184D0068184EFFF7DA
:10C1180012FC184B009395E8030094E80C00019674
:10C12800FFF796FF144B32681A6068686368134912
:10C138001B1A07EE903A124B286893ED007A236891
:10C148001B1A0B600F4BF8EEE77A1A600E4B67EE7E
:10C15800877A1B68FDEEE77ADA880C4BC1ED017A25
:10C168001A8002B070BD00BF341F0020DC10002010
:10C17800401F00203C1F00207C1F0020441F00207F
:10C1880008010020741F0020100F0020701F0020DD
:10C198004279DFED2A5A2A4B9FED2A5A07EE902A58
:10C1A800F8EE677AC27BC7EEA57AB2EE047AC3EDE1
:10C1B800007A07EE902AF8EE677A234ADA60C7EE2B
:10C1C800A57AC3ED017A8179204B07EE901AF8EE33
:10C1D800677A017CDA60C7EE877AC3ED007A07EEEA
:10C1E800901A817E06EE101AF8EE677AB8EE466A63
:10C1F800C7EEA57A86EE056AC3ED017A83ED026A79
:10C20800C179134B06EE901A417CDA60F8EE666A43
:10C21800C6EE876A07EE101AC17EC3ED006A07EE04
:10C22800901AB8EE477AF8EE677A87EE257AC7EE65
:10C23800857A83ED017AC3ED027A70470000C8421F
:10C248004C1F002000007A440000FA445C1F0020C4
:10C25800801F002010B50C4C23789B0713D50B4B7F
:10C268001B78042B0FD90A4A0A4B106852685A6087
:10C278001860FFF760FB084B1A88084B1A80237870
:10C2880043F00103237010BDD4100020DA10002001
:10C29800DC10002048100020B0100020901F002063
:10C2A8001C4B1B681B0307B530D51B4A1B4BD2ED33
:10C2B800007A1B788DF80030B2EE047A67EE877A40
:10C2C800174B9FED187A1B788DF80130FCEEE77A52
:10C2D8000A2017EE903AD2ED017A8DF8023067EE17
:10C2E800877A6946FCEEE77A17EE903AD2ED027A41
:10C2F8008DF80330FCEEE77A17EE903A8DF80430AB
:10C30800094B1B788DF80530FBF7F6FA03B05DF89A
:10C3180004FB00BFE81F0020FC1F0020DA1F0020DC
:10C32800F81F002000007A44DE1F0020054A137819
:10C3380083F001031370044A00231360034A136057
:10C34800AEE700BFDE1F0020F41F0020F01F002012
:10C358000A4B10B519684FF6FB720A401A60084A72
:10C36800927A1C46074B0AB1052200E001221A60A6
:10C3780003F0D6F94FF43643236010BD405C00400B
:10C38800FC140020E42B002010F80A3C0133DBB237
:10C398000A2B84BF10F8131C044A00F80A3C82BF19
:10C3A800002322F8113000F80A3C7047142B0020B3
:10C3B800334A136C90681944081A40F68C23984243
:10C3C80070B513469160D06051603BD9127893F9EB
:10C3D80045108A4210460BD1111F082908D893F836
:10C3E8004610182901D8013103E083F8442002E0FF
:10C3F800002183F8461093F944402149A24219D1FB
:10C4080091F84740B4B10C310024944206DA1D4D2E
:10C4180051F8046F25F814600134F6E70C2805D0AC
:10C428001849002421F810400130F7E71648017830
:10C438000131017083F84520002201211A7083F828
:10C44800471070BD92F84710C9B1A0F2EF2440F22E
:10C45800DA518C4208D811780B2905D80B1D013107
:10C46800117042F8230070BD002283F84720074B63
:10C4780003F13002002143F8041F9342FAD170BD42
:10C48800C0010020142B002084060020CC010020CD
:10C49800024A136C0133194411647047C00100202B
:10C4A800024B53F820301B68196070473015002084
:10C4B800064B53F820301A681B89A1F57A71594345
:10C4C8004FF47A7391FBF3F1116070473015002037
:10C4D800F0B5046D8668236823F00103236083792F
:10C4E800054613F0020F40790CBF4FF0000E4FF4D1
:10C4F800005E13F0040F14BF4FF48067002710F09C
:10C50800010F14BF042100218307206820F00100D7
:10C518002060626822F440524EEA02026260226899
:10C5280022F4B05323F00C0348BF41F008013B4309
:10C538000B432360A36895B023F44073A360684657
:10C54800F9F77CFF284B9C4201D10C9B0EE0274B4E
:10C558009C4201D10D9B09E0254B9C4201D10E9BC9
:10C5680004E0244B9C420CBF0F9B109B2268A879C7
:10C57800170448BF5B00B3FBF6F206FB1233B3EBBC
:10C58800560F236828BF01321E0441BF4FF6F073CF
:10C59800C2F34201134041EA03026B7992B213F0ED
:10C5A800020FA28100F0010114BF4FF400320022F3
:10C5B800DC0748BF42F480322B6D11B159680A4339
:10C5C80002E0596821EA02025A609A6801074CBFE2
:10C5D80042F0080222F008029A601A6842F001024A
:10C5E8001A6015B0F0BD00BF00380140004400409B
:10C5F80000480040004C00402DE9F0471E46A14B82
:10C608008CB09842894690469DF8507040F08580DD
:10C618009D4B9E4A1A609E4A5A6102F580729A6141
:10C628004FF48072DA601A619A4A1A63143A5A63AC
:10C63800A2F54842203ADA6404329A64C3F80880C2
:10C648001865954B9A6942F480429A615A6942F09A
:10C6580001025A6102238DF80830032317F0010AFA
:10C668008DF809304FF000038DF80A3014BF02230B
:10C6780001233A078DF80B3019D54FF090444FF449
:10C68800007501958AF001038DF80A30636A23F07A
:10C69800F0036362636A43F070036362204601A992
:10C6A800FAF742F8BAF1000F27D1A56125E0B307E0
:10C6B80010D50CA94FF4007341F82C3D4FF0904071
:10C6C800436A23F0F0034362436A43F07003436212
:10C6D800FAF72AF8F50710D50CA94FF4806341F84A
:10C6E8002C3D4FF09040436A23F470634362436AE1
:10C6F80043F4E0634362FAF717F80E238DF800302D
:10C708000022012368468DF801308DF802208DF84B
:10C7180003305D4C03F062F973E0604B984240F0DF
:10C7280005815F4B594A1A604FF48072DA601A61CA
:10C738005C4A5A6102F580729A61574AC3F80880C8
:10C748001865D36943F40033D36102238DF80830A8
:10C75800032317F0010A8DF809304FF000038DF814
:10C768000A3014BF022301233C078DF80B3017D57C
:10C778004D4C202501958AF001038DF80A30236A73
:10C7880023F470032362236A43F4E0032362204600
:10C7980001A9F9F7C9FFBAF1000F23D1A56121E07A
:10C7A800B0070ED50CA9202341F82C3D3E48036A5A
:10C7B80023F470030362036A43F4E0030362F9F7A6
:10C7C800B3FFF1070ED50CA9402341F82C3D36489C
:10C7D800036A23F070630362036A43F0E063036251
:10C7E800F9F7A2FF26238DF80030002201236846BE
:10C7F8008DF801308DF802208DF8033003F0EEF843
:10C80800274CC4F82C900025012384F84430256275
:10C81800E561A56265626671C4F80880A771204663
:10C82800FFF756FEF20748D5236B002B3ED001A830
:10C83800F9F722FDE36C01934FF480530A938023A8
:10C848000693E368ADF8103020230993206B6369E1
:10C8580002930B950595079508950395F9F737FD0C
:10C8680001A9206BF9F715FD236B216D1A6842F0B9
:10C8780001021A608A6842F040028A605B689BB2D3
:10C8880023641AE000380140741E0020206A010861
:10C89800E018002058000240001002400044004008
:10C8A800201E0020E01A0020000C0048236D2022E2
:10C8B8001A621A6842F020021A60B3072FD5636B18
:10C8C80043B301A8F9F7D8FCA36C01934FF4805344
:10C8D8000A93802306932369ADF8103000251023AE
:10C8E800606B03930B950595079508950995F9F7DE
:10C8F800EEFC606B01A9F9F7CCFC636B1A6842F097
:10C9080002021A60226D5D605D60936843F08003E7
:10C91800936004E0226D136843F080031360226D76
:10C92800136843F001031360204600E000200CB0B8
:10C93800BDE8F0873D4B1B78012B30B514BF0024B0
:10C948000324B1B9036A23F0010303628169036A0E
:10C9580021F0F30123F00A0341F0010142F0010242
:10C968001A4341EA041181610262836923F00C03CE
:10C978001BE004291DD1016A4FF6EF730B400362D7
:10C988008169056A120121F473414FF65F7342F021
:10C99800100241F480712B4092B2134341EA0431F2
:10C9A80081610362836923F44063836183698361DE
:10C9B80030BD0829016A1AD14FF6FF630B400362A4
:10C9C800C169036A9BB289B223F4206343F480737C
:10C9D80021F0F30143EA022241F0010192B241EA57
:10C9E8000411C1610262C2694FF6F37319E04EF691
:10C9F800FF730B400362C369056A40F6FF411940A3
:10CA080045F6FF732B4043F4805343EA023241F466
:10CA1800807192B241EA0431C1610262C2694FF287
:10CA2800FF331340C361C369C36130BDBC0100203B
:10CA380038B510F80E2C50F8043C044652B90122BF
:10CA480000F80E2C20F80C1C997A18680222BDE810
:10CA580038406FE730F80C2C20F80A1C891A89B284
:10CA680020F8081C074A10F80F0C002522F81010AF
:10CA780004F80E5C1868997A2A46FFF75BFF04F8F9
:10CA8800065C38BD142B0020044B53F820301BB132
:10CA980007289CBF1B681960704700BFE802002088
:10CAA80038B500240B4D6059254402F0E3F9696854
:10CAB80011B10948FAF7CDF9A96811B10748FAF791
:10CAC800C8F90748103402F0D5F9B4F5E07FE9D188
:10CAD80038BD00BF386A0108C6850108CC85010841
:10CAE8004B8F010870B50546284607F014FD064629
:10CAF80058B91A4B1A485A791A4B03EB8203BDE806
:10CB08007040D3F8BC11FAF7A4B928461649324642
:10CB180007F00AFD60B91548154C02F0ABF954F856
:10CB2800041F19B11348FAF794F9F8E7124805E019
:10CB38000024124B53F8241021B91148BDE8704065
:10CB480002F098B92846324607F0EEFC0134002876
:10CB5800EFD1024B0B4D5C71C6E700BF48200020A7
:10CB6800D2850108386A0108DE850108E3850108D5
:10CB7800F46B0108F68501084B8F0108F86B010872
:10CB880006850108E2810108F0B585B0044607F082
:10CB9800C2FC082826D1621EE01D1F4912F8013F79
:10CBA80009681944497801F00301022908BF203BAC
:10CBB80082421370F1D1254604F1080715F8016B7C
:10CBC8001648314607F099FC20B12846314607F04F
:10CBD80094FC10B1FBF73EFB1CE0BD42EED12046B1
:10CBE800F9F73EF90E4802F045F900230D4A1A44B8
:10CBF80004A992F88A210A440849595C02F80C1CD5
:10CC08000133082BF2D1002307488DF80C3001A915
:10CC1800FAF71FF905B0F0BD2001002016830108BE
:10CC2800FA85010848200020EF8D0108234B244C89
:10CC38001D68206880B5FCF70BF82846FCF708F853
:10CC4800206841798B0704D4036841F002015B69CD
:10CC580098471C4B4FF488521A854FF488421A851E
:10CC68002068FEF71CFBA0B1164E4FF48853B36141
:10CC7800134B1868FEF710FB0746FEF7BDFE08B118
:10CC880001F084FB28463946FEF70CFB4FF4885325
:10CC980033852846FEF703FB0028E1D0094ED4F877
:10CCA80000804FF48847B7612846FEF7F5FA014639
:10CCB8004046FEF7F7FA3785D2E700BFB01F0020DD
:10CCC800E01C0020001000482DE9F047054607F059
:10CCD80022FC314E0446D6F8088090B92F4802F05D
:10CCE800C9F82F4B53F8241049B10123A34013EA84
:10CCF800080F02D02B48FAF7ACF80134F1E72A48BC
:10CD080022E028462949224607F00EFC58B928484F
:10CD1800284C02F0AFF854F8041F0029EFD021483E
:10CD2800FAF797F8F7E72B782D2B03BF013504F1B5
:10CD3800FF344FF0010A4FF0000A4FF00009184B7A
:10CD480053F8297027B91C48BDE8F04702F092B89B
:10CD580028463946224607F0E7FBC8B9012000FA01
:10CD680009F0830501D51548EEE7BAF1000F03D0A5
:10CD7800FAF7C4F9124803E040EA0800B060114825
:10CD880002F078F839461048BDE8F047FAF761B87C
:10CD980009F10109D3E700BF4820002000860108F7
:10CDA800606C0108F68501084B8F0108DE850108D3
:10CDB8000A8601085C6C01080685010816860108C8
:10CDC800248601082D860108EE8D010810B5084853
:10CDD80002F050F8074B00241C715C63064B1C7072
:10CDE800FEF7E4FB02F0F8F9044B1C6010BD00BF2D
:10CDF80035860108E01C0020012C0020B01F00200F
:10CE080070B5064600240B4BE518AA8816420AD0CE
:10CE1800E1580948FAF71DF82846002101F0B7FF44
:10CE2800064802F027F8143440F694439C42EAD1AD
:10CE380070BD00BFE86F0108618601084B8F0108CB
:10CE4800F0B504788BB005460CB1002436E04A4BA7
:10CE580019680E2303FB041101F58C70B1F91D51FB
:10CE6800B1F91921B1F91B31009591F820510195BB
:10CE780091F82151029590F90700039001F59071FE
:10CE88003E4891F90210049121460134F9F7E1FF77
:10CE9800082CDCD16DE02D2B14D1072C1BDC284687
:10CEA80007F090FB0AAB661C03EB440424F8100C53
:10CEB80015F8013F303B092BFAD934462B78002B63
:10CEC800E9D104E0A3F13002092A09D8E5E7082CE2
:10CED800BDF8182009D00BB0BDE8F040FBF7BAB98F
:10CEE800202BF8D101352646E7E7072AF3D8BDF805
:10CEF8001A00214BA0F2EE2189B240F2DC55A9427A
:10CF08001B68E8D8BDF81C10A1F2EE24A4B2AC420C
:10CF1800E1D8BDF81E7004B23EB2A642DBDB0DB20A
:10CF2800AE42D8DCA542D6DBBDF92440642CD2D170
:10CF3800BDF8266034B2112CCDDCBDF82050B42DDC
:10CF4800C9D8BDF82240B42CC5D812B24FF00E0E85
:10CF58000EFB0233A3F81B116421A3F81901A3F8EF
:10CF68001D7183F8205183F8214183F81F1183F83C
:10CF780022610BB0F0BD00BF201000206B860108B5
:10CF8800F0B504468FB0204607F0C5FAC5B225BBF8
:10CF9800AC48AD4C01F06EFF94F8D61009B9AB4817
:10CFA80054E049B294F8D42094F8D530009194F81C
:10CFB800D710019194F9D810029194F9D9100391DE
:10CFC80094F8DA100491A24829460135F9F741FF8F
:10CFD800102D04F10704DFD1E1E720469D49052221
:10CFE80007F0A2FA0546B8B929469B48702207F00F
:10CFF8004EFA9A4B196828460E2303FB001301309A
:10D008000022082883F8232183F8242183F8252186
:10D0180083F82621F0D113E120469149042207F034
:10D0280083FA05462046002D4AD1202107F065FAEB
:10D03800002800F00581461C304607F06CFA2C46A3
:10D048000746884B53F824502DB987480FB0BDE8E0
:10D05800F040F9F7FEBE30462946FAB207F064FA06
:10D0680001340028EDD1784A02F1700116460023F8
:10D0780082F8DA3082F8D63082F8D53082F8D430A7
:10D0880007328A42F3D1794901EBC40191F8802231
:10D09800934210DAD1F88472C3EBC302B0183A4451
:10D0A80000F1D4011768C0F8D4709088888092790C
:10D0B8008A710133E7E729466D48F9F7CAFE90E01F
:10D0C8006C49072207F030FA05462046002D4AD160
:10D0D800202107F012FA064607F01DFAC4B274BB05
:10D0E8006548F9F7B6FE214664480134F9F7B1FE00
:10D0F8000E2CF8D15548F9F7ACFE002460482146BB
:10D10800F9F7A7FE0025554A5E4811680E2202FB72
:10D1180004120123D2F823215B49AB4013425B4B35
:10D1280005F1010508BF1946F9F793FE0E2DEAD15E
:10D1380046480134F9F78DFE082CDFD180E03046EF
:10D14800534907F043FA2C4600284CD0022C4FD004
:10D1580007F038FA06AB4E4943F82400002007F0E0
:10D1680035FA0134F0E74A4907F030FA002460B193
:10D17800082C38D007F026FA06AB454943F82400B6
:10D18800002007F023FA0134F1E7082C2BD1069B85
:10D198000F2B28D8DDF81CE0BEF1070F23D8089F15
:10D1A8000D2F20D8099E06F16402C82A1BD80A9DB3
:10D1B800FF2D18D80B98642815D80C99642912D813
:10D1C800884210DA0D9C032C0DD8324AC3EBC303F6
:10D1D800134483F804E05F719E71DD71187259720F
:10D1E8009C722D4CCFE60FB0BDE8F040FBF732B88B
:10D1F800069B072B20D807990D291DD80278722A7B
:10D208000DD06E2A18D1154A12680E2000FB032390
:10D2180001228A40D3F8231121EA020209E00F4AC9
:10D2280012680E2000FB032301228A40D3F8231141
:10D238000A43C3F8232101E0FBF70CF80D4CA2E6E2
:10D248000FB0F0BD93860108482000204B8F0108DD
:10D25800BE860108D68401081C2100202010002069
:10D2680001850108F86B010806850108386A01087C
:10D27800158501088B860108D0850108DA86010822
:10D28800078E0108DF860108CC9101088692010803
:10D29800E386010818210020E28101082DE9F743FF
:10D2A800047805468CB9324D95F89F12B5F89C2242
:10D2B80095F89E322F48009121460134F9F7C9FDAF
:10D2C800102C05F10405EFD14EE007F07BF90F288B
:10D2D800044636DC2846202107F00FF9264EE4B232
:10D2E800D6F83880451CA4000027284607F06AF9BC
:10D2F8005FFA87F9B9F1010F83B208D0B9F1020FCB
:10D308000BD0B3F5B47F24D2B26B13530AE0FF2BD2
:10D318001FD8B36B2344987004E0FF2B19D8B36B64
:10D328002344D87028462C2107F0E7F8054608B1B1
:10D33800013502E0B9F1020F0BD10137032FD4D127
:10D3480012E00E4800210F2203B0BDE8F043FAF7BF
:10D35800FEBE08EB04000021042207F098F803B091
:10D36800BDE8F043FAF776BF03B0BDE8F08300BF2D
:10D3780048200020E5860108E01C0020948401086C
:10D388002DE9F0412DED048BB3498AB0044607F02E
:10D3980087F8B249002820460CBF0126072607F067
:10D3A8007FF8AF490028204608BF022607F078F822
:10D3B800002808BF0426F10740F10681A948AA4CB5
:10D3C80001F058FD002001F05BFBA84801F052FD78
:10D3D800A74801F04FFD6279A64BA74803EB8203EB
:10D3E8002546D3F8BC11F9F734FDA448F9F731FD07
:10D3F8004FF00008274695ED058AB5EE408AF1EE14
:10D4080010FA04D19E48F9F724FD002570E09D48E4
:10D41800D5ED069A95ED079AD5ED088A4146F9F7B4
:10D4280018FDB5EEC08AF1EE10FA02D5202001F001
:10D4380019FDB0EE480A06A8F9F7A0FB0146924884
:10D44800F9F707FDF5EEC09AF1EE10FA02D52020A3
:10D4580001F008FDB0EE690A06A8F9F78FFB01464E
:10D468008948F9F7F6FCB5EEC09AF1EE10FA02D544
:10D47800202001F0F7FCB0EE490A06A8F9F77EFB78
:10D4880001468148F9F7E5FCF5EEC08AF1EE10FA9D
:10D4980002D5202001F0E6FCB0EE680A06A8F9F7EC
:10D4A8006DFB08F1010801467848F9F7D2FCB8F19C
:10D4B8000C0F05F110059ED1A4E749B294F8D420C9
:10D4C80094F8D530009194F8D710019194F9D810B8
:10D4D800029194F9D910039194F8DA1004916C48E8
:10D4E80029460135F9F7B5FC102D04F1070403D0DE
:10D4F80094F8D6100029E0D100254FF00E0808FB5B
:10D5080005F80024634AD26B42440123D2F80A206A
:10D51800A340134240F0948001340E2CF2D101351F
:10D52800082DEAD15C485D4C01F0A4FCD7F80880CE
:10D5380054F8041F19B15A48F9F78BFCF8E70D465F
:10D54800584B53F8254054B10123AB4013EA080F58
:10D5580003D055482146F9F77CFC0135F0E75348DC
:10D5680001F088FC21467B180AAA93F88A311344F3
:10D578004F4A8A5C03F8102C01310829F3D10023A3
:10D5880006A94C488DF82030F9F763FC4A4801F0A9
:10D5980071FC4A48FBF794F9494801F06BFC47488D
:10D5A800FAF75EFE474801F065FC4448FFF776FE4F
:10D5B8004548F9F74EFC4020FFF722FC434801F0AC
:10D5C80059FC3E48FBF722FAB20726D5404801F03D
:10D5D80051FC404801F04EFC384801F091FA3E48B1
:10D5E80001F048FC3548FAF7BFFD3C4801F042FC21
:10D5F8003248FBF7B7F83A48F9F72BFC2F48FAF707
:10D608003BFF384801F036FC2C48FFF719FC2E4840
:10D61800F9F71FFC8020FFF7F3FB730716D5324894
:10D6280001F028FC314801F025FC244801F042FAB9
:10D638002548F9F70EFC4FF48070FFF7E1FB05E091
:10D64800294622462A48F9F704FC65E70AB0BDECEA
:10D65800048BBDE8F08100BFF9860108348B01080E
:10D668000087010806870108482000201487010860
:10D6780026870108386A0108328701083D870108B2
:10D688004A87010857870108CF850108EF8D0108EF
:10D698005F870108E01C00207E8701085C6C010898
:10D6A8008E870108606C01089C870108A98701081A
:10D6B80016830108B5870108BE870108E2810108C1
:10D6C800CD870108D98701084B8F0108E787010832
:10D6D800F487010807880108158801081F880108D0
:10D6E8002E8801083C8801084888010859880108E3
:10D6F8006B880108054B98420CBF054A054A1388F8
:10D7080001339BB213800020704700BF00540040D3
:10D71800E00F0020E20F0020084A13689B050BD594
:10D72800074B00211970074908684FF6FE7303403C
:10D738000B604FF400735360704700BF0000024055
:10D74800FC2B0020300002402DE9F047664D2B6885
:10D7580066490A78581C02F0FF068E460AB103464D
:10D76800F6E72B60687BAB6895F80C80AA7B374698
:10D7780039B2202900F09B80DFF880C10CEB8103CF
:10D788003CF82110DC789B78C3F1FF039BB2002B97
:10D7980065D0C3F1FF0363434FF03C0C1B12B1FB90
:10D7A800FCF9B9F1050F5DD8DFE809F0030B1A2978
:10D7B8003A4AE01ADAB24143B1FBFCF01044C0B275
:10D7C80051E0B1FBFCF00CFB101189B2DAB2C1F1E7
:10D7D8003C01E31A4B432046B3FBFCFC94442CE089
:10D7E800B1FBFCF00CFB10115FFA83F8E21A89B266
:10D7F8004A43B2FBFCF24244D2B2204632E0B1FBCB
:10D80800FCF90CFB191189B25FFA83F8E01AC1F12F
:10D818003C014843B0FBFCF04044C0B2224621E042
:10D82800B1FBFCF80CFB1811D8B289B2E31A01FB62
:10D8380003F2B2FBFCFC224684445FFA8CF412E04B
:10D84800B1FBFCF80CFB181189B2D8B2C1F13C014C
:10D85800E31A4B43B3FBFCF20244D2B203E0224684
:10D86800204600E044464FEA042C4CEA004C4CEABF
:10D87800020C172306F117014FF0010808FA03F804
:10D88800C91A18EA0C0F89B2DFF8748014BF4FF078
:10D8980011094FF0090913F1FF3308F80190E9D293
:10D8A80018360137B6B2BFB2114BA04660E7AA736B
:10D8B800AB60104AE98001238EF800300E4985F8E4
:10D8C8000C8040F22A336873AE80536000234B62A9
:10D8D8000B889BB243F001030B80136843F00103EC
:10D8E8001360BDE8F08700BF201D0020FC2B00203E
:10D8F8002C1D002030000240004401407A0D002019
:10D908003103002073B506460D46002401232A88FA
:10D91800A34013421AD0AA78009302F003038DF8AB
:10D928000430EB78022B03D0032B0CBF0323012315
:10D938008DF805303046C2F301136946C2F38102FF
:10D948008DF806308DF80720F8F7EEFE0134102C1C
:10D95800DCD102B070BD2DE9F04F734EF57B074660
:10D968000C4687B011469A4600686B1C91462246C1
:10D978004FF0020BF37300F041FB3B897868ADF878
:10D98800043001A98DF806B08DF807B0FFF7BAFF8B
:10D998000023ADF80A30ADF81230ADF81630702318
:10D9A8000193BA7A3C68CDF80CA0012306F110085F
:10D9B8002D01ADF808304FF48073A844ADF810B0CD
:10D9C800ADF814300C2A7ED8DFE802F0077D7D7DA3
:10D9D8000F7D7D7D387D7D7D5E00204601A9F8F7AD
:10D9E800EFFCA36943F0080326E0236A4F4823F0BD
:10D9F80010032362236A6168A26922F0807222F40C
:10DA0800E642844242F4E04206D000F500608442D7
:10DA180002D043F0300307E023F0E00321F4406133
:10DA280043F0300341F480616160A261C4F838A01A
:10DA38002362A36943F40063A36144E0236A3B487B
:10DA480023F480732362226A6168E369844223F0C5
:10DA5800730343F0700306D000F50060844202D0DF
:10DA680042F4407207E022F4606221F4405142F42B
:10DA7800407241F480516160E361C4F83CA02262C5
:10DA8800E36943F008031DE0236A284823F4805320
:10DA98002362226A6168E369844223F4E64343F41B
:10DAA800E04342F4405203D000F50060844201D1C3
:10DAB80041F480416160E361C4F840A02262E369F7
:10DAC80043F40063E3613A7B3B681AB15A6C42F451
:10DAD80000425A641A8892B242F001021A80BA7A55
:10DAE8000C2A18D8DFE802F0071717170B171717B3
:10DAF8000F1717171300721903F134010AE072198E
:10DB080003F1380106E0721903F13C0102E07219D1
:10DB180003F14001116135444046A5F818906B6146
:10DB280007B0BDE8F08F00BF201D0020002C014089
:10DB3800F8B53A4E3A4C4000C7B24FF42045306829
:10DB4800C4F8D050D0F818E01EF4004F05D0AE4607
:10DB5800013DBEF1000FF5D116E0D0F804E0314DDB
:10DB68000EEA050545F490353D4345604FF42045E0
:10DB7800C4F8D050D0F818E01EF0020F2DD1AE46F0
:10DB8800013DBEF1000FF5D1C4F8D0501FE0294681
:10DB9800013D0029F8D081694906F8D5C4F8D0506C
:10DBA80020494568294041F0007141F4105141EA8B
:10DBB8000241394341604FF42041A2B13068856980
:10DBC8006D071ED411F1FF31F9D2C4F8D010FFF758
:10DBD80091FD003018BF0120F8BD4FF42045816247
:10DBE800C4F8D050D7E73068C4F8D0100B46826923
:10DBF80092060CD41A46013B002AF8D1C4F8D0305A
:10DC0800E5E7416A03F8011B013AD2B2D3E7C4F849
:10DC1800D0302023C3610120F8BD00BFDC0F0020F5
:10DC2800201D0020009800FC400070B5C5B23248A5
:10DC3800324B00684FF42044C3F8D040866936045C
:10DC480004D52646013C002EF8D113E046682C4C3A
:10DC5800344044F0807444F490342C4344604FF4CE
:10DC68002044C3F8D0408669B60729D42646013C2B
:10DC7800002EF8D1C3F8D0401CE02146013C002911
:10DC8800F8D081690E06F8D544681D49214041F055
:10DC9800007141F48031294341604FF42041C3F8B9
:10DCA800D0108469A40711D40C460139002CF8D18E
:10DCB800C3F8D010FFF71EFD003018BF012070BD5B
:10DCC8004FF420448162C3F8D040DAE782624FF40F
:10DCD8002042C3F8D0208169890606D41146013A4A
:10DCE8000029F8D1C3F8D020E4E7C3F8D0202023D6
:10DCF800C361012070BD00BFDC0F0020201D002083
:10DD0800009800FC026D036B70B50446D5699BB999
:10DD1800A90611D5C36A1BB1908C80B298470BE055
:10DD2800E169928C40694E1CD2B2E6614254E169C5
:10DD3800E268914228BFE361616BA1B92A0612D556
:10DD4800636AA26A9A42236D09D0501CA669A06230
:10DD5800B25C1A852369984205D3A16203E01A6868
:10DD680022F080021A602B0742BF236D08221A6234
:10DD780070BD026BC168034610B5406942B11A6CA8
:10DD88008C1A013A005D08BF0A46C0B21A6410BD79
:10DD98001A6A805C01328A4228BF0022C0B21A6225
:10DDA80010BD436B13B190F844007047836A406A12
:10DDB8001B1A584258417047036B13B15B68016CDA
:10DDC80001E0C369016A8B423CBFC2689B18581ABC
:10DDD800C0B27047836A8169426B1944D160416A55
:10DDE80099429DBF0169CB1A5360CB1A96BF002395
:10DDF800536083624FF0000380F84430136888BF93
:10DE0800816243F0010313607047436A8269D15409
:10DE1800436A02690133934228BF00234362436B7C
:10DE28001BB11B68DB0705D4D4E7026D136843F008
:10DE3800800313607047274A73B55369264C43F42F
:10DE48000013536103236946082501268DF8053020
:10DE5800204600238DF806308DF8073000958DF8A0
:10DE68000460F8F761FC1D4AA561138823F040039C
:10DE78001B041B0C1380138823F038031B041B0C92
:10DE88002B43138013889BB243F040031380242054
:10DE9800258501F07BFD802001F078FDA5616420D7
:10DEA800FCF7FCFF2585202001F070FDAF2001F074
:10DEB8006DFD3046A561FCF7F1FF2585232001F0B3
:10DEC80065FD602001F062FDA5616420FCF7F1FFAB
:10DED80002B070BD00100240001000480030014040
:10DEE8002DE9F0410369C76805460E461F40002F1B
:10DEF80035D0B7FA87F24FF00043D340DB432B61AC
:10DF08001F40A2F11B03042BF1D8DFE803F0221F06
:10DF18001C190300746A24B1013C0023A4B2736283
:10DF280001E0EC6AA4B2D6F82080B8F1000FDED088
:10DF3800D8F80030404621469847D8F80480F4E7DE
:10DF48003068696B07E07068A96B04E0B068E96B3A
:10DF580001E0F068296C036889B29847C7E7BDE813
:10DF6800F0814171FEF7B4BA8160FEF7B1BA014899
:10DF78000149B5E70048014054160020014802490C
:10DF8800AEE700BF003401400416002001480249F2
:10DF9800A6E700BF003401400416002001480249EA
:10DFA8009EE700BF00080040DC1500200148024938
:10DFB80096E700BF00040040B41500204FF08040F1
:10DFC80000498DE78C15002010B5054C0548214601
:10DFD800FFF786FF04F1C8010348BDE810407FE75A
:10DFE80064150020002C014000440140014802490A
:10DFF80076E700BF002C014064150020224B10B5C5
:10E00800224C5A43224BB3FBF2F203880139013AFE
:10E01800A04289B292B29BB20ED004F50064A0422D
:10E028000AD0B0F1804F07D0A4F59834A04203D0AD
:10E0380004F58064A04202D123F070039BB2154C12
:10E04800A04206D004F58064A0421CBF23F44073AC
:10E058009BB203800D4BC162984202850FD003F535
:10E06800006398420BD003F54063984207D003F54C
:10E078008063984203D003F58063984201D100235E
:10E0880003860123436110BD40420F00002C01406C
:10E0980000A24A0400100040134B800A984220D086
:10E0A8000AD84A3B984212D00133984211D0B0F5B1
:10E0B800801F14D1012070470C4B98420BD00133BC
:10E0C80098420AD0053B984209D1042070470220A3
:10E0D8007047032070470520704706207047FE20D0
:10E0E80070470020704700BF4B001000510010001F
:10E0F800F8B50468064620460F461546FFF7CCFFDC
:10E1080006284BD8B27A910847B902238B40D4F835
:10E118000CE0DB439BB203EA0E03E3600A23204AC8
:10E1280003FB001342F82370043342F823501546CA
:10E138003FB1B17AE268890802238B409BB213434E
:10E14800E360282202FB00522032EFF312865023AC
:10E1580083F3128803B203EB8303DB0003F10C01A2
:10E168001C3329442B4451F8047F17B117600A68FF
:10E1780004329942F7D100231360F3B283F3118874
:10E18800282303FB0050036A1BB1E36843F0010333
:10E1980003E0E2684FF6FE731340E360F8BD00BF8A
:10E1A800641500200048ADE5201E00200048A9E5C0
:10E1B800741E00200D4B0E484FF400525A600D4A51
:10E1C80011684FF6FE730B401360D0F88820116871
:10E1D8004FF6FE730B401360826FC36F9A4201D0F3
:10E1E8005430F7E5012380F898307047000002406A
:10E1F800201E00204400024010B54B88DC0641BFB9
:10E208002F4B14791B6853F8244044BF2D4B43F817
:10E2180020404B889B0641BF294B54791B6853F813
:10E22800244044BF274B43F820404B881C070ED599
:10E23800254B0C781B78B3EB141FA1BF204BD47867
:10E248001B6853F82440A4BF1E4B43F820404B885A
:10E258009B070ED51D4B0C781B78B3EB141FDFBF43
:10E26800174B54781B6853F82440DCBF154B43F810
:10E2780020404B88DC070FD5154C0B78247803F029
:10E288000F03A342DFBF0E4B14781B6853F82440DA
:10E29800DCBF0C4B43F820404B885B070FD50B784D
:10E2A8000C49097803F00F038B42A1BF044B927805
:10E2B8001B6853F82220A4BF024B43F8202010BD4E
:10E2C800181D00207A0D00209714002095140020B6
:10E2D8009414002096140020254A26482649002335
:10E2E800F0B5156803700B701C461A462E1976880F
:10E2F8004EB92F5D3FB9037000230A704B70077841
:10E308001C461A460CE0360548BF013204F10404E5
:10E3180003F1010348BFD2B2802CDBB2E6D1EAE7B1
:10E32800E0B2B8420CD215F8240006099E4200F06B
:10E338000F00A8BF731C9042A8BF421C0134EFE72E
:10E348008A704B70C2F3470102F001020A444C1E66
:10E358000A490B480A70C3F3470203F00103134448
:10E3680004700849501E084A08701370F0BD00BFB9
:10E37800801300208C140020C81E00209614002052
:10E388009414002097140020951400202DE9F04FD4
:10E39800C24BDA682DED028B1A61C14A1168D96047
:10E3A800C0490B6843F020030B60BF4B1978012963
:10E3B80090460CBF002201221A70BC4B1A789107B4
:10E3C80089B040F13D83BA490978042940F238837D
:10E3D800B849097801F0040101F0FF0011B922F0F1
:10E3E80001021A701B78DB0702D408B1FDF732FF6F
:10E3F800B149CA78531C052293FBF2F202EB820260
:10E408009A1AAE4BCA701B78039392000023AC4C47
:10E41800DFF8CCC2DFF8D8925CF8231091FBF9F54D
:10E4280004F1080004F1100640F82350A54844F808
:10E43800231000FB051142F2107091FBF0F080B23E
:10E4480026F813004FF0140E04F1140604F13C0AE8
:10E458000EFB036E5AF823605EF802704EF8021045
:10E46800F61B314444344AF82310052691FBF6F193
:10E4780009FB051144F82310039C012C4FEA830B78
:10E48800E24605D10238B0F5797F98BF4BF80C10F9
:10E498000BB90123BBE7884CD8F80030226D9FEDFB
:10E4A8008A7A8A4E8A4D9B1A07EE903AF8EE677A76
:10E4B800D8F800302365C7EE877A7C4B1B78B7EE17
:10E4C800008AF4EEC87AF1EE10FA58BFF0EE487AF6
:10E4D80013F00103C4ED157A12D005AA00927D4B02
:10E4E80006AA01920CCB9AE80300FDF7B1FD64215E
:10E4F800059A069BB2FBF1F293FBF1F3328000E040
:10E5080033802B8094F858306B48002B3BD0D0EDEB
:10E51800157AC26DDAF80030C8EE276A9B1A026EC7
:10E52800022507EE103AB8EEC77ADAF8043027EE7B
:10E53800267A9B1AFDEEC77AB0F9662017EE901A74
:10E5480007EE903A644BB8EEE77AD3ED007A67EEBF
:10E55800277A67EEA67AFDEEE77A17EE903A02FA86
:10E5680083F3B0F9642093FBF5F302FA81F29BB2CE
:10E5780092FBF5F292B2A0F86A30A0F86820A0F8F1
:10E588006630A0F86420012384F85830534BDAF839
:10E5980004101B88DAF80000474D514E216603F03D
:10E5A8003003E065002B00F04B8205F17403009303
:10E5B80005F178030193EA6E2B6FFDF749FD726848
:10E5C8002B6F9B1A07EE903A434B326893ED007A13
:10E5D800EB6EF8EEE77A9B1AEB67384B67EE877AB3
:10E5E8001B78FDEEE77A012BC5ED207A03D0022BCC
:10E5F80000F0DF8024E2D5ED287A3A4BD5ED215A98
:10E6080095ED255A95ED156A95ED264AD5ED274ADB
:10E6180035491D68B1EE677ABDEEC77AFDEEE77A37
:10E6280017EE10EA17EE90CA0020304A91ED007AF2
:10E6380052F8207007EE907AF8EEE77AA2F1140308
:10E6480067EEA57A33F81060FDEEE77A283217EE08
:10E65800903A9B1B9BB222F810301BB207EE903AFF
:10E66800F8EEE77A3B4467EE857A4400FDEEE77AF8
:10E67800CDED037A07EE903AF8EEE77ABDF80C8014
:10E6880067EE847AA7EE867AFDEEC77A17EE902AAF
:10E69800724531DB6245A8BF62462EE0AC06002019
:10E6A8000C200020D010002046100020D41000209C
:10E6B800DA100020FD2B0020C81E00200C0F0020BF
:10E6C800CC1E0020806967FF00007A444E110020AC
:10E6D8005011002048100020080100209811002047
:10E6E800DC100020100F0020400F0020441F0020E5
:10E6F80080969800DB0FC940724607EE902AF8EE24
:10E70800E77A5FED046AC1ED007AFDEEE77A31360B
:10E7180017EE903A43449AB2AB78D1ED027A07EEFD
:10E72800103AB8EE477A4B684F6027EE267AFB1A04
:10E7380088EE077AB6B2622E06EE903AF8EEE66AEE
:10E7480037EE067AC6EE866A86EE077A76EEE76ACE
:10E75800E7EE267AC1ED047AC1ED027A0FD964EEAC
:10E76800A77ABA4EFDEEE77A17EE903AB3F5FA6F4C
:10E77800A8BF4FF4FA63B342B8BF334600E00023A2
:10E7880013441BB240F6B8329342A8BF1346B04AAE
:10E798009342B8BF1346AF4AA352AF4A142303FBB0
:10E7A800002351F8142B1A60002840F049810120F9
:10E7B8003BE7AA4BD5F874801F68D4F878903E8957
:10E7C800DFEDA78A4FEA58039E4228BF1E46B5F8D8
:10E7D800A8301AB29642C3BFD5ED157A9FEDA17A3B
:10E7E80067EE877AB6B2C1BFFDEEE77A17EE906A98
:10E7F800F618B6B2C8BFA5F8A860D4F8AC50C5EBF7
:10E8080009052846FDF768FC0028D8BF404241F2B8
:10E8180093129042CCBF0020012088B307EE905A93
:10E82800B8EEE70A20EE280AF8F741FB07EE908ACF
:10E83800F8EE677A40F6B83320EE270AFDEEC07A84
:10E84800CDED037ABDF80C20A4F8B02012B29A429C
:10E85800A8BF1A467E4B9A42ACBF09EB02034B4451
:10E8680048F6A042934203DDA3F50C43A03B04E025
:10E87800002BBCBF03F50C43A033C4F8B43001E04F
:10E88800C4F8B490D4F8B450C5F50C53283307EE47
:10E89800903AF8EEE77A67EEA88AB0EE680AF8F7D9
:10E8A80069FB8DED070AB0EE680AF8F700FBD4EDB6
:10E8B800317AD4ED2E4AD4ED155A94ED2F4A94EDC1
:10E8C800305A65498DED060AB1EE677ABDEEC77A12
:10E8D800FDEEE77A0DF1180E17EE10AA17EE90BAB2
:10E8E8000020614AFEEC016A32F91030DFF88C91A1
:10E8F80007EE903A07EE106AF8EEE77AB8EEC77AB4
:10E908003C32D6EE877A4FEA400CFDEEE77ACDED41
:10E91800037ABDF90C30B3F57A7FA8BF4FF47A7348
:10E928004B45B8BF4B461FFA83F922F810900FFAEF
:10E9380089F207EE902AF8EEE77A27EEA47ABDEE80
:10E94800C77A8DED037A27EE847AD1ED007ABDF887
:10E958000C90E7EE257AFDEEE77A17EE902A5245FD
:10E9680003DB5A45A8BF5A4600E0524607EE902AF4
:10E97800F8EEE77A9FED3D6AC1ED007ABA7891ED3D
:10E98800027A06EE902AF8EE666A4A684B6066EEEE
:10E99800866A9A1AC8EE266A143106EE102AB8EE6C
:10E9A800C66A76EEA56A86EE256AC5EEA66A36EED2
:10E9B800476AA6EE867A01ED017A01ED037A25EE23
:10E9C800077ABDEEC77A17EE103ABDEEE77A4B44E8
:10E9D80017EE102A13441BB240F6B8329342A8BF70
:10E9E80013461B4A9342B8BF13461A4A2CF8023002
:10E9F8001F4A142303FB0023C3ED007A08B9012042
:10EA08006FE73B7923B1642395FBF3F5194B1D8020
:10EA18003B8898450DD9D4F8AC30A06FC01AFDF7E3
:10EA28005BFB80EAE072A2EBE07242F210739A425A
:10EA380006DD114B01221A700E4BB4F8C8201A805B
:10EA480009B0BDEC028BBDE8F08F00BF30F8FFFFC6
:10EA580048F4FFFF940F0020680F0020100F0020DB
:10EA6800D30237390000C842301F0020DB0FC940ED
:10EA7800400F0020080F00200C0F002018FCFFFF9B
:10EA880007B5064B0093064B01930649064A074B08
:10EA98000748F8F7DEF903B05DF804FBFC7E0108CF
:10EAA800D17E0108868D0108978D0108F07E010846
:10EAB800668D010808B5037833B90C4B0C481978F2
:10EAC800BDE80840F8F7C5B905F07CFD02280CD868
:10EAD800064B1870074B0C2202FB0030064B063021
:10EAE8001860F8F7D3FB0548E5E708BD941F002038
:10EAF8009E8D0108E827002040100020E2810108CF
:10EB080008B503783BB90B4B0B4893F8A417BDE83D
:10EB18000840F8F79EB905F055FD022808D8054BBE
:10EB280083F8A407F8F71CFBF8F7D4FB0348E8E7D9
:10EB380008BD00BF48200020A28D0108E28101081D
:10EB480038B5037803BB214B1B6801330F2B07D85B
:10EB58001F490C2202FB03121C4695682DBB00E0DE
:10EB68001C4601340F2C01DD002400E005D81849AB
:10EB78000C2202FB04129568BDB99C42F1D11548DC
:10EB8800BDE83840F8F765B905F01CFD0F280446C4
:10EB980005D80F4A0C2303FB00239D682DB9214695
:10EBA8000D48BDE83840F8F754B9084B1C60FCF72D
:10EBB800DDFA21462A460948F8F74BF90C235C434D
:10EBC800034B185DBDE83840FCF7E8BA0C0100209B
:10EBD800486E0108AF8D0108C58D0108DD8D01085B
:10EBE80073B5037813B9F9F735FB3DE01F4901AA5E
:10EBF80005F049FD002401462646254699B134B161
:10EC0800012C08D1084605F0DDFC064603E008465D
:10EC180005F0D8FC05461549002001AA05F033FD8A
:10EC280001340146EAE70B2D02D911480C220BE00A
:10EC3800022C10D1A6F57A73B3F57A7F07D90D485F
:10EC48004FF47A714FF4FA62F9F781FA0CE00A4B43
:10EC580003EB45035E80084B084803EB4503294650
:10EC6800B3F90220F8F7F5F802B070BDE3860108A1
:10EC780094840108568A0108941F0020F48D010825
:10EC880038B50D4C23688342054606D1F9F7EBFFEA
:10EC9800204600214C2205F0FAFBE36CAB4209D177
:10ECA8002846F9F7E0FF054800214C22BDE8384026
:10ECB80005F0EDBB38BD00BFAC110020F8110020F5
:10ECC800034B1A68D379591C1344D171187A7047C9
:10ECD8007811002010B5FFF7F3FF84B2FFF7F0FFBB
:10ECE80004EB002080B210BD10B5FFF7F3FF044617
:10ECF800FFF7F0FF04EB004010BD064B10B50446CB
:10ED080021461868FCF7CEFA034B1B6898796040D7
:10ED1800987110BD7C11002078110020014B1B68F0
:10ED28009879EAE77811002038B5044624200D4682
:10ED3800FFF7E3FF4D20FFF7E0FF002C084C14BF5E
:10ED480021203E20FFF7D9FF2368002228469A7128
:10ED5800FFF7D3FF236893F84900BDE83840CCE7B4
:10ED68007811002001460020DEE710B50446C0B245
:10ED7800FFF7C3FF200ABDE81040BEE710B5044600
:10ED880080B2FFF7F2FF200CBDE81040EDE737B581
:10ED980082888368044610060D4641BF2B4991F8C6
:10EDA800A4174FF4CC7000FB0133D10544BF2849A8
:10EDB800097802F03F0244BF01EB410103EB8103F4
:10EDC800042A12D006D8012A0DD0022A32D193F98A
:10EDD800001030E0102A0AD0202A0AD0082A29D1A7
:10EDE800B3F9001027E0197825E0198823E019689D
:10EDF80021E093ED000A6846F7F7C0FE0146154882
:10EE0800F8F727F805B3D4ED037A6846B8EEE70AB1
:10EE1800F7F7B4FE01461048F8F71BF894ED040A1A
:10EE28006846B8EEC00AF7F7A9FE01460A48F8F79F
:10EE380010F809E000210948F8F70BF825B108484F
:10EE4800E1682269F8F705F803B030BD48200020D2
:10EE5800941F0020CF850108C8850108078E010886
:10EE6800038E0108024B0146D869FCF71BBA00BFA4
:10EE7800941F002010B5441E14F8011F21B1034B44
:10EE8800D869FCF70FFAF7E710BD00BF941F002000
:10EE980010B503781BB90A48BDE81040EAE705F049
:10EEA80091FB0446062899BF2146064806480621D4
:10EEB800F7F7CFFF601E40B2BDE81040F9F73CBE3F
:10EEC8000A8E0108518E01087D8E0108F7B52B497D
:10EED8002B4B08782B4D1C682B4B05EB80001A88B0
:10EEE8002A4BD0F8C0101B78294800914FF47A714A
:10EEF800B4FBF1F1F7F7ADFF26484821F7F7A9FF72
:10EF0800254B1F680026F3B205EB8302D2F8D01018
:10EF1800E9B101249C403C4217D0220715D01F4A72
:10EF2800D25C0B2000FB0323164A1D4802EB830327
:10EF3800D3F8F020F7F78DFF022C06D1194B93F880
:10EF4800281011B11848F7F784FF0136DBE7174896
:10EF5800FFF790FF164B17481A68174B9A420CBFD9
:10EF6800164B174B1A88174B198892B24FF4FA634D
:10EF780003B0BDE8F040F7F76CBF00BF20110020D8
:10EF88000C200020486E0108C0100020100100204D
:10EF9800A88E0108EB8E0108D0100020180100206F
:10EFA800FB8E0108941F0020038F01084B8F010876
:10EFB800DC0F0020078F010800540040E00F0020FC
:10EFC800E20F0020D80F00202DE9F04100248046F0
:10EFD80025460F4EA7594146384605F0DBFA58B189
:10EFE80039460C48F7F735FF30190021FFF7CFFEF7
:10EFF8000948FFF73FFF0135143440F694439C421B
:10F00800E7D11DB90548BDE8F04133E7BDE8F08117
:10F01800E86F0108658601084B8F0108068501081D
:10F028002DE9F04F2DED028B83B0054605F073FAFC
:10F03800064620B1012818D12B782A2B15D15C4817
:10F04800FFF718FF00245B4D5B486159F7F701FF94
:10F0580028193146FFF79BFE5848FFF70BFF143479
:10F0680040F694439C42EED19CE028463D2105F0B1
:10F0780044FA002800F08F800346994613F8012DC2
:10F08800202AFAD0441C204605F09CFA80462046E7
:10F09800F7F7EAFCC5EB0909B0EE408A0026DFF86D
:10F0A80034A1142202FB06F40AF5D07B54F80B7045
:10F0B800384605F030FA03461A4628463946019381
:10F0C80005F032FA019B00285BD15FFA89F29A4277
:10F0D80057D10AEB0402D2ED6B7AF8EEE77A0BEB24
:10F0E8000405B4EEE78AF1EE10FA48DBD2ED6C7A4B
:10F0F800F8EEE77AB4EEE78AF1EE10FA3FD8B2F804
:10F10800A431D2F8A82113F0200F08BF08EE108A06
:10F118001C0641BF2A4991F8A4174FF4CC7404FB8C
:10F128000122D90544BF2749097803F03F0344BFAA
:10F1380001EB410102EB8102042B18EE100A0BD0FF
:10F1480004D8013B012B0ED810700CE0102B05D011
:10F15800202B06D0082B06D1108004E082ED008A0F
:10F1680001E082ED008A39461748F7F772FE284613
:10F17800002103B0BDEC028BBDE8F04F07E6134851
:10F1880003E00136A12E8AD1114803B0BDEC028BF1
:10F19800BDE8F04F6EE6284603B0BDEC028BBDE833
:10F1A800F04F11E703B0BDEC028BBDE8F08F00BF54
:10F1B800398F0108E86F0108658601084B8F01083F
:10F1C80048200020941F00204E8F0108598F010805
:10F1D80006850108486E010808B50748FFF74AFE8A
:10F1E800064BD869F9F734FDFCF7BCF9F7F78EFF41
:10F1F800034B044ADA6008BD798F0108941F002088
:10F2080000ED00E00400FA0508B50548FFF732FEF6
:10F2180000F036F8F7F7A4FFBDE80840DCE700BFC8
:10F22800858F010808B50448FFF724FEF7F798FF13
:10F23800BDE80840D0E700BF9B8F01080E4B1A7845
:10F24800692A16D15A88B2F5FA6F12D11A79BE2AEC
:10F258000FD193F8CD27EF2A4FF000000BD113F808
:10F26800012B5040054A9342F9D1B0FA80F0400989
:10F27800704700207047704700F80308D0FF030864
:10F288002DE9F04FEF4C00214FF4FA6285B020468B
:10F2980005F0FDF8EC4B04F537721A60EB4B0022D1
:10F2A8001A70EB4B04F2A6711960692323700323CB
:10F2B80063714FF48073A3604FF41673A4F866313A
:10F2C800FA23A4F86831BC23A4F864314FF4FA7324
:10F2D8002021A4F86E31012384F8623184F86A1180
:10F2E80084F87E316E2184F88631052384F87C11F8
:10F2F80084F81B320A2140F2DC5384F87D11A4F80B
:10F3080098312B2140F24C4384F87F11A4F89A31AC
:10F31800212140F26C7384F88011A4F89C312321D8
:10F3280040F2753384F88111A4F89E314FF4C87106
:10F3380040F64303A4F8A031A4F882112346991893
:10F34800023200254FF01E09242ABE4C81F8A25132
:10F3580081F8A391F3D14FF4FA6340F27E4040F272
:10F368007E57DFF8E4B2A4F8C831A4F8CC31A4F889
:10F37800D031A4F8D431A4F84401052340F23A70FE
:10F38800A4F84C7140F2EA5701264FF47A78C82263
:10F3980019214FF0320A84F8DE31A4F846014FF4FF
:10F3A800C87340F2DC50A4F84E7140F2B457A4F888
:10F3B800E221039284F8959184F8DD6184F8DF11E5
:10F3C800019184F8E06184F8E16184F8E461A4F8CB
:10F3D800E63184F8EA61A4F84A010290A4F8507171
:10F3E800A4F8543184F8ED61A4F8C681A4F8CA8160
:10F3F800A4F8CE81A4F8D281A4F84881A4F852A137
:10F40800A4F856A1F6F7E6FCDBF8003026744FF0B6
:10F41800170E83F815E083F816E04FF0550EE673E3
:10F42800A573A58183F803E04FF00F0E83F805E07C
:10F438000199D9714FF0220E83F806E021214FF08F
:10F448000E0E83F80B9083F80C9083F810E0597433
:10F458004FF0350E53214FF0640928274FF02D0C3B
:10F4680083F81AE0D9764FF05A0E0A2183F81C90D7
:10F478004FF0780983F80DC083F808E0997483F891
:10F488000A901D705F709F70DD7583F804A09D73EE
:10F498001D76DD735D765F7283F814C04FF4FA7CD5
:10F4A800A3F84EC0DFF8C0C1C3F838C0C3F83CC0E9
:10F4B800DFF8B8C1C3F828C04FF07E5CC3F834C089
:10F4C800F7EE087ADFF8A891DFF8A8C1C3ED087A4B
:10F4D800C3F82C90C3ED097AC3F83090C3F848C03C
:10F4E800F1EE047A02989E774FF04B0C4FF000092A
:10F4F80083F8501083F8525083F85170C3F8409045
:10F50800C3ED117A83F84CC084F8A6E7A4F8B007D5
:10F518004FF0410E042084F8A7E784F8A8A784F8E0
:10F52800A95784F8AD5784F8AE5784F8AA5784F8D9
:10F53800AB5784F8AC5783F85C0015200191A3F809
:10F548005850A3F85A50A3F85650C3ED187A83F8C8
:10F5580068004048D866404818674048586783F8AC
:10F5680078603F4883F8647083F86570F6F778FC34
:10F57800DBF800300199039A83F814614FF448705E
:10F5880083F8115183F8125183F8137183F81851D5
:10F59800A3F816015E4684F8D81184F8D921A4F896
:10F5A800DA8119460E2202FB05326FF0170082F845
:10F5B8001901032082F81A016FF02F0082F81B014D
:10F5C800072082F81C016FF0230082F81D01052036
:10F5D80082F81E0101355A2081F8200181F82101A5
:10F5E8006422FF20082D81F81F2181F8220101F1F2
:10F5F8000E01D7D1002183F88911C821A3F88A11F7
:10F60800142183F88C11A3F890211E214FF49672CF
:10F6180083F88D11A3F8922101212822A3F89421BF
:10F6280083F88E11074B03F1C0021F46C3F81490EC
:10F6380010339342FAD10B480021402204F027FFEF
:10F648001AE000BF4820002020100020941F00204E
:10F65800401000209A99193FF6287C3F3D0A773FD1
:10F668008F990108E42200208FC2F53C0000204059
:10F67800CDCCCC3E000040400023264D264C5959A5
:10F68800FA1804330868C2F89C02382BF5D104F53F
:10F6980007700021802204F0FAFE05F1380170227B
:10F6A80004F5077004F0E8FEFEF716FE366800233E
:10F6B8000125314604F274404FF4CC7284F8CC37FB
:10F6C80084F8CA5784F8CB5704F0D6FE04F20C60CD
:10F6D80031464FF4CC7204F0CFFE104B1B681A6809
:10F6E800C4F8B2275A68C4F8B6279A68C4F8BA2783
:10F6F8001A68C4F8BE275A68C4F8C2279A68C4F8BA
:10F70800C627022384F8C85484F8603605B0BDE8DB
:10F71800F08F00BFDC7C010848200020401000204A
:10F728001549D1F8883043F47003C1F88830134B79
:10F738001A6842F001021A605868114A02405A6079
:10F748001A6822F0847222F480321A601A6822F44D
:10F7580080221A605A6822F4FE025A60DA6A22F09D
:10F768000F02DA62186B074A02401A6300229A6095
:10F778004FF000638B60704700ED00E0001002401E
:10F788000CC07FF8CCFC00FF38B5094B93F8CC5778
:10F7980065B9084C2068F9F766FA074B25601B78AD
:10F7A800022B03D1BDE83840F6F7D3BA38BD00BF05
:10F7B80048200020802800207C280020044B93F853
:10F7C800CC371BB9034B1868FBF760BD00207047A6
:10F7D800482000208028002038B5054604462046E9
:10F7E80014F8011B21B1034B1868FBF75BFDF6E722
:10F7F800401B38BD802800200FB407B504AB06496C
:10F8080053F8042B01930020F7F736FA03B05DF89C
:10F8180004EB04B0704700BF8FF90008024B0146A3
:10F828001868FBF73FBD00BF80280020F8B5011F0E
:10F8380006460023083051F8042F02F120043F2C1B
:10F848003AD802F108040F2C06D80232032A04D948
:10F85800002B08BF012300E002238142EBD1012BDA
:10F8680030680ED0022B1AD0736803F003039B0094
:10F8780000F0030043EA0010B36803F003031843E1
:10F8880017E000F00F0040F04000FFF7C7FFB06836
:10F89800736800F00F0040EA0310C0B209E000F0FE
:10F8A8003F0040F08000FFF7B9FF3079FFF7B6FF5F
:10F8B800307ABDE8F840B1E706F10C0734463A461D
:10F8C800002552F8043D03F18001FF294FEA850520
:10F8D80010D903F50041B1F5803F02D245F001058A
:10F8E80008E003F50003B3F1807F34BF45F002055B
:10F8F80045F00305B242E4D165F03F00C0B2FFF71E
:10F908008DFF05F00303022B207807D0032B0CD0C2
:10F91800012B13D1FFF782FF60780FE0FFF77EFF1E
:10F928006078FFF77BFFA07808E0FFF777FF607843
:10F93800FFF774FFA078FFF771FFE0780434FFF752
:10F948006DFFBC424FEAA505DBD1F8BD10B50446F2
:10F95800C0B2FFF763FFC4F30720BDE810405DE7BE
:10F9680010B504467F2C06D964F07F00C0B2FFF7BB
:10F9780055FFE409F6E7E0B2BDE810404EE7430062
:10F9880083EAE070ECE7084648E700BF40F2E93355
:10F998000F4A1289920704D4013B9BB2002BF7D17E
:10F9A8000BE00C4A40F2E933107009490989C9078C
:10F9B8000AD4013B9BB2002BF7D1074A13880133C5
:10F9C8009BB21380FF2070471078C0B2704700BF09
:10F9D800003001400C300140D81F00200C4B0D496D
:10F9E800DA684378D243C2F30222C2F10402934098
:10F9F80002781B010A44DBB282F800330378012243
:10FA0800580903F01F0302FA03F341F82030704746
:10FA180000ED00E000E100E073B505460021006854
:10FA28000122FEF7EBFA2A6813889BB243F0010320
:10FA38001380EB7A8DF804300124002601A88DF894
:10FA480005408DF806608DF80740FFF7C7FFEB7A91
:10FA58001B2B0BD1192301A88DF804308DF8054014
:10FA68008DF806608DF80740FFF7B8FF02B070BD4B
:10FA7800F0B5BE4CA3782DED028B013B012B85B070
:10FA880000F26F81E578854240F06B812379022B83
:10FA980000F06781B64B5B5D6371A3796D00F2EE90
:10FAA800048A1BB16319B3F9083009E06319D4ED6E
:10FAB800037AB3F90830F1EE677AC4ED037A5B4252
:10FAC80008EE103A2369A94EB8EEC88A1A0388EEE0
:10FAD800288A35D5D6ED037AFDEEE77A28EE280A8E
:10FAE80017EE903AD6ED057A8DF80A30FDEEE77AF2
:10FAF80017EE903A8DF80B3004F01EFFFCEEC07A3A
:10FB080096ED060A17EE903A20EE280AADF808306E
:10FB180004F012FFFCEEC07A96ED070A17EE903A51
:10FB280020EE280AADF80C3004F006FFFCEEC07A8F
:10FB38000C2017EE903A02A9ADF80E30F7F7DCFE6C
:10FB4800D4ED077A894BF5EE407AF1EE10FA60D1E0
:10FB5800D3ED067AB4EEE78AF1EE10FA04DDDA683E
:10FB680083ED068A5A61E8E0F5EEC07AF1EE10FA04
:10FB780040F3E38093F8202042B1022A00F2DD80AE
:10FB88005A6B83ED078AFA329A63D6E0D3ED037A8B
:10FB980038EE678AF7EE007AB4EEE78AF1EE10FAEB
:10FBA800ACBF01210021D3ED0A7A69B19FED717ACA
:10FBB80027EE877ADFED707AB4EEE77AF1EE10FA85
:10FBC80058BFF0EE477A03E09FED6C7A67EE877ACC
:10FBD800C3ED0A7A2369654A1B0311D58DF808100D
:10FBE8005379116B0B440B205A788DF80920DA7A77
:10FBF8008DF80A205B7D8DF80B3002A9F7F77CFEA3
:10FC08000123226B84F82030637913440022DA72CE
:10FC180091E0B4EEE78AF1EE10FA48BF83ED078A67
:10FC2800A16B636B94ED067AD4ED076A591AC94340
:10FC3800C90F77EE667A59B9B7EE006AF4EEC67A5C
:10FC4800F1EE10FA79DDB4EEE68AF1EE10FA74DD21
:10FC5800D4ED056A454BB4EEE67AF1EE10FACCBF66
:10FC68000126002666B1D3ED097A9FED427A67EE48
:10FC7800877A9FED427AC3ED097AD3ED0B7A0AE0D1
:10FC8800B0EE007AF4EEC77AF1EE10FA08DDD3EDA3
:10FC98000B7A9FED387A67EE877AC3ED0B7A07E027
:10FCA800D3ED097A9FED357A67EE877AC3ED097A45
:10FCB800D4ED097A206B627967EEA87A1044FCEEDD
:10FCC800E77ACDED017A9DF804304370D4ED0B7AD4
:10FCD8002769FCEEE77A3F03CDED017A9DF8042011
:10FCE80042750ED546EA41018DF808108DF80930A5
:10FCF800C37A8DF80A300B2002A98DF80B20F7F78C
:10FD0800FBFD94F82020194B022A11D1D3ED0A7A71
:10FD18009FED1B7A196B67EE877A002283F8202003
:10FD2800FCEEE77A5A7917EE903A0A44D37202E069
:10FD3800022283F82020FCF7F9FAA2790B4B0AB1CA
:10FD4800104A00E0104ADA602544D4ED037AB5F988
:10FD5800083000EE103AB8EEC00A80EE280A37EEF6
:10FD6800C00A05B0BDEC028BF0BD00BFD81F002053
:10FD7800B47D0108EC51783F6F12833A0AD7833F6C
:10FD880000007A440000A0410000A0C12B4BF0B550
:10FD98002B4D1E6805F110002F78F3192C46597861
:10FDA80001F00401013501F0FF0219B18542F3D1D8
:10FDB8000020F0BD224D631B022B0ADD1AB102EBB5
:10FDC80082025200D2B215F8013B303B1A44D2B23B
:10FDD800F1E70021AC420AD919B101EB81014900D0
:10FDE800C9B215F8013B303B1944C9B2F2E72E2FCE
:10FDF80016D10134042000232578771903EB8303F7
:10FE08007F785B007F079BB244BF303D5B1900F1F0
:10FE1800FF3044BF01349BB210F0FF00ECD100E08A
:10FE2800002308484143642000FB03130620B3FB6A
:10FE3800F0F3054800FB0230F0BD00BF20010020B0
:10FE48001420002040420F008096980030B500230F
:10FE58001A4610498C1894F83C40BCB12E2C06D197
:10FE6800013298B18C180444002584F83C501144A0
:10FE78000A2491F83C106343A1F13004092C9CBF7B
:10FE8800303B5B180E2A03D80132E2E7184630BD32
:10FE9800002030BDD81F00200EB40FB507490190CF
:10FEA80006AB01A8064A0393F6F7E6FE019B00227B
:10FEB8001A7004B05DF804EB03B07047B16900082C
:10FEC800A88401080B4A136913F4805FB2F9523011
:10FED80006D0B2F80822111A8B4208DD104401E05E
:10FEE800B2F80A028342B4BF002001207047012003
:10FEF800704700BFD81F0020064B1B7803F004038F
:10FF080003F0FF001BB1044B1888C0F3C01000F0C9
:10FF180001007047FD2B0020981100202DE9F04FBB
:10FF28002DED028B87B000260493B24B0392B3F9F0
:10FF38000270B3F900300190002FB8BF7F42002B48
:10FF4800B8BF5B429F42B8BF1F46B7F5FA7F8146EC
:10FF5800A8BF4FF4FA77B0460296B3463446A64D8A
:10FF68002B8813F0030F4FEA440A58D0022C56D0BE
:10FF7800A04BA24A33F80A3032F90A20022113FBB7
:10FF88000122039B5B429A4203DB039B9342A8BF77
:10FF980013469B4A32F90A209B1A049A32F9142014
:10FFA800134408EE103AFFF7A7FF68B1B8EEC80A85
:10FFB800944BB2EE048A80EE080A185DFFF758FDEC
:10FFC80020EE080ABDEEC08A18EE102A99F808300B
:10FFD8005343642293FBF2F399F81C206FF0040B4F
:10FFE8000BFB02FB5B4504DB02EB820B9B45A8BFC6
:08FFF8009B46854918EE103A02
:020000040801F1
:1000000051F82420134442F210729342A8BF1346C1
:10001000804A9342B8BF134699F8122041F8243021
:1000200053431B1302932B8803F00302012A01D1CF
:10003000022C3FD17848714A30F90A0032F90A801F
:100040007649019A51F82460557880EAE07EAEEB5B
:10005000E07EBEF5206F4FEA84021EDC022C15D034
:1000600008EB8801090191FBF5F5042190FBF1F003
:100070002D1A2E44B6F57A5F68496948A8BF4FF437
:100080007A568642ACBF5650505008E088EAE87E67
:10009000AEEBE87EBEF1640FE2DD002088505F49E0
:1000A0007D26525892FBF6F6019AD27A7243402688
:1000B00092FBF6F69A0713D5022C11D00298C7F5D9
:1000C000FA7307FB06F507FB08F203FB0B224FF45C
:1000D000FA7103FB005392FBF1F293FBF1F508E098
:1000E000DB0704D5022C02D0029D5A4601E03546BA
:1000F0004246494B33F91410042391FBF3F3494969
:10010000615C4B436FF04F0193FBF1F399F8511091
:10011000D3184FEA440A08EE103AB1B1022CB8EEF7
:10012000C80A414B08D14A0803D09142A8BF1146E2
:1001300000E001213D4802E03D4800EBC400D3ED62
:10014000000AF6F76BFCBDEEC08A334B394A3AF829
:1001500003003AF902302AF8020001B202F1080065
:100160001432CB1A50F824E0042193FBF1F152F839
:10017000243040F8241073440B4499F8501042F88E
:1001800024E04FEA840C00EE103A79B1264B2A485D
:10019000D3ED000ACDF814C0B8EEC00A00EBC400DD
:1001A000F6F73CFCDDF814C0BDEEC00A234A244932
:1001B000125D10EE103A5343202293FBF2F318EE37
:1001C000102A2A44D21A2AF801201E4A18EE101AC0
:1001D0004CF802101C4A4CF802501C4A5B424CF886
:1001E0000230019B01340133032C01937FF4BBAE39
:1001F00007B0BDEC028BBDE8F08F00BFB41000204B
:1002000098110020F62B0020E01F0020486901080B
:1002100024140020F0D8FFFF04100020B0130020A9
:1002200080C1FFFF2C140020AC130020A413002079
:10023000941300201C280020E01300204414002008
:10024000F8130020001400200C14002018140020C3
:100250002DE9F04F2DED088BC94F83B00446009374
:100260003B88019713F0020F0AEE102AF7EE009A6E
:100270004CD0149BC348DD89B0F900305B1B03F2FE
:10028000F31640F2E632964203D8002BB8BF5B4229
:1002900001E04FF4FA73B0F90220521B02F2F31599
:1002A00040F2E630854203D8002AB8BF524201E04E
:1002B0004FF4FA7294F84C0058B39342B8BF134607
:1002C000C3F5FA7307EE903A9FEDAF7AF8EEE77A4E
:1002D0006423C7EE877A93FBF0F307EE103A77EECC
:1002E000E97AB8EEC77AB0EE699AA7EE879AF7EE88
:1002F000006AB5EEC09AF1EE10FA0AD4B4EE669A2E
:10030000F1EE10FAC8BFB0EE669A04E0B0EE699A5A
:1003100001E09FED9E9ACE1C25464FF0000ABAF1EF
:10032000020F16F801BF9A4F4FEA4A09F2EE04AAEB
:100330000ED1B7F904209FED977A0BF10A0B02FB5F
:100340000BF307EE903AF8EEE77AC7EE877A68E0AB
:10035000F8EE4A7A9FED8C6A37F91A30C7EE867A42
:1003600006EE903A8C4B33F91A3007EE103A1AEE3B
:10037000103AF8EEE66AB8EEC77A5B42A6EEA77AC4
:1003800007EE903AF8EEE77AB4EEE77AF1EE10FA7B
:1003900008D4F8EECA7AB4EEE77AF1EE10FAD8BFD4
:1003A000F0EE477A7D4B33F9093008EE103A009BA6
:1003B000B8EEC88A33F91A3077EEC87A08EE103AE8
:1003C000B8EEC88A37EE888A88EE2A8AFFF798FD49
:1003D00040B1734B13F80A00B0EE480AFFF74CFB2C
:1003E000B0EE408A019B1A88D10704D5D4ED117A6A
:1003F00068EE277A15E037F909309FED667A0BF140
:10040000140B03FB0BF307EE903AF8EEE77A930731
:10041000C7EE877A42BF94ED127A28EE078AE8EE9B
:10042000097A604BDFF8ACB133F9093095ED08BAC1
:100430009FED5D8A94F85110DFF89C8107EE103A29
:100440005A4BB8EEC77AD3ED0C6A1AF80B30E7EEC8
:10045000667AF0EE48BAF0EE678A67EE8B7A0BEEBA
:10046000103AB8EECBBA27EE8BBA8BEE08BAC1B110
:10047000BAF1020F0AD14B0803D09942A8BF19461E
:1004800000E00121B0EE4B0A494804E04948B0EED3
:100490004B0A00EBCA00D8ED000AF6F7BFFAB0EE3F
:1004A00040BAD8ED000A444995ED0B7A4FEA8A0725
:1004B00068EEA07A394467EE877A91ED007AA7EE6C
:1004C000AA7ADFED3E7AB4EEE77AF1EE10FAF0EEBA
:1004D00047AA09D4DFED3A7AB4EE677AF1EE10FA62
:1004E000C8BFF0EE67AA01E0F0EE67AA89EEA07A35
:1004F000344AC1ED00AAD119D1ED007AC1ED008ACC
:1005000078EEE77A02F10C013944183267EE877A07
:100510003A4491ED007A92ED000AC1ED007A82ED45
:10052000007A37EE000A94F8501030EE270A21B115
:10053000254800EBCA00F6F771FAF0EE087A80EE73
:10054000270A1BF80A30D5ED0E7A08EE103A60EE55
:10055000277AB8EEC88A27EE880ADFED1C7A80EE8B
:100560002B8AB4EEE78AF1EE10FA37D4DFED187A71
:10057000B4EE678AF1EE10FAC8BFB0EE678A2FE0DA
:1005800098110020242000200000FA430000000001
:10059000B410002000004842F62B0020E01F00208D
:1005A00048690108041000200000C8421C280020EF
:1005B000A4130020941300206C14002000007AC3C0
:1005C00000007A4350280020E0130020000096C36A
:1005D0000000964390130020AC130020B0EE678A11
:1005E0003BEE2A0A0AF1010A30EE080A04F062F929
:1005F000144AB0F57A7FA8BF4FF47A709042B8BF22
:100600001046BDEECBBA104A1BEE103A22F8090094
:10061000FDEEEAAA0D4ABDEEC88ABB500C4A1AEE9E
:10062000903ABB500B4A18EE103ABAF1030FBB5088
:1006300005F104057FF473AE03B0BDEC088BBDE893
:10064000F08F00BF18FCFFFFF813002000140020FB
:100650000C14002018140020044B00221A605A6069
:10066000034B00221A605A60704700BF2414002018
:10067000781400202DE9F04FAC490B7813F0010FEE
:1006800087B003F0040200F04881002A40F0748132
:1006900003F0020000F0FF04002840F03E8143F028
:1006A00004030B70A24B1A88A24B1A80A24B1A6843
:1006B00012F4002F984600F01181A04B80201C708E
:1006C000F5F74AFC08B1FEF7DFFA9D4C2778012FB9
:1006D00040F004819B4D95F8CA2722B195F8CB379D
:1006E0000BB19A4203D3012385F8CA370FE01846AD
:1006F000114630B191FBF0F600FB1616014630466C
:10070000F7E792FBF1F285F8CA2793FBF1F385F83E
:10071000CB3795F8CC371BB18A4B002283F8CC2716
:10072000636895F8CC6703EBC30341F66902934213
:1007300084BF40F2E242B3FBF2F3834A8CBFDBB2E8
:1007400004231370FEB98020FAF7C8FA8146D0B1AD
:100750008021FAF79FFA99F806207C4B207253F813
:10076000223099F90000DFF8D891B3F5613F0CBF52
:100770000222002202218DE8060080213246FAF78B
:10078000A6FBE06008B90023A7E009F1100031469C
:10079000142203F080FE09F13003C9F8243009F176
:1007A000A003C9F8283009F58873C9F82C30684BC4
:1007B000D8F800201B88A9F8803195F89431654855
:1007C00095F886910590002B634B1B68C3F3C00E10
:1007D0006B79A3F1190B02F4006CC2F3400AC2F367
:1007E000C03218BF0122DBF1000141EB0B01012BEC
:1007F00014BF0B46012395F8CAB7049395F8CB377D
:1008000005689B45554B1B7803932CBF4FF0000B9D
:100810004FF0010B791EC9B24B1E132B39D8DFE8FC
:1008200003F00C0C0C0C0C0C0C0C0A833BA7273BA4
:1008300033121212353B049B9BE0039B8B42B4BFE7
:100840000023012324E02B78022B0BD105EB81033D
:1008500053ED027AF5EE407AF1EE10FA14BF01235F
:10086000002315E06B185B79003318BF01230FE0FC
:10087000BCF1000F04D009F1FF304342434100E0D6
:10088000634603F0010374E0134672E05B4670E0D8
:1008900013B101238B401E43142F02D80137FFB23E
:1008A000B8E7059BC4F88461186819217930FAF714
:1008B000A5FA0023C4F88C31A4F89031A4F8923141
:1008C000C4F89C31264BD4F898211B68C4F8A03199
:1008D00084F88801C4F8942102232370204B194A1C
:1008E0001B6892F8DE214FF47A7101FB02331D4A36
:1008F0001360D8F800301A0609D51B4B1B789B07EC
:1009000005D51A4B1B78042B01D9062000E00520E1
:1009100007B0BDE8F04FFAF745BC6ABB012007B04D
:10092000BDE8F04FFAF764BC734622E0FD2B0020CF
:10093000B01000200A0F0020E81F00204D120020F8
:1009400074280020482000201C010020E8630108D2
:10095000C012002020100020D010002060150020C0
:100960000C200020BC0E0020D4100020DA10002043
:100970005346002B8DD191E707B0BDE8F08F10B53D
:10098000154A1378590725D523F004031370134B28
:100990001B681B0319D5124C2378A3F10802012A06
:1009A0000BD8FF200021F6F7ABFF0E4B1B68C4F8F5
:1009B000A031FEF707FF0A2306E0012B05D90A2B19
:1009C00003D0FEF7E5FE012323700420BDE81040AC
:1009D000FAF7E8BB10BD00BFFD2B0020E81F002088
:1009E000742800200C200020034B1A78202A04BF12
:1009F00000221A70704700BF002C0020014B042217
:100A00001A607047E42B0020034B9B7A13B1034B11
:100A100005221A60704700BFFC140020E42B002060
:100A20000D4B0E491A680E4B92B213445B000D4AEF
:100A30001B68C3F3090310B5136013689BB201333D
:100A40005B1000229A4206D0074851F8044B20F868
:100A500012400132F6E710BD505C004020620040B9
:100A60001E3000200C17002011170020014B00221F
:100A70001A607047081700202DE9F843664B674E4F
:100A80001B68DFF8B881664A00254FF0C0099D72E7
:100A900083F80990DD723560D8F8003023F4EC4318
:100AA00023F0700343F400739BB2C8F80030D8F809
:100AB000003023F4E04323F040039BB248F280046B
:100AC00083F010032343C8F80030336812FA83F32D
:100AD0005B0040271A681F6033689BB203F1005324
:100AE00003F540535B0028461A6880221A60D8F844
:100AF000003023F4F8731B051B0D2343C8F80030A6
:100B0000484B93F82C10F5F7EFFAD8F80030464A26
:100B1000464923F4804323F070039BB283F440538F
:100B20002343C8F80030136823F4EC4323F0700328
:100B30009BB21360336811FA83F35B0003201968DA
:100B4000C3F8009013683A4923F4E04323F04003CC
:100B50009BB283F0200323431360136823F4804384
:100B600023F0700323439BB21360536823F4EC43D8
:100B700023F0700343F4C0639BB25360336811FAEF
:100B800083F35B0019684FF480711960536823F494
:100B9000804323F0700323439BB25360536823F4D4
:100BA000E04323F040039BB283F0200323435360D0
:100BB000D8F80C301F4A23F4EC4323F070039BB2A7
:100BC000C8F80C30336812FA83F35B0039461A68B0
:100BD0004FF488721A60F5F787FAD8F80C3023F4CE
:100BE000804323F070039BB283F440532343C8F83F
:100BF0000C30D8F80C3023F4E04323F040031C43BE
:100C0000A4B2C8F80C402846F5F7E2F90A4B0122D5
:100C10001A60BDE8F88300BFA4110020505C0040BA
:100C2000043000201C000020045C0040083000203C
:100C3000103000201C300020E42B0020005C00401D
:100C4000134A144B50681B68181810B5146808D064
:100C500011490822F8F7A7FD204610490422F8F7A9
:100C6000A2FD0F4B1A68002393720E4A01211160F6
:100C70000D4913604FF4E0500B6010600B480B609F
:100C80004FF4364101801160094A136010BD00BF66
:100C9000B0F7FF1FACF7FF1FEE000020FE000020A2
:100CA000A4110020405C0040445C00401C2A00204D
:100CB000E42B0020024B4FF480221A60704700BFE3
:100CC0001404014003788B4286BF024B33F81100B5
:100CD00000207047202A002070B5002213462349C7
:100CE00014180C44247E83EA0423082413F4004FD0
:100CF0004FEA430318BF83F4815304F1FF3418BF54
:100D000083F0010314F0FF049BB2EFD10132192AE2
:100D1000E5D100F1190200F11A050A440D44167ECE
:100D20002A7E02EB062292B29A421ED10F4B93F812
:100D30003950E2B2AA4215D2431C03EB4203DBB2A4
:100D4000CA1801330B44127E1B7E03EB02239BB2B5
:100D50004FF4AF6253431B1303F5487321F814306B
:100D60000134E6E7012381F83A3070BD202A0020E3
:100D700003788B420BD9074B1A78074B890019442B
:100D8000C86B02B1400800F5777080B27047002050
:100D9000704700BF4C120020202A002007299DBF69
:100DA000034B03EB8101B1F86C000020704700BFDA
:100DB000202A0020034B03EB4101B1F88C00C0084E
:100DC000704700BF202A00200A4BDFED0B7A03EBAF
:100DD000810191ED2B7AB8EE477AF6EE046AE7EEE0
:100DE000267A82B0FCEEE77ACDED017ABDF80400F8
:100DF00002B07047202A002000005C44014B33F809
:100E00001100704724200020024B03EB4101B1F890
:100E1000F4007047202A0020024B03EB4101B1F897
:100E2000F4007047202A00200020704770B5334C32
:100E30000546FAF71DF8D4F80C31C4F80C01C31AB2
:100E4000B3F5FA5FC4F8103182BF002384F814317F
:100E500084F8153194F814312BB9A12D02BF274A1B
:100E6000012182F8151194F81511244A29B1D118DD
:100E7000EDB201330D7682F8143194F8145194F8E0
:100E80001631AB4239D11D4B93F81731052B02D0E7
:100E9000062B03D02CE00020FFF71EFF637E1E2BE5
:100EA00026D100200246C1B26B1E994219DA2144B4
:100EB0000B7E0821DBB283EA0206F60744BF83F00B
:100EC0001803C3F3460301F1FF3154BF5B0843F03D
:100ED000800311F0FF01C2F34702ECD101301A4642
:100EE000E1E723441B7E9A4202D10320FFF7F4FE80
:100EF000002384F8153184F8143170BD202A0020B5
:100F000010B50446F9F7B4FF0F4BD3F81821C3F816
:100F10001801821A41F288318A42C3F81C2184BF29
:100F2000002283F8202193F82021074913440F2A37
:100F3000E4B218BF013283F8214112BF81F82021A9
:100F4000012381F8313110BD202A002010B504465C
:100F5000F9F78EFF0F4BD3F83421C3F83401821A0E
:100F600041F288318A42C3F8382184BF002283F8D5
:100F70003C2193F83C2107491344142A18BF01323D
:100F800083F83D4112BF81F83C21012381F85231A1
:100F900010BD00BF202A002038B50446F9F768FFCD
:100FA000274A2749D2F85431C2F85401C31AB3F57D
:100FB0007A6F84BF002382F8583192F8583133B9E0
:100FC000A82C3BD181F85931A1F85A3106E0022B07
:100FD00002D181F85C4101E0242B02D8D11881F8BC
:100FE0005D4192F85C11164D01330231DBB24900CC
:100FF0008B4282F8583118DAB5F85A31E0B283EAF8
:101000000020082310F4004F4FEA400018BF80F47E
:10101000815003F1FF3318BF80F0010013F0FF038C
:1010200080B2EFD1A2F85A0138BD01318B4201BF25
:10103000002385F85831012385F8593138BD00BFA8
:10104000202A002010B50446F9F712FF104AD2F802
:10105000843140F6AC51C31A8B42C4BF002382F8DE
:10106000883192F88831D11881F8894123B90F2C41
:101070000DD10749C1F884010133DBB2192B0449B2
:1010800082F888310CBF0123002381F8A23110BD02
:10109000202A0020094B1A68137844F6FB7103EBF1
:1010A000431300FB03135078C0EB0030B3FBF0F3A5
:1010B0009078B3FBF0F080B2704700BFBC10002006
:1010C000114BD3F8A43103EB4002117E01290DD05E
:1010D00002290FD0022805D9032807D10B4A12682C
:1010E000D20401D5D8897047988A7047084B33F8E5
:1010F00010007047507E00EB800000EB800000F293
:10110000EE2080B2704700BF202A0020E81F002098
:1011100024200020044B1B6842F201021A420CBF3B
:1011200001200020704700BFE81F0020114B93F8FA
:10113000A821012A10B51C460ED008D3022A0FD1CF
:101140000D4A938A9BB283F48853938208E00A4B3A
:101150004FF488521A8503E0074B4FF488529A6186
:10116000F9F786FE00F5F42000F59070C4F8AC01A4
:1011700010BD00BF202A002000100048022803D024
:10118000431E584258417047064B1B681B7823B1D9
:10119000054B1868C0F3C0407047044B1878C0F383
:1011A000800070475C060020E40F0020FD2B00202B
:1011B00010B50A4C5E280146206805D15D21FAF77A
:1011C00075F820683E2105E05D2903D1FAF76EF835
:1011D00020683D21BDE81040FAF768B8D02B002008
:1011E00030B50028104C114AB8BF40423C2590FB56
:1011F000F2F304FB030068430D4D90FBF2F22D68FF
:101200002D7B25B903EB830303EB830301E0C3EBE1
:10121000031302EB83030B8004FB02024FF47A7387
:1012200092FBF3F24A8030BD806967FF8096980098
:10123000C410002010B50446C0B2FFF7B9FFC4F3D4
:101240000720BDE81040B3E7024B5E211868FAF7AB
:101250002DB800BFD02B002038B5064C05465E21C6
:101260002068FAF723F820682946BDE83840FAF7E5
:101270001DB800BFD02B0020674B73B51878674DA1
:10128000FFF77CFF2B788342044620D0C8B1644B23
:101290001B68E3B193F9000002230093614B1B68C4
:1012A0005B78003318BF0123019304214FF41653D8
:1012B0000022F9F70CFE5C4B186040B101232B7043
:1012C00005E0594E3068F7F7D2FC34602C70574B6C
:1012D000574D1878FFF752FF2B788342044618D0F9
:1012E00088B1544B1B68A3B10022012493F900007C
:1012F00000944FF4964301920821F9F7E8FD4E4B14
:10130000186028B905E04C4E3068F7F7B0FC34603F
:101310002C704A4B4A4D1878FFF730FF2B788342E8
:1013200004462E4642D0002837D0464B1A68002A81
:101330003CD0D37992F90000434C002B08BF022324
:1013400002220092002254F8233001921021F9F772
:10135000BEFD3E4B0546186040B33D4C94F84A3004
:10136000022B0BD094F89620022A01D14C3405E0D0
:1013700023B1002A04F14C0418BF0024354B1C6033
:1013800044B1204600214C2203F085F80223256059
:1013900084F84A300123337008E02C4E3068FDF7A2
:1013A00073FC3068F7F763FC34602C702A4B2B4DCC
:1013B0001878FFF7E3FE2B788342044629D000B368
:1013C000274B1B682BB3274A93F900001268527809
:1013D000002A0CBF082209220323009301924FF434
:1013E000614320210022F9F772FD1F4B186080B184
:1013F0001E4A012313702B701D4B1A681D4B1A6077
:1014000007E0194E3068F7F732FC184B34601C7057
:101410002C7002B070BD00BF64060020A010002038
:1014200060060020C4100020D02B0020650600209C
:10143000E4100020681100205811002070060020E0
:101440006E1100206C060020E86301087011002076
:10145000AC110020741100207C06002084110020B3
:101460007806002074060020881100208C110020CE
:101470000C2000209011002008B5044B1B7803F0CD
:101480000503052B01D1FAF771F8FEE7D42B0020F4
:10149000D0400B1C1141203A03D49C461341184301
:1014A0006346524293401843704700BF7BB972B9FC
:1014B0000029BEBF00204FF0004106E008BF002811
:1014C0001CBF6FF000414FF0FF3000F073B882B0E6
:1014D000EC462DE9005000F03DF8DDF804E002B0E4
:1014E0000CBC704707EE900AF5EEC07AF1EE10FAE8
:1014F00001D400F009B808B580F0004000F004F80D
:10150000404261EB410108BDD0B500F0B9F90022BD
:101510000E4B06460F4600F007FA00F017FC044693
:1015200000F08CF900220A4B00F0FEF902460B464F
:101530003046394600F044F800F008FC234600220B
:1015400042EA000210461946D0BD00BF0000F03D3F
:101550000000F0412DE9F041069C154606460F4675
:10156000984600F013FC05FB01F300FB0838A5FBCF
:101570000023B21A434467EB0303C4E90023BDE828
:10158000F08100BF2DE9F041069C904606460F46CB
:101590001D4600F049FD00FB05F5A0FB082308FBF4
:1015A0000155B21A2B4467EB0303C4E90023BDE8DD
:1015B000F08100BF704700BF81F0004102E000BF32
:1015C00083F0004330B54FEA41044FEA430594EA03
:1015D000050F08BF90EA020F1FBF54EA000C55EA3E
:1015E000020C7FEA645C7FEA655C00F0E2804FEA0F
:1015F0005454D4EB5555B8BF6D420CDD2C4480EAF1
:10160000020281EA030382EA000083EA010180EA20
:10161000020281EA0303362D88BF30BD11F0004F6E
:101620004FEA01314FF4801C4CEA113102D04042A4
:1016300061EB410113F0004F4FEA03334CEA1333DF
:1016400002D0524263EB430394EA050F00F0A780F7
:10165000A4F10104D5F1200E0DDB02FA0EFC22FAF2
:1016600005F2801841F1000103FA0EF2801843FAE6
:1016700005F359410EE0A5F120050EF1200E012AD7
:1016800003FA0EFC28BF4CF0020C43FA05F3C01815
:1016900051EBE37101F0004507D54FF0000EDCF18E
:1016A000000C7EEB00006EEB0101B1F5801F1BD337
:1016B000B1F5001F0CD349085FEA30004FEA3C0C3B
:1016C00004F101044FEA445212F5800F80F09A8031
:1016D000BCF1004F08BF5FEA500C50F1000041EB35
:1016E000045141EA050130BD5FEA4C0C404141EB39
:1016F000010111F4801FA4F10104E9D191F0000F60
:1017000004BF01460020B1FA81F308BF2033A3F1E2
:101710000B03B3F120020CDA0C3208DD02F1140CD9
:10172000C2F10C0201FA0CF021FA02F10CE002F114
:101730001402D8BFC2F1200C01FA02F120FA0CFC0D
:10174000DCBF41EA0C019040E41AA2BF01EB045156
:10175000294330BD6FEA04041F3C1CDA0C340EDC54
:1017600004F11404C4F1200220FA04F001FA02F397
:1017700040EA030021FA04F345EA030130BDC4F155
:101780000C04C4F1200220FA02F001FA04F340EA4A
:101790000300294630BD21FA04F0294630BD94F0FB
:1017A000000F83F4801306BF81F480110134013DE2
:1017B0004EE77FEA645C18BF7FEA655C29D094EA53
:1017C000050F08BF90EA020F05D054EA000C04BFD1
:1017D0001946104630BD91EA030F1EBF00210020BC
:1017E00030BD5FEA545C05D14000494128BF41F05B
:1017F000004130BD14F580043CBF01F5801130BDBF
:1018000001F0004545F0FE4141F470014FF0000049
:1018100030BD7FEA645C1ABF194610467FEA655CFA
:101820001CBF0B46024650EA013406BF52EA03359C
:1018300091EA030F41F4002130BD00BF90F0000F8A
:1018400004BF0021704730B54FF4806404F13204C6
:101850004FF000054FF0000150E700BF90F0000F7F
:1018600004BF0021704730B54FF4806404F13204A6
:1018700010F0004548BF40424FF000013EE700BF76
:1018800042004FEAE2014FEA31014FEA02701FBF06
:1018900012F07F4393F07F4F81F06051704792F0D8
:1018A000000F14BF93F07F4F704730B54FF4607452
:1018B00001F0004521F0004120E700BF50EA01029D
:1018C00008BF704730B54FF000050AE050EA01024A
:1018D00008BF704730B511F0004502D5404261EBBA
:1018E00041014FF4806404F132045FEA915C3FF4FB
:1018F000DCAE4FF003025FEADC0C18BF03325FEA94
:10190000DC0C18BF033202EBDC02C2F1200300FA48
:1019100003FC20FA02F001FA03FE40EA0E0021FA6D
:1019200002F11444C1E600BF70B54FF0FF0C4CF457
:10193000E06C1CEA11541DBF1CEA135594EA0C0F0D
:1019400095EA0C0F00F0DEF82C4481EA030621EA48
:101950004C5123EA4C5350EA013518BF52EA033583
:1019600041F4801143F4801338D0A0FB02CE4FF035
:101970000005E1FB02E506F00042E0FB03E54FF065
:101980000006E1FB03569CF0000F18BF4EF0010E5D
:10199000A4F1FF04B6F5007F64F5407404D25FEA59
:1019A0004E0E6D4146EB060642EAC62141EA55510C
:1019B0004FEAC52040EA5E504FEACE2EB4F1FD0C4E
:1019C00088BFBCF5E06F1ED8BEF1004F08BF5FEACC
:1019D000500E50F1000041EB045170BD06F000467E
:1019E00046EA010140EA020081EA0301B4EB5C042B
:1019F000C2BFD4EB0C0541EA045170BD41F4801123
:101A00004FF0000E013C00F3AB8014F1360FDEBF47
:101A1000002001F0004170BDC4F10004203C35DA23
:101A20000C341BDC04F11404C4F1200500FA05F3A6
:101A300020FA04F001FA05F240EA020001F0004247
:101A400021F0004110EBD37021FA04F642EB0601BD
:101A50005EEA430E08BF20EAD37070BDC4F10C04E7
:101A6000C4F1200500FA04F320FA05F001FA04F2AB
:101A700040EA020001F0004110EBD37041F1000197
:101A80005EEA430E08BF20EAD37070BDC4F12005A2
:101A900000FA05F24EEA020E20FA04F301FA05F20A
:101AA00043EA020321FA04F001F0004121FA04F2B2
:101AB00020EA020000EBD3705EEA430E08BF20EA82
:101AC000D37070BD94F0000F0FD101F000464000BC
:101AD00041EB010111F4801F08BF013CF7D041EA3E
:101AE000060195F0000F18BF704703F00046520042
:101AF00043EB030313F4801F08BF013DF7D043EA13
:101B00000603704794EA0C0F0CEA135518BF95EAC8
:101B10000C0F0CD050EA410618BF52EA4306D1D14F
:101B200081EA030101F000414FF0000070BD50EA6E
:101B3000410606BF1046194652EA430619D094EAF8
:101B40000C0F02D150EA013613D195EA0C0F05D1E2
:101B500052EA03361CBF104619460AD181EA030136
:101B600001F0004141F0FE4141F470014FF00000EE
:101B700070BD41F0FE4141F4780170BD70B54FF089
:101B8000FF0C4CF4E06C1CEA11541DBF1CEA135509
:101B900094EA0C0F95EA0C0F00F0A7F8A4EB0504EB
:101BA00081EA030E52EA03354FEA013100F08880E2
:101BB0004FEA03334FF0805545EA131343EA1263AB
:101BC0004FEA022245EA111545EA10654FEA002660
:101BD0000EF000419D4208BF964244F1FD0404F519
:101BE000407402D25B084FEA3202B61A65EB030575
:101BF0005B084FEA32024FF480104FF4002CB6EB32
